:020000040800F2
:100000000002002029050008C5040008810400083A
:10001000D5040008E5040008F5040008000000000D
:10002000000000000000000000000000450400087F
:100030000505000800000000290400081505000857
:100040008901000889010008890100088901000868
:10005000890100088901000899160008991600080E
:1000600099160008991600089916000889010008D9
:100070008901000889010008890100088901000838
:100080008901000889010008890100088901000828
:1000900089010008890100088901000899160008F3
:1000A0008901000889010008890100088901000808
:1000B0003118000889010008890100088901000839
:1000C00089010008890100088901000889010008E8
:1000D0008901000889010008491200084F12000830
:1000E00099160008890100088901000889010008A3
:1000F00089010008890100088901000889010008B8
:1001000089010008890100083718000889010008E2
:100110008901000889010008890100088901000897
:100120008901000889010008890100088901000887
:100130008901000889010008890100088901000877
:100140008901000889010008890100088901000867
:100150008901000889010008890100088901000857
:100160008901000889010008890100088901000847
:1001700089010008890100088901000800000000C9
:10018000000000008901000800F0C4B900F004BBC1
:100190007047000070B50C46064600F061F9094B47
:1001A000094A1D682919914202D8084A914204D28D
:1001B0000C2333604FF0FF3500E0196000F058F970
:1001C000284670BD0002002000000220C45100201B
:1001D0001946104600F0ECBA1946104600F0F0BA85
:1001E000132303604FF0FF307047132303604FF079
:1001F000FF307047132303604FF0FF307047022930
:100200004FF0000303608CBF002001207047000006
:10021000114B70B500241C60104B114D18682E68EE
:1002200000F09CF80F4B53F820301B68A3F1080234
:1002300096420FD026B13179092904BF0A213171C4
:10024000092103F8041C33F9021C074B2A601980AA
:10025000012070BD204670BDD0020020A403002004
:10026000D8020020E0020020D4020020082930B586
:10027000037919D9082B32D842791A4B53F82250F6
:1002800000F108042DB12D68856053F822502C60D0
:1002900000E0846043F82240134C4279012303FAC2
:1002A00002F22368134319E0082B18D945790D4B46
:1002B00053F825203AB11468A2420BBF00222468EB
:1002C00043F825201460427953F822303BB9064C9C
:1002D000012303FA02F2236823EA02032360017177
:1002E00030BD00BFE0020020A403002008B50A4B87
:1002F0001B681A79082A02D95B7983420AD900F06F
:10030000BAF818B1054B01221A6008BDBDE80840D3
:1003100000F082B808BD00BFD8020020D002002043
:1003200008B500F09DF8094B094A1B88094D1BB21E
:10033000002442F82340084A286813682146013BFC
:100340001360FFF793FF2C6000F062F8D4020020E6
:1003500020030020D8020020DC0200200023C20776
:1003600002D440080133FAE718467047134423F0DB
:10037000030310B54FF077321C1F43F8042C6207BB
:1003800042BF4FF0883243F8082CA3F108044FF025
:10039000807304E909000F4B44F80C3C002344F837
:1003A000103C032344F8143C2246022344F8183C32
:1003B000012344F81C3C42F8201D0B2342F8043D65
:1003C000013B032BFAD120466FF0020340F8443D75
:1003D00010BD00BF21030008064B0749074A1868F3
:1003E000884203D1934201D20433F8E70348C01A8C
:1003F000704700BF00000020FEE7FEE7000200207B
:10040000EFF30880704700000048704700000020AC
:1004100000F02AF801DFFEE7024A536843F08053F8
:100420005360704700ED00E0EFF3098020E9F00F22
:1004300040F804ED02490968086000F003F8000084
:10044000D8020020FFF7E4FE04480068016801C9F3
:10045000B1E8F00F81F3098800470000D8020020BE
:10046000EFF3108072B6704762B6EFF310807047FA
:1004700080F310887047EFF30580C0B2704700002A
:100480000D490E4A0E4B6846904203D8984201D956
:10049000002102E009468D460121042072460242F5
:1004A00002D1EFF3088001E0EFF309802DE9F00FAE
:1004B0006B4600F06FF800BF000200200000022031
:1004C0006005002008B50249042000F08DFB00BF44
:1004D0004C05010808B50249062000F085FB00BF65
:1004E0005805010808B50249072000F07DFB00BF50
:1004F0006B05010808B50249082000F075FB00BF34
:100500007D05010808B50249092000F06DFB00BF18
:100510009105010808B502490A2000F065FB00BFFB
:10052000A30501087047704708B5FFF7FBFF6A464F
:10053000114B1249934202D243F8041BFAE7104AC6
:10054000104B11498B4204D252F8040F43F8040BAC
:10055000F8E70E4B0E4A0021934202D243F8041BE7
:10056000FAE7FFF7E0FF00F01FFB0EF0D3F8BDE85D
:10057000084000F073BB00BF00000020FEE7FEE76C
:100580008C40010800020020CC020020D002002094
:10059000C45100202DE9F04F9A46494B8FB0934645
:1005A0009A6B03925A6B04929F6ADA6A05921A6BED
:1005B000DB6B0793434B06921A68434B9A420446FF
:1005C000884602D041480EF08FFBB8F1000F05D0ED
:1005D0003F4800250EF088FB2E4626E094E80E00EA
:1005E000E068D4F81C9008902069099060690A902E
:1005F00019F4007F3748A6690D930CBF04F120055C
:1006000004F124050C920B910EF06EFB089B0093F5
:100610000BA90EC930480EF0DDFACDF80090334634
:100620000A9A09992D480EF0D5FA2D480EF05CFB78
:1006300039462C480EF0CEFA05992B480EF0CAFA2E
:1006400006992A480EF0C6FA079929480EF0C2FA10
:100650003A0403D5039927480EF0BCFA3B0603D5AC
:10066000049925480EF0B6FA24480EF03DFB594691
:1006700023480EF0AFFAB8F1000F1BD121480EF05D
:1006800033FB314620480EF0A5FA69461F4BC91AC4
:1006900003D549421E480EF09DFA20468268C36881
:1006A00001698C4641698E46AD46514691E8F00F8E
:1006B0004168006801BE1749052000F095FA00BFA7
:1006C00000ED00E000000020FEE7FEE7B1050108B4
:1006D000C7050108F6050108110601084E060108C4
:1006E0008C06010895060108A5060108B506010853
:1006F000C5060108D5060108E5060108F50601084A
:10070000FA0601080C0701083D07010858010020FE
:10071000650701089207010810B568B1012815D1D5
:10072000174A136823F003031360136843F400733C
:1007300043F0010313601BE0114B1A6842F00E02F4
:100740001A605A6842F480725A6011E00D4A1369C7
:1007500023F0040313610024FFF782FEBFF34F8FE1
:1007600030BFFFF785FE54B1BDE8104000F010BC6B
:10077000044A136943F0040313610124ECE710BD3C
:100780000070004000ED00E008B5FFF769FE0020B2
:10079000BDE80840FFF7C0BF034B044A4FF4E13106
:1007A000002000F0C7BC00BF04020020270E000894
:1007B0000A460146014800F041BB00BF0402002088
:1007C00010B50A460C460146002000F019FD2046EF
:1007D00010BD002000F0D6BF034B1968024611B9C6
:1007E000084600F0AFBF7047EC03002010B5094A7F
:1007F00013685BB19C6881688C4202D21A461B6800
:10080000F7E703D15C6841688C42F7D90360106058
:1008100010BD00BFF8030020F0B51F4E1F4D336818
:100820001F4C013333601F4B00201A6818602B687F
:10083000226019460746B64641B1DEF800C08E6810
:10084000664503D80F4601200968F5E700B1296025
:1008500007B9F0BD00213960E2B133B15168586881
:10086000814294BF1146194600E0114608461268BD
:100870001B680AB903600BE00BB9026008E0556819
:100880005E68B54294BF15461D4605602846EEE7F2
:100890002160F0BD2360F0BDF0030020F8030020CC
:1008A000F4030020E80300202DE9F0412E4F2F4CE7
:1008B00001233B6023683BB9FFF7AEFFFFF789FFD9
:1008C0000130FBD0002502E0FFF783FF05464FF023
:1008D0000008236823B9FFF77CFF854214D91AE08A
:1008E0005E68FFF776FF854208D923685E68FFF7E8
:1008F00070FFA8422CD3B042F7D329E08642F4D946
:10090000361A132EE7D8F0E7236843B9FFF761FFE3
:10091000854206460BD9FFF77FFF0025D9E75E68C1
:10092000FFF757FF063E14308642D2D309E010F19C
:10093000140F04D3FFF74DFF8642FBD9EBE74FF0CE
:10094000FF3600233B603046BDE8F041FFF744BF6F
:1009500023681A682260C3F80480C3F80880DA6844
:1009600018699047B5E700BFEC030020F4030020AE
:10097000144B1A6882420AD112681A6012B1506888
:10098000063801E04FF0FF30FFF726BF13461A6824
:1009900022B19042FAD102681A6070470A4A13687D
:1009A0001BB1984203D01A46F9E7084A05E00368EC
:1009B000136070479842FAD01A461368002BF9D199
:1009C000704700BFF4030020E8030020F803002074
:1009D00008B500231846054A054900F0E5FE4FF02A
:1009E000FF30BDE80840FFF7F7BE00BFA9080008C8
:1009F00040420F0070B5084EFFF7EBFE3468054625
:100A0000FFF7E7FE8542F7D800222346141843F18A
:100A100000052046294670BDF0030020F8B50446C5
:100A20000D46FFF7D6FE002385420646236010D30D
:100A3000A5F10A0383420CD20A35FFF7CAFE8542AC
:100A4000FBD3FFF7C6FE8542FBD8E36820699847D1
:100A50003EE0FFF705FD63680746002B34D1A3682D
:100A6000002B31D11B4B65601A681B68B54238BF3B
:100A70000132A260A2689A4203D92046FFF7B6FE6F
:100A80001EE0B54202D9144B19460EE0134A136812
:100A900023B159688D4201D31A46F8E723601460E8
:100AA0000EE05068854203D313461A68002AF8D135
:100AB00022601C600B689C4202D1A81FFFF78CFECD
:100AC0003846FFF7D5FC03E02046FFF751FFC9E7A2
:100AD0000020F8BDF0030020F4030020E80300200C
:100AE00038B50446FFF7BCFC6368054633B9A36814
:100AF00023B92846BDE83840FFF7BABC2046FFF7C7
:100B000037FFF6E7C36870B504460D46C3B1FFF77B
:100B1000E7FF092D0CD8FFF75CFE0646FFF759FEEC
:100B2000801B8542FAD8E3682069BDE87040184709
:100B3000FFF74FFE29182046BDE87040FFF76EBF53
:100B400070BD00002DE9F04704460E4690461AB9E4
:100B5000BDE8F047FFF7D6BFFFF782FC63680746A2
:100B6000E3B9A368D3B9DFF83CA0FFF732FEDAF8A7
:100B700000508146FFF72DFE8145F6D8304408EB42
:100B80000502864288BF01326060A2602046FFF7FE
:100B90002DFE3846BDE8F047FFF76ABC2046FFF758
:100BA000E7FEE0E7F003002008B50121094800F066
:100BB0009BFC0121084800F097FC0121074800F048
:100BC00093FC0121064800F08FFCBDE8084000F0CE
:100BD00021B900BF0D0C02400C0C02400E0C02406B
:100BE0000F0C02407047000008B50F4B1A680C4606
:100BF0009AB9012203281A6003D171460B480DF0FF
:100C0000E9FF21460A480DF0E5FF00F04FF90948D9
:100C10000DF0E0FF08480DF0DDFFFFF721FCFFF7C6
:100C2000E1FFFFF7B1FD00BFFC030020B70701089B
:100C3000BB070108E3070108D707010808B500F062
:100C400047FF03480DF0C6FF00F020FE002008BD5E
:100C5000E507010808B500F00BF9FCE71FB5FFF741
:100C6000FFFB0E4B0E481B68029300240D4B0093B4
:100C70000F220C234FF48071019400F055F80A4BB9
:100C80000A481B6802930A4B009307220C234FF477
:100C9000C061019400F048F8FFF7BAFB1802002089
:100CA00000040020550C00081C0200200005002054
:100CB0003D0C000808B5FFF7D3FB094B1B681A79F8
:100CC000082A07D95A79074B53F8221011B109683D
:100CD00043F82210FFF7CCFBBDE80840FFF79CBBB0
:100CE000D8020020E002002038B50B79082B03D988
:100CF00008490320FFF778FF4C7901F108020368E7
:100D00002BB113F8035CAC4201D31846F7E78B60B4
:100D1000026038BDA5070108031F53F8042F9A424B
:100D2000FBD0181A704700000F2A2DE9F74F05462F
:100D30008B4691469A462AD810F003031BBFC3F195
:100D40000403ED180B46CB1A303B23F003031AF0D3
:100D5000080F05EB030405D02A46A24203D2126015
:100D60000432FAE72D600193FFF77AFB2749019BD4
:100D70008046012251F8227016B25FB10132212A59
:100D8000F8D14046FFF774FB6FF08A003BE06FF04C
:100D9000150038E01D490C9841F822402A46E680AB
:100DA0000D99FFF7E3FA0E9B194AA3624FF0FF3348
:100DB000E3611368206001331AF0010F6562C4F823
:100DC0002CB084F805902771A760E7602761676100
:100DD000A7612762136004D001212046FFF746FA7D
:100DE0000DE00A212046FFF741FA1AF0040F06D160
:100DF0004046FFF73DFB4846FFF778FA02E04046E1
:100E0000FFF736FB304603B0BDE8F08F200300202B
:100E1000DC02002008B501F0CDF800F0B9F8BDE81B
:100E2000084000F01CB838B50446043000F01BFD43
:100E30000546204600F0BEFE284638BDF8B50446FB
:100E40000E461746051D3A463146284600F0F6FC88
:100E500020B90121204600F07DFEF4E7F8BD08B579
:100E6000002000F01BFA0120BDE8084000F016BA8F
:100E7000F8B50D4B1E68C6F307221D4622B9F4B221
:100E8000003418BF012400E00224FFF7E9FA2B68C0
:100E90009E42074602D12046FFF73EFC3846BDE899
:100EA000F840FFF7E5BA00BF200200202DE9F04F1F
:100EB0002C4B2D4A1B882D492D482E4EDFF8CCB0E7
:100EC0008BB00DF1280906F1800A29F8043D0DF0D8
:100ED00081FEFFF781FA0546FFF796FA0446FFF711
:100EE0008FFA2A46009023464FF4007122480DF0F5
:100EF00071FE25EAE5754FF4007856F8044B14B3FB
:100F00002779E26A5BF82730606A0793904406927B
:100F1000FFF702FF069AB4F90610079B101A226821
:100F20000592626A04920390E26A029262790192E7
:100F3000082FD4BF4F4609F1010700970544A26A64
:100F40000E480DF047FEB245D7D10D4B02958DE806
:100F500008010C4A0C4819460DF03CFE0BB0BDE8E8
:100F6000F08F00BF3D0801086C08010872080108F5
:100F70007708010824030020BF08010809090108B7
:100F800045090108470901084B0901084008010803
:100F900038B5FFF765FA1B4C0023E360054600F007
:100FA00037F84FF41443A360A268164B12F00C0FED
:100FB000FAD1154A40F20571116081221A601A684F
:100FC00042F480321A601A6812F4003F0D4AFAD0D7
:100FD0000E4B5360136843F0807313601168094B24
:100FE0008901FBD59A6842F002029A609A6802F081
:100FF0000C02082AFAD100F017F82846BDE838405C
:10100000FFF736BA00380240003C0240042A40078D
:10101000044B1A6842F001021A601A689207FCD564
:10102000704700BF00380240044B9A6812F00C0F62
:101030001EBF1A6822F001021A6070470038024091
:10104000034B044A00280CBF10461846704700BFE7
:1010500000BD010580DE800204281CD8DFE800F016
:1010600003080D1217000D4B1A6C1143196412E09E
:101070000A4A536C194351640DE0084A136B194333
:10108000116308E0054A536B1943516303E0034AB7
:10109000936B19439163BFF34F8F70470038024041
:1010A000042821D8DFE800F003090F151B000F4AC0
:1010B000136C23EA0101116470470C4A536C23EA54
:1010C000010151647047094A136B23EA010111635E
:1010D0007047064A536B23EA010151637047034A84
:1010E000936B23EA01019163704700BF003802400F
:1010F00038B514230C4A4343D4582568AA0608D5AA
:101100000A4B616803EBC002C9B253F83030506833
:1011100098472B0748BF6368054B1B681BB1BDE8A8
:101120003840FFF7C7BD38BDC4090108000B0020D7
:10113000D002002001282DE9F04780460D461746D1
:1011400003D92B490320FFF74FFDDFF8B090294A60
:10115000142404FB009442F83070E66802EBC002ED
:1011600001215360304600F0BFF9304600F080FAAC
:101170003046617C00F054FA4E464FB1D4F80890E6
:101180000021484600F0B0F9217C484600F048FABA
:10119000142303FB08F806EB080999F812A0D9F804
:1011A00004105046FFF758FF56F808400023E3604C
:1011B000504623616361FFF743FFB0FBF5F080B257
:1011C000A06077B199F8133001215AB203F01F03E0
:1011D00001FA03F35209084941F8223042F22C0384
:1011E00001E042F20803E3600020BDE8F08700BFA1
:1011F000A5070108000B002000E100E0C409010878
:10120000012838B505D80E4C14230A4403FB0043CB
:1012100009E00C490320FFF7E7FC25682D06FCD503
:1012200011F8015B65608A4201D01C68F5E7142360
:101230005843034B1A5813685B06FCD538BD00BFF2
:10124000C4090108A50701080020FFF751BF0120CC
:10125000FFF74EBFF8B5104C04EB4014012167684E
:10126000384600F041F9A6680021304600F03CF90C
:10127000E5680121284600F037F9247D38462146EB
:1012800000F0CEF92146304600F0CAF92146284642
:10129000BDE8F84000F0C4B9F809010801282DE9BB
:1012A000F041044603D910490320FFF79DFC0F4B82
:1012B000DFF83C80002543F820506401FFF7CAFFA7
:1012C00008EB04031E7F9F6930463946FFF7C4FED2
:1012D00058F8043039461D603046DD615D60BDE878
:1012E000F041FFF7DDBE00BFA5070108100B00208D
:1012F000F8090108012870B50C4621D84A1C22D0F3
:1013000021F0FF0313F5807F11D114F0FF041AD1EF
:101310000E4B03EB40152E69731C14D0012130468F
:1013200000F0E2F8297D304600F07AF906E001216C
:10133000204600F0D9F8204600F09AF9002070BD50
:101340004FF0FF3070BD6FF0010070BDF80901086B
:10135000042B2DE9F84304460E461546984603D95A
:1013600017490320FFF740FC1648DFF8609067013B
:10137000012100EB840000F0EDFB09EB07031C7F6B
:1013800099692046FFF768FE0F4B59F8071004EBE8
:1013900084041C4416F5807F14F8082045EAC20531
:1013A00045F004050D6015BF0B684B6843F44073AE
:1013B00043F0040314BF0B604B600020BDE8F883CA
:1013C000A5070108100B0020EC090108F809010825
:1013D0000B4A430110B50446D018D3588169007FE9
:1013E00000221A605A6822F004025A60FFF758FE81
:1013F000044800EB8400BDE8104000F0DBBB00BFF8
:10140000F8090108100B00202DE9F843089E099FF8
:10141000884691461D4623B91EB931490320FFF77E
:10142000E3FB304B400118F5807F1C58236843F0E4
:101430004003236005D0B8F1FF3F02D0404600F0E2
:1014400020F9A6B92F44AF4206D0A3689E07FCD569
:1014500015F8013B2373F6E7A3689807FCD5A3684A
:101460001906FCD4A368DA0720D5E368FAE70DB1C2
:10147000002319E030463744B84217D0A3689B07D1
:10148000FCD52573A368DE07FCD5237B00F8013B60
:10149000F2E7A2689007FCD5EA5C2273A268D10744
:1014A000FCD5227BF2540133BB42F2D1A3689A07E8
:1014B000FCD5A3681B06FCD4B9F1000F0ED1B8F11E
:1014C000FF3F0BD0236818F5807F23F04003236093
:1014D00004D04046BDE8F84300F0CAB8BDE8F88340
:1014E000A5070108F8090108F8B50D460126C0F363
:1014F000832120F00F0400F00F0706FA01F102200B
:10150000FFF7AAFD07FA06F00323216883406FEA7C
:10151000030C01EA0C012160216805F0030E0EFAAC
:1015200000FE4EEA01012160E2680CEA0202E2607C
:10153000E168C5F3810282400A43E2606268BE400E
:1015400022EA060666606268C5F30015BD401543D1
:101550006560A2681343A3600020F8BD2DE9F04147
:1015600000F00F0415462B4A42F8343002EBC40257
:10157000069B536006468846C0F383274FF480419C
:101580000120FFF769FD41463046FFF7ADFF042C0F
:10159000214B03DCA11D01228A4003E0092C03DC5E
:1015A0004FF400021A6002E04FF480725A601B4B45
:1015B0000120996800FA04F2D243114099609968B9
:1015C00005EA000E0EFA04FE4EEA01019960D968A0
:1015D0000A40DA60C540DA68A54004F00C0404F162
:1015E000804404F59C341543DD6006F00302A568D1
:1015F00092000F21914025EA0101A160A168974066
:10160000B0400F43A76058611A681043186000206B
:10161000BDE8F081180B002000E100E0003C014033
:1016200020F00F0300F00F02F0B51E6857000325ED
:10163000BD4026EA05051D601D680224072A04FA3C
:1016400007F444EA050494BF002201221C6003EB66
:10165000820300F007001C6A80000F22824024EA07
:1016600002021A621A6A814041EA02001862F0BD61
:1016700020F00F02012300F00F0003FA00F0906148
:10168000704720F00F0200F00F001030012303FA22
:1016900000F0906170470000104B2DE9F0415E6949
:1016A0001A680F4F164000244FF001081D4608FA33
:1016B00004F31E4206D06B6107EBC40357F83420D5
:1016C000586890470134102CF1D1064B1B681BB1B0
:1016D000BDE8F041FFF7EEBABDE8F081003C014003
:1016E000180B0020D00200202DE9F843124ADFF841
:1016F000508003010746D5582E69EB6800241E4030
:1017000008EBC0090223A3401E4209D0EA68D9F8B9
:10171000040022EA0303EB60214658F8373098476B
:101720000134042CEED1054B1B681BB1BDE8F84316
:10173000FFF7C0BABDE8F883380A0108D0020020DC
:10174000980B0020032910B516D80D4B00011C186A
:101750001B586068024001F10C0003EB80004260FE
:101760001869022202FA01F120EA01021A61DA681C
:101770001143D960002010BD4FF0FF3010BD00BFF5
:10178000380A01080001024B1B58586A704700BF15
:10179000380A0108034B00011A58136843F001038B
:1017A00013607047380A010801282DE9F8430546FF
:1017B000884630D81A4E1B490401371941F83020A9
:1017C00097F80C9001EBC00148464B60B968FFF7F1
:1017D00043FC36597B680024346048467460F362E9
:1017E000FFF72EFC104B7A7B13F809305843B0FBFF
:1017F000F8F3013BB36251B2012302F01F0273619F
:1018000049099340094A284642F82130FFF7C2FFB0
:101810002046BDE8F8834FF0FF30BDE8F88300BFF5
:10182000380A0108980B0020580A010800E100E07E
:101830000020FFF759BF0120FFF756BF70B51346D0
:101840007BB18568C468A5420BD084680668651CB6
:1018500085604568013D2C40013B345D01F8014B3A
:10186000EEE7D01A70BDC368426830B584681B1BB0
:10187000934208D0C3680468013A5D1C1340C560F8
:10188000E154002030BD4FF0FF3030BD00B50821DD
:10189000A1B0074800F07AFB06480DF025FA06488B
:1018A0000DF022FA80226946044807F069FB00BF68
:1018B000A80B00205A0A0108810A0108D00A010871
:1018C0002DE9F04F012889B006460D4602DC096873
:1018D000664882E0664968680DF006FB0446002809
:1018E00071D1042E02DC2968624876E0052E0AD008
:1018F00068690CF0BFFC062E814606D0A8690CF082
:10190000B9FC074602E04FF001095B4FAB68019359
:1019100001992B69EE68029304A807F0DFF908B972
:10192000564898E030460CF0A5FC1FFA80F8824635
:10193000B8F1000F01D000260DE051488BE01FFAEE
:101940008AF3019A03994F480DF044F90021384673
:101950000AF062F901364E4500F0848002980DF0DD
:101960008FFC002302460299184603F05FF90546F2
:1019700008B945486FE0C36803934246414606F004
:10198000E5FE834608B9414818E004AA002100F0AA
:1019900011FF054638B93E480DF0A6F929465846CC
:1019A00003F036FA5EE0034640F202223949042091
:1019B00002F09CFC83460028C1D137480DF094F911
:1019C00059462846ECE7354968680DF08DFA00283D
:1019D00044D1022E05D1296831480DF0FBF80124CD
:1019E00040E03049A8680DF07FFA0446F8B9032EAC
:1019F00002D129682C48F0E72C4EB6F9083013B113
:101A000071682B4810E0E8680CF034FC85B20DB921
:101A1000284820E0284B75601B883381314604201C
:101A200002F00AFF254829460DF0D4F81AE02449AF
:101A3000A8680DF059FA044680B91C4DB5F9083074
:101A40001BB920480DF0C6F80CE00420294602F02E
:101A500013FF1D482C810DF047F903E01B480DF0E2
:101A600043F90024204609B0BDE8F08FE80A0108D8
:101A70008C090108010B010840420F003E0B0108D0
:101A8000690B01082B0C0108910B0108BD0B010823
:101A9000E20B01080000FFFF080C01083E0D0108E1
:101AA000500C01086F0C0108750C0108240200207D
:101AB000930C0108BE0C010860310020DC0C010809
:101AC000050D01080A0D0108290D0108450D010841
:101AD00008B5002007F0FAF9FEF77AFF03F08AF85C
:101AE00003F06CFA04F0F4FE00F03EFC06F040FE59
:101AF00000F006F801F084F9BDE8084003F07CBA74
:101B000013B50E4C0E490F480AF0F2F80D49204665
:101B100002F086FD002806DA0B48002102B0BDE87D
:101B200010400DF057B80094084B094802224FF4BA
:101B3000806102F00BFE02B010BD00BF401000201B
:101B40005C0D0108E80F0020740D0108AE0D0108BE
:101B5000E80B002070B505460C46FEF781FC2B68AB
:101B600006462BB94FF0FF332B60FEF781FC18E0DF
:101B7000CCB10F4B1C6802212046FEF777FB2B6887
:101B8000013305D104F108032B600023A36003E0B7
:101B900021462846FFF7A8F83046FEF769FCFEF715
:101BA0003BFC012070BDFEF763FC204670BD00BF0A
:101BB000D802002070B50446FEF752FC25680646A0
:101BC0001DB16B1C05D100232360BDE87040FEF7FA
:101BD0004FBC28460A2150F808392360FEF746FB1F
:101BE000236813B94FF0FF33236015F8034C3046D8
:101BF000FEF73EFC2046BDE87040FEF777BB0000D4
:101C0000F8B505460E46FEF72BFC364B364A1B88C8
:101C10001BB2074652F82320D2F820E0BEF1000F95
:101C20001AD054699369A34216D9631C5361D369CE
:101C30001C4046B9136933B9631C04D13846FEF71A
:101C400017FC2046F8BD002C0ADB0EEBC40393E81A
:101C5000030085E8030004E04FF0FF34002EE9D0D4
:101C6000D560166976B333681361002C0CDB956977
:101C70005169D369691A8B42A9BF691C4FF0FF35BE
:101C80001D4091610EEBC505736893E8030085E87C
:101C9000030016F8043C052B09D0002373600A21C9
:101CA000A6F10800FEF7E2FA16F8034C00E00F2454
:101CB0003846FEF7DDFB0E2C02D82046FEF716FB59
:101CC0000120F8BD002C09DA10460321FEF7CEFAF8
:101CD0003846FEF7CDFBFEF79FFBF1E73846FEF7EF
:101CE000C7FBEDE7D40200202003002010B5836974
:101CF0004469C2691C1BA24201DA002010BD5C1CB1
:101D000013408461F9D4026A03C902EBC30383E878
:101D10000300012010BD00002DE9F8431E46264BAC
:101D200053F82150254B1B880380074691462DB957
:101D30003046FEF79DFB4FF0FF3439E02B79032B43
:101D400028D01F4B01462846D3F80080FFF7CEFF6E
:101D5000044638B13046FEF78BFB98F80430052B6B
:101D600025D122E0B9F1000F03D13046FEF780FB08
:101D70001EE098F80430C8F80C70052B0CBF052144
:101D800004214046FEF772FA414605F11000FEF7C5
:101D9000ABFF07E003C8EB6883E803000A2128468D
:101DA000FEF764FA3046FEF763FBFEF735FB0124CD
:101DB0002046BDE8F88300BF20030020D4020020A5
:101DC000D802002038B50446FEF74AFB074B1B88B3
:101DD0002380074B214605461868FFF787FF044616
:101DE0002846FEF745FB204638BD00BFD402002040
:101DF000D802002008B50F4B53F82130B3B121228F
:101E000002801A79032A0BD103C8DA6882E803003A
:101E100018460A21FEF72AFA074B0120186008BD70
:101E200001461846BDE80840FFF760BF4FF0FF309D
:101E300008BD00BF20030020D002002070B504467A
:101E40000D46FEF718FB28B129462046BDE8704034
:101E5000FFF7D0BF094B1B881BB29D4204D120461F
:101E6000BDE87040FFF7AEBFFEF7FAFA2946034619
:101E700001222046BDE87040FFF74EBFD40200208B
:101E800070B504460D46FEF7F6FA064628B1294617
:101E90002046BDE87040FFF7ADBF0A4B1B881BB260
:101EA0009D4204D12046BDE87040FFF78BBFFEF78E
:101EB000D7FA3246034629462046BDE87040FFF770
:101EC0002BBF00BFD40200202DE9F041124F3B8808
:101ED0001BB2934206460C46154603D10F49032018
:101EE000FEF782FEFEF7BCFA3A880D4B12B280462E
:101EF00053F8227005213846FEF7B8F996E803003A
:101F0000FC60434684E80300012229462046BDE8E0
:101F1000F041FFF701BF00BFD4020020A507010870
:101F20002003002070B504460D46FEF799FAB4F977
:101F30000020114B53F8224006461CB90F490320DC
:101F4000FEF752FE2379052B04D0FEF791FA4FF0ED
:101F5000FF3070BD95E80300E36883E803000A21C1
:101F60002046FEF783F964793046FEF781FA204671
:101F7000FEF7BCF9012070BD20030020A507010871
:101F80000021FFF73DBE0121FFF73ABE08B5074B20
:101F90004A1E1B681140186203D005490320FEF752
:101FA00023FE59619961DA6108BD00BFD8020020A3
:101FB000A50701080F4BD3F8882042F47002C3F83C
:101FC00088200D4A9A60102283F822200021DA77B7
:101FD00001F1604000F561400131522980F8002391
:101FE000F6D11A6942F010021A615A6942F400727D
:101FF0005A61704700ED00E0000000080346002031
:102000001BB1DA685B681044FAE7704710B5082224
:10201000094904460CF0A6FB48B12378FF2B08D1F0
:10202000607800F00F00831E5842584110BD012017
:1020300010BD002010BD00BF7C0F0108002102F080
:10204000E7BE38B5CBB2002114460246084602F07E
:10205000BDFB054618B92046FFF7F0FF0FE094F9E5
:10206000103001330AD1A36882681B7903F03F0363
:1020700021462046137102F08BFC04466C60284612
:1020800038BD00002DE9F0478C68074610468846A9
:102090001546FFF7B3FFA37940BAFF2BA0800AD102
:1020A0002B7C023BDBB2022B03D8214AD35CFF2BF3
:1020B00000D13B23A371E37943B90FB9402304E076
:1020C000384600F0F9FC90F8CA31E37104F10806D3
:1020D0001022184930460CF045FB8246D0B904F175
:1020E00018091549102248460CF03CFB014630B94E
:1020F000102230460CF066FC0123E3750AE04946E5
:102100005246384600F0B2FD014618B11022304662
:102110000CF05AFB4146284602F0F4FB002804DA92
:10212000831C08BF0020BDE8F0870020BDE8F087D1
:10213000BD0D0108CC0F0108DC0F01088B6870B5DC
:1021400058800C46054600F0B7FC014618B91949FD
:102150000320FEF749FD66683046FFF74FFFB1F8F0
:10216000C831984204D92046BDE87040FFF766BFE9
:10217000D1F81C320133C1F81C323046FFF73EFF64
:10218000D1F824321844B1F8C631C1F82402DB0773
:1021900008D5234640F202220749012002F0A6F8A2
:1021A00030B9E0E72146284602F0CBF80028DADD16
:1021B00070BD00BFA50701080000FFFF2DE9F04F2B
:1021C00085B090F91030013300AF044689460AD13A
:1021D0008368B3F9026002F029FE00286AD04368E0
:1021E0000446984601E080460026404602F01EFE66
:1021F000054600285ED04445836818BF60601A46D3
:102200001B7ED0F8048008BF0446FF2B2BD186B973
:1022100007F1080002F0C4FA00284BD00021224642
:102220000846B7F90860FFF70CFF0446002800F0E5
:102230009380B9F1000F06D0424629463046FFF799
:1022400021FF002836DBA268137943F040031371A5
:10225000304600F089FE4368013343602146304632
:10226000FFF76CFF78E01346183310223C491846FC
:102270009B460CF077FA40B15946002E39D1381DF3
:1022800000F098FC0646002838D0B9F1000F06D0BF
:10229000424629463046FFF7F5FE00280ADB28466D
:1022A000FFF7ACFE002102460223084602F0BEFC06
:1022B000064608B9204619E083689846EA68A96886
:1022C00040460CF081FAEB686D6842461A4490462D
:1022D000002DF3D12046FFF7B1FE224B3146B3F972
:1022E000000002F03BF8002836DC3046FFF7A6FE7F
:1022F00032E0304600F036FC0028C6D107F110016C
:10230000082301F80D3D32465B4607F1080005F051
:1023100087FDEA46064640B1B9F1000F09D04246B2
:102320002946FFF7AFFE002803DA2046FFF786FEB6
:1023300011E02246F97807F10800FFF782FE044613
:1023400048B1304600F010FE0368013303602146B7
:102350003046FFF7F3FED5461437BD46BDE8F08F93
:10236000DC0F0108841000201FB50F4CB4F90030B9
:1023700063B90E4A01930E4B029200930422082384
:102380004FF480610B48FEF7CFFC20800A480B4BCE
:10239000036001230371142383600AF03AFEB4F949
:1023A000000004B010BD00BF84100020B80D01086B
:1023B000612600088610002050100020881400209C
:1023C000292B2DE9F84381460F4614461D4606D0B9
:1023D0003A2B06D0112B0CBF0423002302E002236A
:1023E00000E00323292D3B7401D03A2D03D1A742ED
:1023F00059D1012605E0A74202D063689F4252D11D
:1024000000267B6893F91000022805D016B301213D
:10241000204602F0EBFC1DE0294602F057FA18B9FD
:1024200086F0010836B101E04FF000080121204696
:1024300002F0DCFC234640F201221E4997F910000D
:1024400001F054FF10B92046FFF7F8FDB8F1000F76
:10245000DCD00AE0234640F201222946022001F0A6
:1024600045FF10B92046FFF7E9FD06B3292D07D037
:102470003A2D18D121464846BDE8F8430AF092BFEC
:1024800000232374616839B191F91030022B03D114
:10249000204602F07DFAF5E7022323742046BDE8CA
:1024A000F84300F00BB804490320FEF79DFBBDE89C
:1024B000F88300BF0000FFFFA50701082DE9F047E2
:1024C000044618B964490320FEF78EFB4FF0FF3134
:1024D00002F029FA0546A0B18368B3F90260002E24
:1024E000F0D0304600F040FD4369013301464361BE
:1024F0002046FFF783FDEA688B699B1A18448861C0
:1025000000E006462746254695F91030022B08D1F3
:10251000EB68282B05D1AB681B7803F0F003602B28
:1025200008D0D5F804802F46B8F1000F6ED045468C
:10253000EAE73C46D5F80880E368B8F8041049BAE1
:1025400089B2994203D2204602F0F8FB0FE02246FE
:102550000023D068034492F91000022803D1283BDD
:10256000994204D95DE05268002AF2D1F7E708F1F8
:1025700018091022394948460CF0F4F8002855D0C3
:102580004846FFF743FD494600B136B9002000F048
:1025900011FB002E08BF064602E0304600F0E2FACA
:1025A000B0FA80F04009002840D008F10800FFF799
:1025B0002DFDB0BB4846FFF729FD90BB98F80730CA
:1025C000013BDBB288F807305BB3284602F02EFCF3
:1025D00038B34FF0FF31204602F0A5F9014610B1A3
:1025E000204602F0D5F921460025084602F01EFCDF
:1025F00018B92846FFF722FD13E0416845600546FB
:102600000029F2D1BDE8F047FFF7D8BDA3681B78D9
:1026100003F0F003602B04D1204602F007FC0746CC
:1026200068B92046BDE8F047FFF708BD98F80630C6
:10263000224639463046BDE8F047FFF7C1BE0222C8
:10264000282102F00DFB87F81080054600287FF452
:1026500070AF3846E6E700BFA5070108DC0F0108A8
:1026600010B598B0514B0693514B08211B88ADF81B
:102670001C3008A800240594FFF788FC05A9022057
:1026800002F0DAF840F20523ADF80E3001A8FFF7AA
:102690007AFCBDF806306FF400721344222BF5D893
:1026A00001A252F823F000BF352700083D2700089B
:1026B00047270008472700088D2600088D260008B8
:1026C0008D2600088D2600088D2600088D2600081E
:1026D0008D2600088D2600088D2600088D2600080E
:1026E0008D260008572700088D260008632700085C
:1026F0008D2600088D2600089B2700088D260008DF
:102700006B2700088D2600088D2600088D260008FE
:102710008D2600088D2600088D2600088D260008CD
:102720008D260008732700087B27000883270008F0
:10273000932700080298FFF7C1FEA7E7012102983E
:10274000FFF73CFDA2E76FF0850303A901A80493FE
:10275000FFF7E8FB9AE7029A537E23F008035376CB
:1027600094E7029800F072FF90E7029800F0FCFFF7
:102770008CE7029805F0CEFA88E7029805F020FB76
:1027800084E7029B587C00F00F0004F00DF90474FC
:102790007CE7029805F07AFD78E7029A0023194653
:1027A000B2F91A0001F040FB70E700BF0000FFFF24
:1027B000D4020020F8B50F46164602232822002135
:1027C00002F034FA054600B38468102204F10800D0
:1027D000394617B10BF0F8FF01E00CF0F3F804F103
:1027E00018001022314616B10BF0EEFF04E00CF099
:1027F000E9F8012384F82730602200232270FF22A9
:102800006370A370E370A271E3712846F8BD0121E3
:10281000FFF7A0B92DE9F84300F5E0750746284613
:102820008846FFF7F4FF00244FF0380909FB0476CF
:102830004146304606F035F938B1102200213046C5
:102840000CF0C0F80023337402E00134082CEDD101
:102850002846BDE8F843FFF7ADB9000008B51022DF
:1028600003490BF07FFFB0FA80F0400908BD00BFBC
:10287000CC0F010810B50822094904460BF072FF7D
:1028800048B12378FF2B08D1607800F00F00831E39
:102890005842584110BD012010BD002010BD00BF9E
:1028A0007C0F01082DE9FF47002605468846924621
:1028B00099463446AF194146384606F0F2F80028EA
:1028C0007FD13846FFF7CAFF10B1002C08BF3C4645
:1028D0003836B6F5E07FEDD12746002C71D01022B6
:1028E000414620460BF070FF237884F811A0FF2B9F
:1028F00084F8109016D0B5F8C631DA0712D501F079
:10290000E1F8814670B105F5E0763046FFF752F9FF
:10291000B5F9C4014B464A46214601F083F93046D9
:10292000FFF775FF98F80030FF2B04D1237C43F0AC
:102930000103237441E04046FFF79CFF8146C8B97C
:10294000B5F8C62102F00602062A17D105F5E07691
:102950003046FFF72FF9B5F8C631DB0706D54B46F1
:102960004A464946B5F9C40101F05EFA3046FFF720
:102970004EFF03E0237C63F07F032374B5F8C63178
:1029800003F00303012B18D040F2FF220023CDE90E
:1029900000234FF080730293FF238DF80C3098F8DA
:1029A0000D308DF80D30B8F80E30ADF80E308022B5
:1029B000002369462846FFF775FF40F2112363861E
:1029C0006463384604B0BDE8F08703885BBA23F03F
:1029D0003F031B041B0C4FF6C062934209D00378DF
:1029E000FF2B08D1407800F00F00052818BF0E20FB
:1029F0007047052070470E2070472DE9F0470025ED
:102A0000804691461F460C462E464FF0010A3FB1C4
:102A10003A780AFA05F31A421AD0237CDB0717D456
:102A20002046FFF71BFF98B94946204606F04EF8AE
:102A300037B999F80030FF2B02D0637C834207D866
:102A4000B04205D9B8F1000F01D0C8F800400646E1
:102A50000135082D04F13804D9D13046BDE8F0879E
:102A600070B5134CB4F9C451A84206461ED0EDB956
:102A700004F5E070FFF7CBFE4FF4A063A4F8C83173
:102A8000402384F8CA31A4F8C4612B46A4F8C65187
:102A9000802208492046FFF705FF04F5E070FFF7A4
:102AA00089F82046BDE8704000F06CBE70BD00BFE4
:102AB000081700209C0F0108034BB3F9C421824280
:102AC0000CBF18460020704708170020B0F8C63128
:102AD000DA0707D511B143F0020301E023F0020346
:102AE000A0F8C6317047B0F8C631DB0701D505F054
:102AF0008DBB70472DE9F0410D4617469846FFF70C
:102B0000DBFF044610B90020BDE8F0810029FAD0AF
:102B10000846FFF7A3FE0028F5D1802FF3DC04F56B
:102B2000E0763046FFF773FE43463A462946204694
:102B3000FFF7B8FE04463046FFF73CF82046BDE8F4
:102B4000F081000010B520B90548B0F9C43133B1A7
:102B500001E0FFF7B1FFBDE81040FFF75BBE10BD1D
:102B6000081700202DE9F8438946FFF7A5FF044622
:102B7000E8B100F5E0763046FFF749FE002504EBAA
:102B800005084946404605F08CFF074628B1304607
:102B9000FFF710F84046BDE8F8833835B5F5E07F1B
:102BA000EDD13046FFF706F83846BDE8F883BDE8BA
:102BB000F883000038B5084C0546B4F9C4011DB9C6
:102BC000FFF7D0FF20B938BDFFF7CCFF286008B170
:102BD000B4F9C40138BD00BF081700202DE9F34146
:102BE00002AD00260E4C45F8046D8846074604F5F4
:102BF000E070FFF70CFE3346424621462846FFF7B9
:102C0000FCFE20B1019B3B60B4F9C44100E00446E6
:102C10000448FEF7CFFF204602B0BDE8F08100BFB8
:102C200008170020C81800202DE9F34102AC002746
:102C3000884644F8047DFFF73FFF00F5E07506463F
:102C40002846FFF7E4FD20463B4642463146FFF763
:102C5000D4FE044628461CB1FEF7ACFF019802E002
:102C6000FEF7A8FF204602B0BDE8F0812DE9F04F45
:102C700087B00F461546FFF71FFF00F5E07380464B
:102C800018460193FFF7C3FD0122002102A80BF0B3
:102C900099FE4646C3464FF0FF3A00244FF0010923
:102CA0009BF80020FF2A12D05846FFF7D7FD70B9D5
:102CB00045B99DF8081009FA04F20A438DF8082076
:102CC000A24604E05846FFF7D5FD0028F1D10134B3
:102CD000082C0BF1380BE3D1BAF1FF3F00F08780ED
:102CE00004AD2246002128460BF06CFE3B78FF2BFA
:102CF00004D197F8019009F00F0309E03846FFF777
:102D0000B9FD20B93846FFF760FE009001E00223CC
:102D100000934FF000094C469DF80810012303FA78
:102D200004F2114232D039463046B34605F0B9FEBE
:102D3000002855D13046FFF79DFD18B93046FFF702
:102D400044FE00E00220009B834208D12A5D043249
:102D5000D2B22A554A4588BF4FF004090AE009D982
:102D60002A5D0232D2B24A4513462A5538BF4B4635
:102D70005FFA83F9B2694AB12A5D0132D2B24A459B
:102D800013462A5538BF4B465FFA83F90134082CA5
:102D900006F13806C0D10122002102A80BF012FE74
:102DA00000209DF80820014601246E5C4E4504BFBA
:102DB00004FA01F0024301F1010104BFD2B2012083
:102DC0000829F2D108B18DF8082006A8002340F8A0
:102DD0000C3D3A4602AB4146FFF70FFEDDF80CB062
:102DE000BBF1000F05D1382202FB0A8B01E04FF046
:102DF000000B0198FEF7DEFE584607B0BDE8F08FE5
:102E00002DE9F04F8DB005A801F0CAFC0026544F03
:102E100003900DF11205B146039B9E4200F09D8088
:102E200035F9020FFFF748FE0446002800F09180B4
:102E300000F5E07A5046FFF7EAFC0123B5F90000FF
:102E4000009300220DF1130317218DF8139001F068
:102E500093FA86302CD09DF91330012B28D108230A
:102E60000DF13008ADF818304FF6FF7328F8103D1B
:102E7000B7F8C631B5F9000043F003034FF0020B79
:102E8000A7F8C631002206AB0521CDF800B001F04D
:102E900099FAB5F90000CDF800B01121434600229F
:102EA00001F06AFABDF82010B5F9000005F03AFB10
:102EB0004FF00808B5F90000CDF8008006AB0022FD
:102EC000414601F059FA00280FDB424606A90AA83C
:102ED0000BF07AFC4246234908A80BF075FC00234E
:102EE000402208A92046FFF7DDFC0223B5F90000C7
:102EF000009300220DF11603112101F03DFA002884
:102F000006DBBDF81630B3F5A06F28BFA4F8C831B2
:102F100000231A462421B5F90000CDF8009001F0F5
:102F20002BFAB4F8C6310028CCBF43F0800323F05D
:102F30008003A4F8C6315046FEF73CFE012120462E
:102F4000FFF7C4FDB4F8C631DB0702D5204604F014
:102F5000A9FE013607F50C775EE70DB0BDE8F08FEE
:102F6000081700207C0F010808B5FFF7A5FD00F544
:102F7000057008BD2DE9F3410746884616461C46F4
:102F80000AF0A8FB054640B9032300933246A3B2DA
:102F9000414638460AF030FB20E0437E03F0070349
:102FA000012B01D103210DE0027EA3B29A4200F170
:102FB00010070CD031462C76224638460BF004FC24
:102FC0000321284602B0BDE8F04100F08FBE224642
:102FD000394630460BF0C6FB0028EBD102B0BDE805
:102FE000F08100002DE9F04F1D46D37991B0FF2B01
:102FF0008046069116461A9F40F0B4806B78002BED
:1030000040F0B080172F40F2AD802B7AFF2B00F0FC
:10301000A98002F108095549102248460BF0A2FB8D
:1030200070B105F108014046FFF79CFD05900028AE
:1030300000F098800023183F1C4619469A461BE072
:103040000D224B4906F118000BF08CFB002800F014
:103050008980E6E70AF1180205EB020BAA5C012A57
:103060000DD0212A08BF5C469BF801200AEBC20A5A
:103070001FFA8AFAA7EBC207002FEBDC0BE008ABC4
:103080002A780698009331465B4601F00DF8031E3E
:1030900068DB5946E8E7404607930691FFF70CFDC9
:1030A0000699079B18B933490320FDF79DFD08AA2F
:1030B000002942D0002C40D0B0F8C61101F0030125
:1030C00003293AD12978029301924B460A4600948B
:1030D0003146404604F094FF002304F108020F211A
:1030E000074604F073FF054617B91022494620E051
:1030F000237A83F002038DF82830637A8DF8293023
:10310000A37A8DF82A30E37A8DF82B30237B8DF863
:103110002C30637B8DF82D30A37B8DF82E30082268
:10312000E37B8DF82F300AA90EA80BF04DFB124956
:1031300008220CA80BF048FB09E049464046FFF77F
:1031400019FF102249460CA80BF03EFB0025337EE8
:103150000095A3F1FF025342534105990CAA404642
:1031600000F0D4FC11B0BDE8F08F00BFCC0F010817
:10317000BC0F0108A50701087C0F01082DE9F04FDD
:1031800089B003F108099246059149461D468046DB
:10319000129E0AF09FFA9AF80730FF2B40F0B58094
:1031A0006C78002C40F0B180172E40F2AE802B7A64
:1031B000FF2B00F0AA80002800F0A780183E2746C9
:1031C000002E27DD07F1180305EB030BEB5C022B48
:1031D0000DD0212B16D10023029301932A78CDF82C
:1031E00000B04B465146404604F00AFF0AE006ABE9
:1031F00000932A7805985B46514600F09CFF041E18
:10320000C0F283809BF8013007EBC307BFB2A6EB87
:10321000C306D5E74FF0FF31059801F084FB08B1F4
:10322000876800E00746494640460AF053FA0646DA
:1032300000286AD0437E03F00703022B12D127B186
:103240003B7813B17B78002B31D106A9A6F81A8000
:103250003476224606F110000BF0B6FA2B795906A7
:1032600016D512E01FB13B780BB17B7813BB002C55
:1032700049D1377E003718BF01272B799A062AD407
:103280004FB3A4BB2B795B0601D5072101E01FB129
:103290000321304600F02AFD95F90430002B737E9F
:1032A000B4BF43F0080323F0080373762DE0002C2D
:1032B000CBD12AE02CB3337E9C4209D0224606A90A
:1032C00006F110000BF04EFAB0FA80F0400900E071
:1032D00000200746D1E7002CD4D0A6F81A80347617
:1032E000224606A906F110000BF06EFACAE7737EBB
:1032F00003F00703072B08D10321304600F0F6FC4A
:1033000003E02746B9E70027B7E709B0BDE8F08F2B
:103310002DE9F04F87B01546984681460291109FDF
:10332000FFF7CAFBB0F8C6319A07064669D5EB79B4
:10333000FF2B66D198F80140002C62D1072F60D98D
:1033400005F10803083F0DF1100A0393002F1FDD5C
:1033500004F1080308EB030B18F80330012B0FD11D
:1033600098F800200298CDF800A05B46294600F0AE
:103370009BFE031E45DB524603994846FFF7FAFDC4
:103380009BF8013004EBC304A4B2A7EBC307DDE74D
:10339000B6F8C63113F0040F05F1080528D013F074
:1033A000010F194B194C18BF1C4605F095FD06F589
:1033B000FC7780463846FDF793FBB6F8C631DB074D
:1033C00016D5294648460AF085F988B1B8FBF4F1CC
:1033D00040F21523A6F80E320D4BC6F81002B3F9D1
:1033E000003006F5037204FB1181384608F03EFCFC
:1033F000294648460AF06EF918B1437E23F00803C7
:10340000437607B0BDE8F08F80841E0020A107003E
:10341000841000202DE9F04F89B092460591814635
:103420001E46FFF749FB0AF1080B054608228449AE
:1034300058460BF097F9002840F0FF809AF80830C2
:10344000FF2B00F0FA809AF80730FF2B40F0F58050
:103450007378002B40F0F180129B0F2B40F2ED802F
:10346000594648460AF036F9074650B90B230093EF
:1034700002460346594648460AF0BEF8074668B970
:10348000DBE0437E190706D5F28852BA92B212B930
:1034900023F0080301E043F008037B76F3889CB235
:1034A00064B15CBA674B68491B88A4B21BB207F1D0
:1034B0003002614307F11C0008F0D8FB33790BB1EF
:1034C00085F8CA31B5F8C631C3F30D02A5F8C62197
:1034D00073791B0203F440431343A5F8C631B06867
:1034E000A8B1D5F8D03190FA80F898450FD005F002
:1034F000F3FC0A22B0FBF2F303FB1200053008FBD9
:1035000000F0C5F8D081B0FBF2F0C5F8D401F36843
:1035100013B11BBAC5F8D83105F5E070FEF74AFBC8
:10352000129B103B0393002302930493039B002BF5
:1035300058DD029B103306EB0308F35C052B1CD00F
:1035400004D8012B0DD0032B1ED03FE0222B2AD014
:10355000232B3BD14346129A3146484604F0CEFE17
:1035600034E006AB0093327805984346514600F0AC
:103570009BFD031E049329DA5FE0424631784846FA
:1035800000F013FE10BB58E042463178484600F088
:1035900029FE002851D0D8F804301BBAB3B19C42A0
:1035A00028BF1C4612E04146307804F0FBFD00289D
:1035B00043D0B8F806305BBA9BB23BB13C22B4FBB7
:1035C000F2F2934202D23C2202FB03F498F801305B
:1035D000029A02EBC30292B20292039AA2EBC303D5
:1035E0000393A3E7049B06AA59464846FFF7C2FC8B
:1035F00005F5EE70FDF774FAB5F8C631DA071CD59B
:1036000004EB4404042C88BFA1084FF0000498BFC9
:103610000121384685F8CB4104F0ACFC3B463A46E4
:103620002146B7F91A0000F0FDFAB5F8C6319B073C
:1036300003D501212846FFF756FA09B0BDE8F08FFF
:103640007C0F0108D402002040420F002DE9F04118
:10365000437E03F00703022B86B0044601D0052BFE
:103660007BD194F89420B4F91A50012A71D9022B15
:1036700011D14FF080730493FF238DF81430637BD6
:103680008DF8153040F2FF200021E389ADF81630A7
:10369000CDE902010BE094E8030002AB83E80300EC
:1036A00004F1080393E8030006AB03E90300013AC1
:1036B00084F894201DBB01AE304601F071F8074636
:1036C000BD4208D036F9150002AB2246002100F0B9
:1036D000A9FA0135F4E7224B04F13805B3F900608B
:1036E0002846FDF7FDF940F21223A4F84E3004F10C
:1036F0004C0233461B49284608F0B8FA2DE028460C
:10370000FFF7DAF90646224602AB06F5E075B4F992
:103710001A00002100F086FA01212846FEF71AFA65
:103720000F4BD6F8D871B3F9008004F13806304653
:10373000FDF7D6F940F21223A4F84E303046434646
:1037400004F14C02394608F091FA2846FEF732FAA5
:1037500003E02146284609F0E5FF06B0BDE8F08108
:103760008410002040420F00437E03F00703042B27
:1037700003D0072B04D1032100E0052100F0B6BAE5
:103780007047000038B500F5E07504460121284671
:10379000FEF7E0F905F0A0FB0A210A4BB0FBF1F2BD
:1037A00002FB11000530C4F8D0314343B3FBF1F301
:1037B000C4F8D431044BC4F8D8312846BDE83840A9
:1037C000FEF7F8B980C3C90140420F0010B50446A6
:1037D00008462378FF2B14D000221823872109F0F4
:1037E0004BFE002270B183681A715A719A71DA71B6
:1037F00021686268DA609960A168E2685A611961BB
:1038000010BD002010BD38B50B78FF2B05460C46C7
:10381000104616D000221823882109F02DFE002220
:1038200080B1836825F01F051D71DA719A715A7194
:1038300021686268DA609960A168E2685A6119617A
:1038400038BD002038BD08B500220823852109F0C5
:1038500013FE28B1836800221A715A719A71DA71C5
:1038600008BD10B5002304461046CA1D02F0F80238
:10387000194601F0DBF920B182681470C368DB08D7
:10388000537010BDF8B516460F461A46B11CFFF727
:10389000E8FF044660B18568C2680235023A00213B
:1038A00028460BF08FF83246394628460AF08CFF3E
:1038B0002046F8BD13460A4601460120FFF7E2BF45
:1038C00013460A4601460220FFF7DCBF2DE9F0410E
:1038D00080460F4616461D46002210238621079873
:1038E00009F0CAFD60B1069B846827F03F0776BAED
:1038F0002DBA1BBA84F804806771E680A560E36086
:10390000BDE8F0812DE9F0410746884616462021A2
:10391000079A03201C46FFF7A4FF0546C8B180683C
:1039200024BA0021846028F03F0800F1100436BA60
:10393000017341738173C173877080F8038046609F
:10394000102220460BF03EF83A460699204605F034
:10395000E3F82846BDE8F08110B50A460446082180
:103960000520FFF77EFF28B18368002224BA9A70F1
:10397000DA705C6010BD000008B5102203490AF03F
:10398000F1FEB0FA80F0400908BD00BFCC0F01087D
:1039900010B50822094904460AF0E4FE48B123782C
:1039A000FF2B08D1607800F00F00831E5842584169
:1039B00010BD012010BD002010BD00BF7C0F01080C
:1039C00070B5064608461946FEF7F4FE0446A0B157
:1039D0008368FF22DA7100231A461946184600F060
:1039E000F5FE054620B92146204600F0D1FF02E051
:1039F00083685E804460284670BD70BD002101F080
:103A000007BA0000F7B51F46537C802B05460E46CB
:103A1000144603D911490320FDF7E6F81046FFF7D5
:103A2000ABFF08B1002017E02046FFF7B1FF0028E8
:103A3000F8D1217CCB07F5D43388607C626913F020
:103A4000010F14BF002680268DE89000A369314342
:103A5000FFF758FF2860012003B0F0BDA50701085B
:103A600030B585B0022300930D460DF10E03002200
:103A70000521044600F080FC002803DBBDF80E3071
:103A8000062B10D80823009300222B460221204643
:103A900000F072FC002802DBADF80E000EE00023FF
:103AA000ADF80E300AE00823009300222B460321D4
:103AB000204600F061FC0628E4DDEDE7BDF80E00CD
:103AC00005B030BD38B5002009F04EFE044658B1AF
:103AD000637E03F00703013B012B03D90A4B00224D
:103AE0001A600EE02046EFE7074D286809F03CFE1B
:103AF000034618B909F038FE034610B12B6018468A
:103B000038BD204638BD00BF381900202DE9F743E5
:103B10000A9C0F46994680461646FEF7CDFFB0F840
:103B2000C631990701D4002507E04046FEF7C4FFDF
:103B3000B0F8C6315A07F6D580253046FFF71CFF8E
:103B400038B11022334930460AF03EFE022373702A
:103B500001E045F04005B9F1000F0BD06946404641
:103B6000FFF77EFF30B1C1B222466846FFF7A8FEDC
:103B700068B1044624B13B7CDB0758BF45F0200503
:103B8000224639462846FFF73EFE814608B92046C0
:103B90003BE00146002332464046FFF711FF054651
:103BA00008B9484631E03B7CDFF8749013F0010F10
:103BB00023D005F091F9184BB0FBF3F7314607FB22
:103BC0001307404609F086FD044618B9134903203F
:103BD000FDF70AF800F154063046FCF781FF40F289
:103BE0000223A4F86A30E566B9F9003004F16802EE
:103BF0003946304608F03AF809E00146B9F90000C4
:103C000000F09FFB002802DC2846FFF7F7FE03B018
:103C1000BDE8F0838C0F010840420F00A5070108A2
:103C2000841000202DE9FF4707460D46904699462F
:103C3000FEF742FF824618B92A490320FCF7D4FF59
:103C400035B92A4641463846FFF710F8054668B1AF
:103C500002A93846FFF704FF064650B1C1B2002260
:103C600002A8FFF727FE044620B935E006460446C1
:103C700000E00446BAF8C631DB0714D5082E0AD096
:103C80000823009300226B440321384600F074FBA4
:103C900080B208281FD1234602AA0F21002004F079
:103CA00095F9C0B1044621464046FFF78FFD064610
:103CB00088B101462B464A463846FFF781FE044646
:103CC00008B9304608E0084B0146B3F9000000F09F
:103CD00038FB002802DC2046FFF790FE04B0BDE868
:103CE000F08700BFA5070108841000202DE9F041EE
:103CF000437E23F007030B4305290446437620D077
:103D0000072903D004294BD1264E05E0B0F91A004B
:103D1000FEF7D2FED0F8D461234B04F13805B3F995
:103D200000702846FCF7DCFE40F21723A4F84E3062
:103D300004F14C023B4631462846BDE8F04107F00D
:103D400095BFB0F91A00FEF7B7FE032306462246D8
:103D500006F5E07584F89430B4F91A002346002182
:103D6000FFF760FF01212846FDF7F4FE0E4BD6F861
:103D7000D871B3F9008004F138063046FCF7B0FE84
:103D800040F21223A4F84E303046434604F14C0270
:103D9000394607F06BFF2846BDE8F041FDF70ABF42
:103DA000BDE8F081404B4C00841000202DE9F34128
:103DB0001B4D002918BF0D46002229468046FEF7FC
:103DC00055FF074670B169464046FFF749FE38B1D6
:103DD000C1B200226846FFF76DFD044618B91AE02B
:103DE000044600E004462046FFF72DFD064688B154
:103DF00001463B462A464046FFF7E2FD044608B925
:103E0000304608E0074B0146B3F9000000F099FA8C
:103E1000002802DC2046FFF7F1FD02B0BDE8F0818A
:103E2000AC0F0108841000202DE9F04F8BB0002763
:103E300091468A46039302900797FEF73DFE964B04
:103E4000064600F5E07801214046B94508BF99468D
:103E5000FDF780FEB6F8C65115F001051BD13446BA
:103E600006F5E377B3465C4500F0ED80627C9BF895
:103E700011309A4240F0E4805946204604F026FE74
:103E8000637C834200F2DC8000E01D463834A045AC
:103E9000E8D1079D4FE004F0E9F9054600284AD033
:103EA000846906F5E37BECB163689E4218D1AB6987
:103EB0009C4200F0D780A268996892F811E0487C93
:103EC000864540F0E38010460593049204F0FEFD21
:103ED000049A059B527C824200F2D88000E01F4683
:103EE0002468E0E74FF0010B05EBD4039A7D04F062
:103EF00007030BFA03F31A420CD0E0B202F054FDB0
:103F0000428A417C0346007C009704F0C9FA07907E
:103F100060B107460134102CE6D12A46A98A2869E7
:103F20003B4604F0E3FA0546079020B94046FDF70A
:103F300041FE384681E0B6F8C6311B0707D5294651
:103F4000B6F8C801FFF708FD0790F8B10546BAF1C9
:103F5000000F0FD14046FDF72DFE49460122029881
:103F6000FEF784FE012182464046FDF7F3FDBAF1DB
:103F7000000F10D008A90298FFF772FD58B1C1B226
:103F80002A4608A8FFF796FC079018B94046FDF7A7
:103F900011FE3DE00546B6F8C62102F01004A4B2B9
:103FA0000CB196F8CA4102F020039BB24BB1D6F88F
:103FB000D4313A498B4206D84FF47A7BB3FBFBFBF2
:103FC00003E09B4601E0DFF8DCB002F04007BFB23F
:103FD0002FB1D6F8D8714FF47A73B7FBF3F7039B80
:103FE00013B9B6F8CC2100E0002240460392FDF759
:103FF000E1FDB6F8C611039A019509122046009713
:104000005B4601F0C001FFF761FC0446079008B968
:10401000284612E0014653464A460298FFF7D0FC74
:104020000146079008B9204607E01D4BB3F9000090
:1040300000F087F900282BDC0798FFF7DFFC27E06A
:104040000BF1380B0FE72B462246394607A8FFF73E
:10405000D9FC00283FF41AAF079B002B7FF415AF63
:1040600028460DE03B46A268594607A8FFF7CAFC60
:1040700000283FF435AF079B002B7FF430AF384664
:10408000FFF7BCFC4046FDF795FD01E01B680FE71C
:104090000BB0BDE8F08F00BF9C0F010800A493D6C1
:1040A0008410002080EE3600F8B51E469F1C5B7819
:1040B0000446154613B96FF01500F8BD01F108006C
:1040C000FFF75AFC0028F6D17CB394F91030013385
:1040D00004D1A3681C78022C04D001E06468F3E7E3
:1040E000082C06D17378012B14D0022BE3D10824BD
:1040F00011E0853D022D1BD884B9727808236FF03A
:10410000010413FB024402FB036616F8013D2BB9C0
:10411000013CFAE70224853D022D09D822463946A2
:1041200006980AF051FB2046F8BD853D022DE4D9E2
:104130006FF08500F8BD70B51D465B7804461646E5
:1041400013B96FF0150070BD01F10800FFF714FC02
:104150000028F6D1882E27D1A91CA4B194F91030DB
:10416000013304D1A3681C78022C04D001E06468F8
:10417000F3E7082C06D16B78012B0ED0022BE0D18F
:1041800008240BE054B96C78E408023CE4B20B1943
:1041900013F8013C13B9013CF8E7022422460498C5
:1041A0000AF012FB204670BD70BDF8B517460D46EB
:1041B000FEF782FC7C78012C06460FD1862D0FD1AC
:1041C00000F5E07521462846FDF7C4FC7B681BBA64
:1041D000A6F8C8312846FDF7EDFC01E00020F8BD47
:1041E0002046F8BD2DE9F0415378042B86B00746F0
:1041F000154671D186294ED102F110084046FFF7CD
:10420000C7FB0646002846D13846FEF755FCB0F8F5
:10421000C631DA0703D595F90330002B3BDB414665
:104220003846FEF79FFC044618B1427CAB789A42B0
:104230002AD06B6843B31022002102A80AF0C2FB07
:10424000EB785B0616D4AA78414602A804F064FC19
:10425000EB78AA7803F0C00302A93846FEF74AFCBF
:104260000446002839D03846FEF726FC012103F029
:10427000CDFF09E00821009104AB0022384600F090
:104280007BF80028DFDA28E06B6833B91CB12146DF
:104290003846FEF757FC01261FE01BBA6361AA6887
:1042A000013312BAA2610CD00E4B69680E481B880C
:1042B00009BA41431BB204F1300204F11C0007F0BB
:1042C000D5FC237C23F07F03DBB22374EA7822F051
:1042D0003F0213432374DEE70026304606B0BDE8F4
:1042E000F08100BFD402002040420F002DE9F341CD
:1042F0000446884617461E4600F0E8FA0546E0B137
:104300004146204600F0D0FA691E0446304600F0CF
:104310006DFD94B1B4F90810ADF8027068460196CD
:10432000FDF7AEFD002803DC0021304600F070FDF3
:10433000204600F0DFFA0446EBE7284602B0BDE86D
:10434000F08107B540F20223019101466846ADF8BD
:104350000230FDF795FD03B05DF804FB07B540F2B0
:104360000123019101466846ADF80230FDF788FD52
:1043700003B05DF804FB000000B589B006930A9B0A
:10438000ADF81C304FF401738DF81410ADF8162001
:10439000ADF80630024605AB03A901A80293FDF76C
:1043A00093FDBDF80E2040F205239A4203D0044944
:1043B0000320FCF719FC049809B05DF804FB00BF6A
:1043C000A507010800B589B006930A9BADF81C301B
:1043D00040F203238DF81410ADF81620ADF8063026
:1043E000024605AB03A901A80293FDF76DFDBDF8D8
:1043F0000E2040F205239A4203D004490320FCF723
:10440000F3FB049809B05DF804FB00BFA5070108A1
:104410002DE9F04384680746208F638D8FB000F04C
:10442000280EADF818304EF0010E0E4611B96FF09F
:1044300015005DE091F91030013354D18D682B796E
:104440002A7813F0C00F03BF02F108035B1995F837
:1044500001C0294B18BF4FF0020C12B105F1080141
:1044600007E0420747BF04F12E01082204F12C01A6
:10447000022294F8360000F1010884F83680049096
:104480000DF12008BDF81800ADF80800ADF80400E3
:10449000CDF80CE0CDF800C0404604F09BF9814611
:1044A0000028C4D0304607A900F046FA0646E8B115
:1044B000816881E800032B7913F0C00FBB6815BF3A
:1044C0001A69DA680132013214BF1A61DA602368AE
:1044D000079A1B682046984700210446304600F0A2
:1044E00097FC204604E06FF04C0001E06FF068009C
:1044F0000FB0BDE8F08300BF7A0F01082DE9F0434B
:1045000087683B685C68002387B01A4619463846BE
:10451000A047041E15DD002322461946184600F068
:1045200085FB054668B13B6881685E6822466B463C
:104530003846B047B0F1000805DC0021284600F0FD
:1045400067FC002466E03E8F06F00206B6B2002E3D
:104550005BD1A86804F0D2F9044608B9014637E0F7
:104560000146C0EB08083246284600F079FB814638
:1045700008B90146E2E7866801AA04A9304604F0BA
:1045800033FA01AA044602A9304604F0DBF9002CF4
:1045900001DA00241BE00028FBDBC1B2E3B204AA6D
:1045A00002A800F013F906460028F2D0022C0CD124
:1045B0009DF81030FF2B08D19DF81130FF2B01BF63
:1045C0008268137963F07F031371344626B90021A2
:1045D000284600F01DFC1DE0B3689DF801209A718B
:1045E0009DF800205A710D4A12885A8097F8283099
:1045F0002B744946284600F0CBF9002373602B4604
:104600005A680AB11346FBE75E604146284600F04F
:1046100095FB2C46204607B0BDE8F083D40200206D
:10462000034B0360034B436081600020704700BF71
:1046300011440008FD440008F0B5254E8468338815
:10464000838195B00821054604A8FDF79FFC3088BA
:10465000204B6360A56000B200F090F8236820460C
:104660009B68984740F2032741F234266846FDF7DD
:104670008AFCBDF80230BB4213D0B3F5017F08D2EB
:1046800040F202229342F1D12B68019928469847C3
:10469000EAE70AD0B342E9D123682046DB689847AD
:1046A000E2E7236801995E6902E0236801991E69C7
:1046B0000B894A6809782046B04740F205230390E9
:1046C00002A96846ADF80A30FDF72CFCCCE700BF24
:1046D000D4020020D946000813B50346806879B992
:1046E00041F234230190B0F90C10ADF80230684665
:1046F000FDF7A4FB002822DC12480AF0F5FA1EE0C0
:10470000042919D0072913D0022918D143689847E2
:104710000446A0B103460C4990F9100040F2012272
:10472000FFF7E4FD014650B9204600F071FB06E0BA
:104730009A6901329A6102E05A6901325A6102B003
:1047400010BD00BFC00D01080000FFFF30B585B0EF
:10475000089C6CB1A5685DB10293074B009301946E
:104760000823FCF7E1FA0028D8BF6FF0150001E03C
:104770006FF0120005B030BD39460008074B10B588
:10478000B3F90040A04201D1002010BD14B16FF078
:104790000B0010BD1880FEF763F9F5E73C19002007
:1047A000044BB3F9003013B1038001207047184661
:1047B000704700BF3C190020034BB3F900301B1AAF
:1047C00058425841704700BF3C1900202DE9F04184
:1047D000174603F108020A440E46002180461D4692
:1047E00008464FF0FF3300F021FA00220446F8B1EA
:1047F00083681E705D705A805A719A711A71B8F18F
:10480000000F08D03EB180680278B24203D1414621
:10481000083009F0D9FF5FB155B1A0684378AB42C9
:1048200006D1037808332A463946184409F0CCFFEC
:104830002046BDE8F081000008B50C4BB1F9082016
:1048400053F822301B6A1BB909490320FCF7CCF945
:10485000C3B2042B9FBF074B53F820200A6043F8D4
:10486000201094BF00206FF0150008BD2003002029
:10487000A507010840190020C3B2042B11D8094A2A
:1048800052F820308B4206D11B6842F82030704726
:10489000914204D013461A68002AF9D101E00A684F
:1048A0001A60704740190020C3B2042B09D8064B88
:1048B00053F8200020B143688B4203D00068F9E729
:1048C00070470020704700BF40190020C3B2042B7E
:1048D0000BD8074B53F8203000202BB15A681B68C7
:1048E0008A4208BF0130F8E770470020704700BFD8
:1048F0004019002028B14368006810B14268934213
:10490000FAD1704749B190F91030032B03D0042B32
:1049100006D103F001BF08F0BFBD6FF0150070476E
:104920006FF00100704728B190F910308B4201D030
:104930004068F8E77047000070B504460E4619B9A4
:1049400012490320FCF750F910B90020306070BD07
:1049500001460025496801350029FBD16FF00103AC
:10496000EA00204600F062F90028EED08368002BB0
:10497000E6D00833A26843F8082CE268646843F87C
:10498000042C0833002CF5D1356070BDA507010853
:1049900010B504468C42084601D1646808E02346FD
:1049A0005A682AB1904201D01346F9E742685A602A
:1049B0000021416000F02CFA204610BD70B555680A
:1049C00004460846EDB129464B680BB11946FBE792
:1049D0001CB91A490320FCF707F90028F9D0002A6E
:1049E000F7D043685360844206D023465E6826B100
:1049F000B04219D03346F9E7144653684B6055600E
:104A000015E0002CE5D00029E3D0002AE1D04B6866
:104A100053608C4206D02346596841B1884205D084
:104A20000B46F9E7144602E05A60E6E75A600021B7
:104A3000416000F0EDF9204670BD00BFA5070108F8
:104A400070B503461A4A072B88BF033310688CBF22
:104A500023F003030823002140B34468A34202D992
:104A600001460068F8E7E41A072C0344114E05D804
:104A7000046809B9146011E00C600FE0C6F1080584
:104A80001D44B5F5C05F02D90021116003E009B9EA
:104A9000136000E00B60026883E81400064A9B1B69
:104AA00011889BB2994201D2138070BD70BD00BFC6
:104AB000581900205C1900205419002001210148D8
:104AC000FDF748B85C310020204A38B5831AB3F5A9
:104AD000C05F39D21E4D2C68002324B1844202D21B
:104AE00023462468F9E707298ABF0331082121F00A
:104AF00003010460141AC1F5C0522244072A98BF6A
:104B0000891841600BB9286011E05A6818601A448E
:104B1000821A072A0BD818B90E490320FCF764F84B
:104B2000026841681A60C21A0A445A60184603684B
:104B300053B1426802449A1A072A05D81A680260DB
:104B40001A1A5B681344436038BD00BF5C1900202B
:104B500058190020A50701082DE9F84381461420C3
:104B60000F4616469846FFF76BFF0446D8B15EB174
:104B70003046FFF765FF054638B920461421FFF798
:104B8000A3FF2846BDE8F88335460123C4F8049006
:104B9000A560E66084F81080236027B1324639466C
:104BA000284609F011FE2046BDE8F883F8B50F4D00
:104BB00004460026CCB1631BB3F5C05F03D30C4998
:104BC0000320FCF711F894E88800012B09D1E16873
:104BD000A0682660FFF778FF14212046FFF774FFD6
:104BE00001E0013B23603C46E4E7F8BD5C1900208E
:104BF000A507010808B5FFF761FF094A094B1360D3
:104C0000182100221A705A709A70DA701A7159714C
:104C10009A71DA710448BDE80840FCF7CBBF00BFC9
:104C2000581900205C1900205C310020B2F5C05FEB
:104C3000F8B505460E4614461F460DD8FFF73EFF51
:104C400022463B4631462846FFF786FF0446034886
:104C5000FCF7B0FF2046F8BD0020F8BD5C31002015
:104C600007292DE9F84388BFCF1C0D468CBF27F0DC
:104C70000307082704469146FFF720FF2DB124B112
:104C8000E3689D4201D8A3682BB92B48FCF792FF3B
:104C90000020BDE8F8831420FFF7D2FE0646002866
:104CA000F3D0E3689D422ED0AF4202D85A1B072AA8
:104CB00029D82846FFF7C4FE074610B9142130460C
:104CC0000BE0E068401BFFF7BBFE804640B91421B3
:104CD0003046FFF7F9FE29463846FFF7F5FED4E7E0
:104CE0002A46A168384609F06FFDE268A168521BA8
:104CF0002944404609F068FDE168A068FFF7E4FE3A
:104D0000C4F8088005E0A7689D4214BF7B19002302
:104D1000A360E36808485B1BE3606368736001237A
:104D2000B760F56086F8109033606660FCF742FF6C
:104D30003046BDE8F88300BF5C310020072970B51C
:104D400088BFCE1C04468CBF26F0030608260D46FD
:104D5000FFF7B4FE1CB922490320FBF745FFE368C7
:104D6000A06813B90028F6D106E00028F3D01D4A48
:104D7000821AB2F5C05FEED29D422CD02DB930B16F
:104D80001946FFF7A1FEA56024E09D4202D8991BB9
:104D9000072917D82846FFF753FE064620B91248C0
:104DA000FCF708FF0C2070BDA16829B1E268AA4297
:104DB00028BF2A4609F008FDE168A068FFF784FED5
:104DC000A66007E0033323F003039E4202D230447F
:104DD000FFF77AFEE5600448FCF7ECFE002070BDAA
:104DE000A50701085C1900205C31002038B5044695
:104DF0000D46FFF763FE24B123682B4423606468EB
:104E0000F9E70248BDE83840FCF7D4BE5C31002029
:104E100010B50446FFF752FE2046FFF7C7FE0248D2
:104E2000BDE81040FCF7C6BE5C31002038B5044632
:104E3000FFF744FE0CB1E26822B90E48FCF7BAFE57
:104E4000002038BD2368012B0FD994F91030A168D8
:104E50006068FFF781FE054610B12368013B2360BF
:104E60000448FCF7A7FE284638BD0248FCF7A2FE1E
:104E7000204638BD5C310020F8B5002607460446C0
:104E80003546002C48D02946E268294809F0A2FEA0
:104E900094F910104B1C052B31D8DFE803F0060302
:104EA0000F182028002123482AE04FF0FF31224824
:104EB00009F090FEA06808F03FFD28E001211F489E
:104EC00009F088FEE168A06806F03AFC1FE00221C4
:104ED0001B4809F07FFEA06803F07AFF17E003216A
:104EE000184809F077FEA06803F060FC0FE0042189
:104EF000154809F06FFEA06806F060FE07E0134851
:104F000009F068FE1022E168A06803F0ADFFE368D5
:104F1000646801351E44B4E7294632460C4809F05E
:104F200059FE21463846BDE8F840FFF771BF00BF83
:104F3000E60D01080B0E01081F0E0108330E0108D3
:104F40004B0E01085E0E0108730E0108850E010864
:104F50009B0E010800B595B0082104A8FDF716F8CE
:104F60006FF08503039340F20523ADF80A306846DD
:104F7000FDF709F8BDF802306FF400721344032BFB
:104F800011D8DFE803F002040B0B094800E00948E0
:104F900009F0AAFE0198FFF76FFFE8E702A968464B
:104FA000FCF7C0FFE3E7044809F09EFEDFE700BF1F
:104FB000C80E0108E00E0108F70E01081FB50A4CE3
:104FC000B4F9003063B9094A0193094B0292009386
:104FD000062208234FF4C0610648FBF7A5FE208097
:104FE000B4F9000004B010BD603100201E0F0108AC
:104FF000554F00086231002007B501A8FFF7D0FB2C
:10500000BDF9040000F006F903B05DF804FB0000F0
:105010002DE9F043082187B07648774C774FFCF7AD
:10502000B5FF40F20523ADF81230264602A8FCF782
:10503000AAFFBDF80A30B3F5017F09D840F2032278
:10504000934280F0CF8040F20122934277D0EDE787
:10505000B3F5106F04D040F60112934264D0E5E737
:10506000674D05F1900815F8013CD3B1D5F817301C
:10507000022B0DD9042B05D8D5F813302946986991
:1050800000F0E0FAD5F81730023BC5F8173008E019
:10509000D5F81390681F01F0C7F80021484601F0C9
:1050A00051F93035A845DED16378ABB394F98C3033
:1050B000002B20DC96F83730022B18D894F83510E6
:1050C00051BB94F83430032B07D93C2384F8373094
:1050D00084F8341084F835101EE0013394F8292048
:1050E000206A84F8343000F0ADFD032300E0023B79
:1050F00084F8373010E0E269002ADBD1218E4FF6C8
:10510000FF729142D6D1023B5BB2002B84F88C3007
:10511000D0DC394801F0E3F8B7F90030394A3A49B0
:105120003A4806F0A3FD81E7039800283FF47EAFDC
:105130004369002B3FF47AAF06F0E2FC76E7039D6B
:105140001DB933490320FBF74FFD02212846FFF725
:10515000EAFB4FF0FF3180462846FFF7E4FBB8F149
:10516000000FEED018B18368B3F9021000E00146D9
:10517000A868D8F808204378032B2ED8DFE803F07E
:10518000020D182393885BBA9BB20093043002F19E
:105190001803083200F098FA1FE093885BBA9BB2BC
:1051A0000093043002F11803083200F0A9FB14E068
:1051B00093885BBA9BB20093043002F11803083263
:1051C00000F0AAFE09E093885BBA9BB2009304301A
:1051D00002F11803083200F0F9FE00212846FFF71B
:1051E00017FE23E76FF0850304A902A80593FCF7D7
:1051F00099FE1BE764370020603C002062370020E6
:10520000B53700203002002080841E00483800207E
:10521000A50701087FB51C4CB4F90050064625BB14
:105220001A4B1B481D701B4B02931B4B009301959F
:10523000082305224FF48061FBF776FD208000B340
:1052400016499B22088103204A60FFF7F5FA00F017
:1052500005FF134A13491448B4F9003006F006FD5F
:1052600080222946114809F0ADFB00238022104915
:105270003046FDF73FFC00200D4900F0E3F9B4F99A
:10528000000004B070BD00BF62370020403800202D
:105290005C380020360F010811500008A4370020A8
:1052A0003002002080841E0048380020F03C00209E
:1052B000260F0108012380F82F30002380F82C30BE
:1052C00080F82D3070473C2380F82F30002380F881
:1052D0002C3080F82D30704710B501210446094864
:1052E000FCF738FC084B1878421C1A7014B140F0D7
:1052F000800401E000F07F040248FCF75BFC2046DC
:1053000010BD00BF443800204038002013B50C46C3
:1053100012B11846FFF7E0FF2146022201F0E2F841
:10532000044678B30022032180F8252080F8271056
:10533000012314220A2180F8243080F8262080F8E6
:10534000281084F82F3084F832304FF4807323868D
:1053500094F83630052043F0030384F8290084F8DC
:1053600036303C20094B6085F02084F82E00B3F9DC
:10537000000001910092082340F6011204F1380167
:1053800006F0E4FB204602B010BD00BF62370020EB
:105390000021FFF73DBD10F0800F4BB202D0002B73
:1053A00011DA01E0002B10DB884204D2C1F1800346
:1053B00003440F2B09DD884205D9401A0F28CCBFC2
:1053C0000020012070470020704701207047000036
:1053D000F8B5074615461E460C4639B92046194908
:1053E000FDF7E8FB044608B9384625E035B916490B
:1053F0002046FDF719FC05460028F5D0114A29463C
:10540000002E18BF32463846FDF7D4F9064600286C
:10541000EAD000231A4619461846FFF7D7F98368E1
:105420000A495C8005464660034640F2022202209B
:10543000FEF75CFF20B92846BDE8F840FFF7A8BF9B
:10544000F8BD00BF260F01087C0F01080000FFFF18
:10545000002370B510220C4619460646FFF7E6FBFE
:10546000054618B93046FFF793FF24E0836804220D
:105470001A7000210E225A709970A27FDA70E27FB2
:105480001A7194F820205A71A269B2F88A2052BA8F
:10549000DA80A269B2F8882052BA1A81A269D2F8D9
:1054A00084201288197352BA5A8194F821205A73B1
:1054B000628C52BADA81284670BD002370B5202272
:1054C0000E4619460446FFF7B1FB054618B92046BB
:1054D000FFF75EFF1EE08068082303701E23437001
:1054E0004023C37033695A6942609A6982605B7C69
:1054F0008370002100F11004017341738173C17343
:105500001022204609F05EFA336931465A7C204663
:1055100003F002FB284670BD2DE9F3410F46044617
:10552000002800F0898090F8363003F0020300F183
:10553000080603F0FF0533B131460020FFF7BDFF39
:105540000546002878D094F83630DB070CD528467D
:105550003146FFF77DFF054600286DD094F83630C0
:1055600023F0010384F83630002318221946284618
:10557000FFF75CFB804608B9284637E0836822784D
:105580001A7094F82E205A7094F83220022A04D10E
:105590004FF0FF329A70DA7002E0228E52BA5A80CF
:1055A00094F8802094F82F10D20042EAC11294F8A7
:1055B00025100A431A7194F824205A7100229A7116
:1055C000DA713546083304F1180E2A4603CA7245CB
:1055D00018605960154603F10803F6D1042301222F
:1055E0009B21404607F048FF28B9404602B0BDE87D
:1055F000F041FFF7CDBE03460022D9685B680A443C
:10560000002BFAD10E4B17B13978FF290DD19969CA
:1056100001319961D9690A44DA61B4F92C10009614
:105620003B460022FFF7D4FE06E0196901311961FB
:1056300059690A445A61F0E702B0BDE8F08100BF41
:10564000F03C0020F0B51E4B85B0002205461868DE
:1056500003900F460A239B21104607F00DFF0646D4
:1056600058B38068002404714471042203A90630F1
:1056700009F0AAF832462346D16852680B44002A42
:10568000FAD1104A17B13978FF290FD1916B013146
:105690009163D16B0B44D36305B1083500220095AB
:1056A0003B4611463046FFF793FE06E0116B013191
:1056B0001163516B0B445363EEE705B0F0BD00BFBF
:1056C0003A0F0108F03C002030B41948BDF80850EA
:1056D0005BB11978FF2908D0046A01340462446A76
:1056E0002C444462052D07D820E0846A013484628A
:1056F000C46A2C44C462F5E71B780E48FF2B09D11D
:1057000043789BB190F83230022B0FD0383030BC48
:1057100006F006BA43784BB190F8363043F00103F7
:1057200080F83630114630BCFFF7F6BE30BC70470B
:10573000F03C0020603C00202DE9F04F8BB00026AB
:10574000159F07933E600C46154600F048FF8246C1
:10575000002800F0CF80B0464FF47A7B079B43458A
:1057600040F2C8802B78082B00F2BD80DFE803F000
:10577000050FBBBB147698BB4C003B6808F10108D1
:1057800043F001033B601FFA88F80135E6E73B6808
:1057900043F002033B60A6E03B6843F010033B602C
:1057A00094F8363043F0010384F83630688940BA03
:1057B00080B200F05BFC10B1C4F8840003E000F09C
:1057C00055FCC4F88400E87884F8260095F804E0D5
:1057D00084F827E0697984F82810EB885BBAA4F88C
:1057E0008A302B895BBAA4F888306B7B84F8293027
:1057F000EA8984F83900012352BA03FA0EF362856C
:10580000E36384F838106EE03B68B4F92C0043F48D
:1058100080733B6094F83630082143F0020384F82B
:105820003630009108AB0022FEF7A6FD002802DA10
:10583000EB785B0657D5082208A905F1100905F198
:10584000180008F0C1FF0023AA78B4F92C004946DB
:10585000FDF750F9002846D0A06144E03B68B4F958
:105860002C1043F020033B6094F82900638DEA7804
:1058700043430BFB03F3002E08BF2E460493802AFC
:105880004FF0010394BF12060022149803931023D3
:105890000190009202932A1D184807F045FA22E071
:1058A0003B6843F040033B600EB900261BE04FF01D
:1058B00010096A79638DCDF8009053430BFB03F315
:1058C000029395F902300D48DB43DB0F0193311D44
:1058D000149B102207F0B0FA737802331E44337819
:1058E000052BE6D0E1E76B78023398441FFA88F87D
:1058F0001D4433E750460BB0BDE8F08F5010002038
:105900002DE9F04786B017460022039204460D4663
:10591000BDF83860A74A5BB11B78FF2B08D013682D
:10592000013313605368334453601B2E07D83DE1A5
:10593000936801339360D3683344D360F5E71C3E2A
:1059400003A92078B6B200F0ABFB002800F08980F4
:1059500063885BBA9BB24FF6FF72934200F02381DB
:105960002379DDF80C80C3F3C20388F8803000206F
:1059700000F07CFBC8F884004DB928468E49FDF73D
:1059800019F9054618B98D490320FBF72DF92A4668
:10599000002304F10801039800F0B2FB039D06AA5E
:1059A00005F10808002342F8083D3946404600F05A
:1059B000E7FB18B9049B002B00F0F580637885F8AD
:1059C0002E3023790399DB0985F82F30237903F0F2
:1059D000070385F825306388049A5BBAD38206AB47
:1059E000002243F8042D012001930097334604F16F
:1059F0001802FFF7A1FE002800F0D580059810F0EE
:105A0000100407D1039800F06AFC39462046FFF7DE
:105A100019FECBE0AB6943B94146B5F92C00FDF75F
:105A200003F9002800F0BF80A8614046FFF742FC60
:105A3000634A95F82730B2F9000095F828200192C2
:105A400095F826200092012202FA03F305F13801AD
:105A500040F6011206F07AF80499404600F072FC14
:105A6000A4E0039D002D00F0A18005F1080810229C
:105A700004F10801404608F075FE8146002840F018
:105A80009580039A237992F88020C3F3C2039A4247
:105A900040F08C80627895F82EA010465146FFF7B2
:105AA0007AFCC8B195F83230012B0FD1130601D51D
:105AB000FF2A00E07F2A1ABF0132D2B24A4685F897
:105AC0002E2005F1380006F02BF80BE085F82E208B
:105AD000404600F015FC05E011465046FFF75BFC20
:105AE000002837D195F83230012B0BD163885BBA8F
:105AF0009BB24FF6FF72934205F138002CD006F0AE
:105B000058F853E006AA002342F8083D39464046BB
:105B100000F036FB049B08B9002B47D01BB105F100
:105B2000380006F046F8049900293FF42CAF63884A
:105B30005BBACB82404600F005FC049B1A7972B92F
:105B400063885BBA9BB24FF6FF7293422ED12A8EC6
:105B50009A422BD005F1380005F0E2FF26E0EA6911
:105B6000934223D15A7D63799A4202D04046FFF78F
:105B7000A1FB049B62795A7523790399DB0985F8A7
:105B80002F30237903F0070385F8253006AB002278
:105B900043F8042D012001930097334604F11802C5
:105BA000FFF7CAFD10B9039800F099FB06B0BDE8F5
:105BB000F08700BFF03C0020260F0108A507010870
:105BC00062370020F8B500230C4616461946142209
:105BD0000746FFF72BF8054618B93846FFF7D8FBFC
:105BE00011E0836805221A7012225A7000229A70FE
:105BF000DE702146043304F1100251F8040B43F81F
:105C0000040B9142F9D12846F8BDF8B500230E46A1
:105C10001546194606220746FFF708F8044618B944
:105C20003846FFF7B5FB0AE0836806221A700422A3
:105C30005A70ED0100229D70DA701A715E71204673
:105C4000F8BD00002DE9F04F8DB00E4606920546D6
:105C5000002800F0FD8090F83230012B00F0F88031
:105C600021B9C669002E00F0F38005360CA805F1B5
:105C700008030024194640F8044D059309940A943A
:105C8000FCF7ACFF0B9B002B00F0E2800121724877
:105C9000DFF8D8B1FBF75EFFA04604940394DBF86D
:105CA00008309C4268D2DBF8007007EB4417D7E954
:105CB000022313435ED0BB69DA070CD4039BD3B92C
:105CC000012206991846FFF7A0FF0A9088B962489A
:105CD000FBF770FFBCE0049B83B91A46069918468F
:105CE000FFF793FF804609900028F0D0012304932A
:105CF00004E0012303930DF1280901E00DF12409CB
:105D00007B699A78FF2A03F1020A07D1D87800F05C
:105D10000F00A0F10E035842584120E008224F49DD
:105D20000793504608F01EFD079B08B9002016E0B7
:105D30009A78FF2A04D1DB7803F00F03022BF5D009
:105D400010224749504608F00DFD0028EED01022E1
:105D50004449504608F006FD003018BF012048B104
:105D6000FA7CD9F800005146FFF72CFFC9F8000073
:105D70000028ACD0013492E73748FBF71BFF0A9BA1
:105D8000B8F1000F02D0C8F8043000E00993802277
:105D90000B990998FFF716FF04460990002857D081
:105DA00095F90070002F07DA002310220599FEF7FD
:105DB0003DFF0A9030B30990DDF8248000230422CF
:105DC00019464046FEF732FF04460A9008B940469D
:105DD00019E083682A781A70002FB4BF402200228D
:105DE0005A705A78099062F07F025A7095F8332001
:105DF000DA7000279F70022204239B2107F03CFBEE
:105E00000A9018B92046FFF7C3FA21E0099002462C
:105E10003B46D16852680B44002AFAD13278FF2AF7
:105E2000114A0ED0116D01311165516D0B4453654E
:105E3000059BB5F92C10009300223346FFF7C8FAF2
:105E400006E0916D01319165D16D0B44D365EFE7AB
:105E50000DB0BDE8F08F00BF5C1000207C0F010882
:105E6000CC0F0108DC0F0108F03C0020501000208E
:105E70002DE9F7430E4691460446002846D090F996
:105E80000080B8F1000FACBF0823182303229B2128
:105E9000002007F0F1FA0546002837D087682378FC
:105EA0003B71B8F1000F09DA80237B71102204F1F5
:105EB000080107F1080008F087FC01E000237B716E
:105EC000002387F80690FB712A46D16852680B447C
:105ED000002AFAD10F4A16B13178FF290FD1916FFC
:105EE00001319167D16F0B44D367B4F92C1008349A
:105EF0000094334600222846FFF76AFA06E0116F45
:105F000001311167516F0B445367EEE703B0BDE8F1
:105F1000F08300BFF03C00202DE9FF411746054605
:105F2000BDF82840284A8BB11B78FF2B0ED0136C8C
:105F300001331364536C234453646B7813F0400FA4
:105F40000CBF082318239C423AD306E0936C01331C
:105F50009364D36C2344D364EFE7287800F0C2F84D
:105F6000064668B36B785B0605F1040106F1080884
:105F700001D4083C07E01022404608F0F3FBF8B9D2
:105F800005F11401183C96F83220022AA3B217D06A
:105F900004AA002042F8040D0097019202200A464C
:105FA0003146FFF7C9FB58B195F90130002B04DAEF
:105FB000EA7839463046FFF75BFF4046FFF77AF94B
:105FC00004B0BDE8F08100BFF03C002070B5224A6B
:105FD0000446BDF81000A3B11978FF2911D0116E45
:105FE00001311166516E014451661B78FF2B32D08E
:105FF00094F90130002BACBF0823182398422AD112
:1060000006E0916E01319166D16E0144D166ECE7F4
:10601000207800F067F80546E8B194F90130002BCC
:1060200005F1080602DBE37843B90CE01022211DDC
:10603000304608F097FB0028F5D070BDA27895F89F
:1060400033309A4207D1012385F835303046BDE818
:106050007040FFF738B970BDF03C002008B500F083
:1060600021FB014B186008BD703D0020054B1B68EB
:106070000BB900F017BB1A8882420CBF18460020EB
:10608000704700BF703D002090F83220022A02D1F4
:10609000383005F08BBD0149FFF73EBA260F0108E5
:1060A00010B500230E4A0B6054780CB90A6004E066
:1060B0001478844201D10A600FE00B686BB118704C
:1060C0000B68012058700B6800224FF48071A3F810
:1060D0008A20A3F88810DA6110BD184610BD00BFF1
:1060E000603C0020054A53782BB1137883420CBFE3
:1060F0001046002070471846704700BF603C0020E3
:10610000F8B5044608B1407818B91B490320FAF7DE
:106110006BFD0D4604F1080701F1100E286869684F
:106120003E4603C6083575453746F7D14FF6FF7131
:1061300021861249E164142184F82610032184F891
:1061400027100A2184F82810052184F829103C2101
:106150006185F020002184F8330084F8321084F83F
:10616000241084F83410246584F835102462A28544
:10617000A3610120F8BD00BFA507010889600008E0
:106180002DE9F8430026264F166080460D4614463A
:106190004FF0010917F8013C33B9B9F1000F14D0E1
:1061A0007A1F2260994610E0D7F8133043450CD18E
:1061B0002946384602F075FC38B11A4A302303FBF1
:1061C000062626600020BDE8F8830136032E07F17D
:1061D0003007DFD1206800B3C0F8188023680022A0
:1061E0001A60D8F8143033B11A680AB11346FBE7C5
:1061F00022681A6002E02368C8F81430236801227C
:106200001A7123682946053305F1100251F8040B71
:1062100043F8040B9142F9D10120BDE8F88300BF97
:10622000B5370020B037002030B5044687B018B924
:1062300020490320FAF7D8FC85696B6998422AD176
:1062400010221D491D4806F040FE2368D3B10020EE
:10625000FBF798FA22681A4BB0FBF3F0D369B5F953
:106260002410181A4FF47A7358430532012303930C
:106270000192102300220490009202930E4A0F48CC
:1062800006F052FD6B699C4205D123686B6108E002
:10629000944204D013461A68002AF9D101E022681A
:1062A0001A6030220021204608F08CFB012007B044
:1062B00030BD00BFA5070108CC0F01085010002019
:1062C00040420F0038B50446406920B10568FFF729
:1062D000ABFF2846F9E74FF6FF73238538BD10B5AD
:1062E00004460830FFF7EEFF04F1380005F05EFCCD
:1062F00090220021204608F065FB012010BD00001F
:1063000010B5037F013303774369044633B1FFF7C8
:10631000D9FF102209490A4806F0D7FD228D4FF611
:10632000FF739A4208D0238504F1300005F0F8FB92
:10633000A369052283F88C2010BD00BFCC0F010893
:10634000501000202DE9F04F0A4689B00446E1B113
:10635000438C90F821105943D16141698A4214D18C
:10636000B0F9241090F8210043434FF47A7043436E
:10637000053204930123039301921023002200921B
:106380000293564A564806F0CFFC6369228D069266
:10639000002B00F099804FF0010B002266696261CA
:1063A00092469146002E36D00AF1010A3546002762
:1063B0002D6801370DB9D84610E05F45F8D1FAE7EE
:1063C000B8F1000F0DD12A4635463668013FB9F1C4
:1063D000000F1CD0C9F80050A9461546002FEFDC6D
:1063E00001E02DB9EFE7B8F1000F12DD8DB157B123
:1063F000A2690793D2F884202946D2683046904794
:106400000028079BDFDD2A6808F1FF38DFE76561B8
:10641000E2E72E46C6E7B9F1000F01D0C9F80060E7
:10642000BAF1010F4FEA4B0BB7DC6269D08A4FF625
:10643000FF71884248D0934223D0A06990F8802011
:10644000023A012A06D80022591DFFF7FBFB20461D
:10645000FEF730FF638C94F82120B4F92410204813
:106460005A434FF47A73534362690493053201230C
:10647000039301921023002200920293174A06F020
:1064800053FCA3696069D3F8843000215B689847A6
:10649000069B2085834203D004F1300005F040FBC9
:1064A000606978B1A369228DB3F88810C38AB2FB02
:1064B000F1F2B3FBF1F39A42056801D8FFF7B4FE9D
:1064C0002846EEE763692BB9204609B0BDE8F04FD6
:1064D000FFF716BF09B0BDE8F08F00BFCC0F010871
:1064E00050100020334BB3F900302DE9F34106463C
:1064F0000C4615460BB9002058E0002301930B7899
:10650000FF2B0BD14B7803F00F030E2BF3D1214659
:106510006846FCF74FFB074608BBECE70822264914
:10652000204608F01FF9A0B12378FF2B04D163782F
:1065300003F00F03022B0CD010222049204608F054
:1065400011F930B110221E49204608F00BF900283D
:10655000DDD123780433DBB2012BD8D9CBE7DDF8CA
:106560000080B8F1000FC6D001A93046FFF798FDB2
:106570000028C0D00020019EFFF778FDC6F88400F7
:1065800001984FF48073A0F888300023A0F88A3077
:10659000214680F8805043463A46FFF7B1FD044655
:1065A000019814B9FFF79BFEA5E7006202B0BDE8B1
:1065B000F08100BF623700207C0F0108CC0F01087A
:1065C000DC0F0108022380F82A3000218069FEF7E1
:1065D000A3BF002380F82A30303005F0A1BA70B58F
:1065E00000249C422ED21578082D25D8DFE805F02E
:1065F00005242424091319240E000134A4B2013205
:10660000EFE7012822D155780E2D14E001281DD185
:1066100055781E2D0FE0022818D15578122D0BD970
:1066200014E0022812D191F880505678012D14BF41
:1066300004251425AE4209D1557802352C44A4B264
:106640002A44CEE70CBF0120002070BD002070BDA1
:10665000704711B970B1C18A00E020B183699B69AC
:10666000B3F8880001E04FF480700844814201DCF7
:1066700080B270474FF6FF707047C28ACB8A9A4249
:1066800003D38CBF0120002070474FF0FF307047CC
:1066900038B50446FFF7F1FF0028CCBF0846204676
:1066A00038BD704700487047380200200021FEF7CF
:1066B000AFBB00002DE9F0419CB000230993A3F586
:1066C00080330A937F4B08211B88ADF82C300CA82F
:1066D000FBF75CFC09A90120FEF7AEF840F20523A8
:1066E000ADF8163040F2032440F2012503A8FBF771
:1066F0004AFCBDF80E30B3F5017F09D8A34280F003
:10670000D880AB420CD040F2022293426ED0EDE72B
:1067100040F225229342E9D1049800F0EDF9E1E737
:10672000049D2846FEF782FB044600287ED0012106
:10673000FEF7F9F8054608B1C3681BB92046FFF714
:10674000B5FFCFE783681B78412B11D1FEF76EFBB5
:1067500005460028F2D001221146FEF781FA0146D3
:106760000028EBD02046FEF713F90223044631E05F
:1067700003F0D802C02A03D1204600F0B1FAB1E7F5
:1067800003F0E003602BD9D1002102232822084620
:10679000FEF74CFA079010B9079890B9CEE702AB14
:1067A0000093002321461A4607A800F0DFFC0146AB
:1067B0000028F1D001222046FEF752FA014618B90E
:1067C0000798FFF773FFB9E72046079AFEF7F6F838
:1067D000002304462B7440F2012223463A4902204A
:1067E000FDF784FD00287FF47DAFA7E7049DEDB1A0
:1067F000EB68072B1AD96B68C3B193F91030022BE1
:1068000014D12846FEF712FB044678B18768B7F921
:10681000020001F095FE61688046002619B1CB6840
:1068200049681E44FAE7B8F1000F01D1284686E70F
:1068300098F8043023B1204600F086FF70B97DE758
:1068400001231A460846FEF7F1F900283FF476AF17
:10685000636843606060836841221A706268002345
:106860001AB1D16852680B44FAE7B8F8021099429D
:1068700008D32146B7F90200FDF763FD00283FF772
:1068800031AF5BE7114B596800297FF457AFB6F57C
:10689000006FBFF453AF79889A8107A840F2252290
:1068A00019805C609E60ADF81E200893FBF78AFAA1
:1068B00018E76FF0850305A903A80693FBF732FBE1
:1068C00010E700BFD40200200000FFFF743D00204D
:1068D0001FB50A4CB4F9000000280DDC084B0293E8
:1068E00000230193074B0093032208234FF4806198
:1068F0000548FAF719FA208004B010BD8441002041
:106900003E0F0108B5660008843D002038B50E4BE7
:10691000142404FB00340546638A63B10020FAF7AF
:1069200031FF0A4BB0FBF3F0094B53F8253083429B
:1069300006D800236382637C23F01003637438BDA0
:106940001B1A638238BD00BF864100200087930375
:10695000C84200202DE9F041012180461048114D28
:10696000FBF7F8F8002426462746E0B2FFF7CEFFF3
:106970002B7C53B14146284602F0A8F82B7C834279
:1069800003D8B84284BF2E4607460134102C05F1C7
:106990001405EAD10248FBF70DF93046BDE8F08155
:1069A00008430020864100200F2838B5044615D83A
:1069B00001210B48FBF7CEF82046FFF7A7FF094B54
:1069C000142000FB043506482C7C1CB1FBF7F2F8C0
:1069D000284638BDFBF7EEF8204638BD002038BD0C
:1069E00008430020864100202DE9F8430F28064681
:1069F000884615461F469DF820903FD8002A40D073
:106A000001212148214CFBF7A5F8002F4FF014037A
:106A100003FB064308BF4FF00009802D88BF80228A
:106A20005F828CBF1A741D74B9F1000F02D046F05A
:106A3000100300E03346142000FB06444146637413
:106A4000204602F02EF8014640B91022204607F0F9
:106A5000B9FF227C4146204602F05EF80020FAF79A
:106A600091FE0B4BB0FBF3F00A4B0744064843F88A
:106A70002670FBF79FF82046BDE8F8830020BDE8AC
:106A8000F8831046BDE8F8830843002086410020C3
:106A900000879303C84200200021FEF7B9B9F8B57A
:106AA0000E4601784378174601F108020244054674
:106AB0000830FDF78BFE0446E0B18368B5F902208B
:106AC0005A802A791A716A795A71AA799A71B742E9
:106AD0004FF000013A464FF0010328BF3246084606
:106AE000FEF7A4F8054620B92046FFF7D5FF284653
:106AF000F8BD60602046F8BD2DE9F04F054685B031
:106B0000B0F9000001F01CFDD5F80480D8F804406D
:106B100083464FF0000A1CB1E36864689A44FAE7C0
:106B2000BBF1000F05D14046FFF7B6FFC5F804B032
:106B3000D0E0B5F80C90B9F1000F42D1674FAE68C4
:106B40003B88D8F8080001333B80CAEB06039AB2B1
:106B5000BBF80230043B134403F0F8039B1A1FFAFE
:106B600083F909F104025146FFF799FF0346002813
:106B70003AD04268D2F808A076BAAAF800609AF82B
:106B8000002062F03F028AF800203A8852BAAAF840
:106B90000220D8F80470002F7CD0FA68B9680093FE
:106BA000C4EB0906964228BF1646201D34443246DF
:106BB0005044A4B207F008FEA145009B6AD97F6843
:106BC000E9E7D14580F08280BBF80260D8F8080080
:106BD000AF68053E06F0F806C9F10501721D514483
:106BE000FFF75DFF034628B96868FFF755FF0023EC
:106BF0006B606FE042689268511D009179BA118014
:106C0000117861F01F01117034494F440988CAEBB3
:106C1000070A49BA4FEADA0A518082F804A0D8F884
:106C20000470FFB1A1451BD0FA68A11889B289454B
:106C300013D2C4EB09041FFA84F9C9EB0204B4426D
:106C4000B9680098019328BF34462246494407F0AA
:106C5000BBFDA4B27F68019B05E07F680C46E0E7BE
:106C6000002400E03C46A64214D99FB1FA68019383
:106C7000C4EB06089045009BB96828BF90461819D8
:106C800044444246A4B207F09FFDA642019B01D0B6
:106C90007F68EAE71946BBF900000093FDF751FB56
:106CA0000028009B02DC1846FFF7F6FE002C9BD064
:106CB000AB8903951C44AC8140F2252302A8ADF8B2
:106CC0000A30FBF77FF8F9F7F5FF03E04046FFF7DE
:106CD000E3FE6C6005B0BDE8F08F00BF0C43002000
:106CE00010B58268137803F0F803C02B044606D071
:106CF000E02B0DD11379C268DB00053A02E0C268CF
:106D00000023043A60682146806800F013F82046AA
:106D1000BDE81040FFF7C0BE002203682BB1196820
:106D20009A80DA801A600160F7E7436070470021BB
:106D3000FEF76EB82DE9F04F8FB0814600209246E5
:106D400004911F468E68AA4DFAF71CFDA94A834696
:106D500005F190082C46606858B1A368C3EB0B039B
:106D6000934206D90292FFF7E2FF2046FFF7D4FFD5
:106D7000029A24344445EED199F800B009F1080391
:106D800007930BF108034B44069399F801300293E3
:106D900033885BBAC3F30A03059373885BBAADF813
:106DA000263000209BB20A93FAF7ECFC00230890EF
:106DB0001C4603936A68A846002A00F02581D26821
:106DC0000599914223D1EA8B0A998A421FD12A7FE1
:106DD00093451CD16A7F0299914218D15A4607996E
:106DE0000B9305F10C0007F0BDFC0B9B78B9029AE0
:106DF000069905F1140007F0B5FC0B9B38B97C4CE3
:106E0000039A242303FB0244089BA3604EE014B9B9
:106E10006A6802B92C463BB1A9689A68521A764949
:106E20008A4294BFA8469846039B0133042B0393E0
:106E300005F1240501D04346BCE784B9B8F1000F41
:106E400003D16E490320F9F7CFFED8F804000028DB
:106E5000F7D0FFF76CFF4046FFF75EFF4446002186
:106E60000223059A0846FDF7E1FE6060002800F065
:106E7000DD80836800210020C3E90001089BA36036
:106E80005A46079904F10C0007F09EFC029A0699F5
:106E900004F1140007F098FC9DF808306377BDF802
:106EA0002630E383002384F81CB0238425680FBBBD
:106EB0003379412B03D105360AF1FF331FE003F08C
:106EC000E003602B06F1040618D10EAB204643F810
:106ED000047D50F8042F0093D2680499042300F035
:106EE00045F900287CD00D9A28320AEB02030644AB
:106EF0001B1A05E005365346002201E053463A4688
:106F00006068C16803EB070E8E456AD81FFA87FEDA
:106F10000EF1FF31194489B26DB1B5F804804145D5
:106F2000C0F08280B5F806C0E6457DD8C6456FD171
:106F300061456DD178E01FFA83F80EF1FF314144CD
:106F4000DFF8C0A089B2AC460AEBCC05B5F806B0B4
:106F5000BBF1000F11D1ADB1E98021682960A5F81E
:106F600004E0218C256080684144174421849A1AEA
:106F70003146384407F028FC04E00CF1010CBCF168
:106F8000340FE1D16368228CDB689A424ED1637F73
:106F9000217F04F1140204F10C00FDF717FCF8B195
:106FA0008368B9F902205A8099F804201A7199F877
:106FB00006209A7199F805205A710023436063688E
:106FC0002BB15A680AB11346FBE7586000E06060D5
:106FD00063680B4940F201220220FDF787F910B9DE
:106FE0006068FFF7A4FE2046FFF796FE1EE000BF94
:106FF00010430020C0C62D00FEFFFF7FA50701083B
:107000000000FFFFA0430020002C7FF404AF01E745
:10701000FFF78DFE2046FFF77FFE3B465246049960
:107020004846FFF787FE01E02D6875E70FB0BDE821
:10703000F08F00BF037823F00F0343EA11130370AE
:10704000437803F00F0343EA0111417070470000D9
:107050000822014907F0B8BB7C0F0108102200216B
:1070600007F0B0BC10B508220949044607F07AFBC6
:1070700048B12378FF2B08D1607800F00F00831E01
:107080005842584110BD012010BD002010BD00BF66
:107090007C0F010873B51546194A04460E46106860
:1070A00051686B4603C32CB3637CDB0624D4227C7B
:1070B000802A1DD0402A1FD9D208D11F501C294434
:1070C000C2F10F02304407F04DFBA8B9237CD90868
:1070D0000D44725C15F8080C03F0070302A90B4479
:1070E000424013F8083C1A420CBF0120002004E083
:1070F000012002E0204600E0002002B070BD00BF89
:10710000420F01080023042A10B54370037016D003
:10711000082A02D0022A26D118E00B7883F0020355
:1071200003704B7843708B788370CB78C3700B7986
:1071300003714B7943718B798371CB7911E00B78B3
:1071400083F0020303704B7843700223FF24002274
:10715000C470FE24827004714271CA5C82710B4457
:107160005B78C37110BD184610BD00002DE9F74FC4
:107170001E464B6800920F46D3F808A0D1F808B01D
:10718000019018B9C0490320F9F72EFD019B1B6837
:10719000002BF7D0DA68272AF4D90BEB06089D6894
:1071A00098F90130002B2B7803F00F0343F06003B4
:1071B0002B701BF8063003F01803ACBF0224032425
:1071C000082B27D017D8002B52D118F804102846C6
:1071D000FFF730FF08EB04014B7803F00F026B78E8
:1071E00013436B708978AA78E31C0A43AA7018F8D5
:1071F0000320043429E0102B2AD0182B38D1002189
:107200002846FFF717FF6B7823F00F036B700023FE
:10721000AB702CE018F804309B099B0043F060032E
:107220002B706B7803F00F01697018F8043003F0CD
:107230000F0308EB04020B436B705178AA78A31C70
:107240000A43AA7018F803200334EB7813430EE0C6
:1072500018F804102846621CFFF7ECFE6B7823F048
:107260000F036B700023AB70EB70144600E0EB7003
:107270001BF806305B075CBF18F80430AB711BF8D5
:10728000063003F0030358BF0134022B08D0032B50
:1072900008D0012B07D018F80430EB71013403E05B
:1072A000402300E0FF23EB7198F8013003F0400227
:1072B00002F0FF0972B118064ABF98F802000020D8
:1072C000000913F0300905D0FFF76EFB8146002856
:1072D00000F0318298F8013003F07003302B42D077
:1072E0000FD8102B1CD0202B26D0002B40F08C80E8
:1072F00008EB0401102205F1080007F065FA1034CC
:1073000082E0502B3BD006D8402B7DD105F1080000
:10731000FFF7A4FE78E0602B45D0702B62D073E0BD
:1073200005F10800FFF794FE082208EB040105F1BF
:10733000100007F049FA34E005F10800FFF788FE75
:107340004FF0FF320023EA746FF001022A752B74AC
:107350006B74AB746B75022208EB040105F1160027
:1073600007F032FA3CE0514605F1100011F8082B05
:10737000FFF7C8FE05F10800FFF76AFE44E0B9F127
:10738000000F3FF4FFAE082208EB040105F11000E6
:1073900007F01AFA99F81020494605F1080001F0A3
:1073A000BBFB083430E0B9F1000F3FF4EBAE4FF017
:1073B000FF320023EA746FF001022A7508EB040122
:1073C00002222B746B74AB746B7505F1160007F019
:1073D000FBF999F81020494605F1080001F09CFBE3
:1073E000023411E0B9F1000F3FF4CCAE514605F183
:1073F000100011F8082BFFF785FE99F81020494678
:1074000005F1080001F088FB98F8013059070FD505
:107410001A064ABF98F80200002000F00F0013F08F
:107420000B0F05D0FFF7C0FA8146002800F08381DA
:1074300098F8013003F00F030C2B00F27C81DFE899
:1074400013F00D001600250042007A015100610082
:1074500082000D009400A600B800C60008EB0401ED
:10746000102205F1180007F0AFF91034D9E005F14A
:107470001800FFF7EDFD082208EB040105F12000DC
:1074800007F0A2F93CE000BFA507010805F11800CC
:10749000FFF7DEFD4FF0FF32002385F823206FF069
:1074A000010285F8242085F8203085F8213085F800
:1074B000223085F82530022208EB040105F1260070
:1074C00007F082F93DE09AF800109AF8012008319F
:1074D000514405F12000FFF715FE05F11800FFF7F4
:1074E000B7FD9EE0082208EB040105F1200007F03B
:1074F0006BF999F81020494605F1180001F00CFBD2
:1075000008348EE04FF0FF32002385F823206FF01F
:10751000010285F8242008EB0401022285F82030BE
:1075200085F8213085F8223085F8253005F12600D0
:1075300007F04AF999F81020494605F1180001F0C2
:10754000EBFA02346DE09AF800109AF80120083145
:10755000514405F12000FFF7D5FD99F81020494668
:1075600005F1180001F0D8FA5BE005F11800FFF70B
:1075700075FDFF232B7618F804306B76611C05220D
:10758000414405F1230007F01FF9063449E005F1F5
:107590001800FFF763FDFF232B7618F804306B7695
:1075A000611C0322414405F1250007F00DF9043464
:1075B00037E005F11800FFF751FDFF232B7602237A
:1075C0006B7618F8043085F82730013429E005F18E
:1075D000180099F810A0FFF741FD99F81030402BE2
:1075E00084BF402389F81030FF232B7618F804302D
:1075F0006B7608EB040349465B78AB7699F810305C
:10760000EB7699F8102005F1580001F085FA211D5C
:107610000422414405F1240007F0D6F8063489F825
:1076200010A0009B13B9FB681B1B01E0009B283BCB
:107630005BBAAB801BF806305B077ED518F80430C8
:1076400003F0F803F02B78D1019BBD68D3F800A0BC
:10765000009BDAF80890344404F1010815F804B0EE
:107660004BB90099042308220846FDF7DFFA0028E9
:1076700065D0826802E009F1280200200BF00303C4
:10768000022B14D0032B1FD015F808101170012BFA
:1076900005EB04039978517004D0D97891700534C2
:1076A0001B790FE0DB780434A3F5805318E015F85C
:1076B0000830A3F580535BBA13802B1904349978F2
:1076C0009170DB78D3700DE015F808301909A1F539
:1076D000756149BA03F00F0302341180A3F5756395
:1076E0005BBA53801BF0040F03D00021FDF790FB21
:1076F00025E02B5D9371A31C2C446178D17118B1E6
:10770000F9680831C91A01E00099283949BA91800D
:10771000112189F806109288A9F8042018B1019A5D
:10772000C0F804A0106053B19C1B0C9B0C9A1B6802
:107730000833136001E0002003E0204601E000244C
:10774000F3E703B0BDE8F08F2DE9F04F4268D0F8C1
:1077500008909668D268002189B0824601230846C5
:10776000FDF764FA029038B38568AB4960232B704B
:1077700006F1080B00236B701022584606F0F2FF4A
:1077800038B15846FFF7E6F8804610B1437CD90679
:1077900001D44FF00008337EFF2B00F0628206F127
:1077A0001800FFF7D7F80746002800F05A82437CFC
:1077B000DA0640F1568201E0029858E2B8F1000F73
:1077C00004D098F811301B0703D15FB17B7C1C07F4
:1077D00008D06B7863F07F036B700023AB700324D9
:1077E00001E04746022431683378727821F4704111
:1077F00021F0FF011B01A9B943EA121313F0FF0F97
:107800002B7803D143F018032B7036E043F01003BC
:107810002B70737831781B09621C43EA01132B55D6
:1078200094B22AE05BB203F030011209114304F173
:1078300001010ED12B7843F008032B7032688BB214
:10784000317812BA8910C2F3034242EA81122A55F2
:1078500009E013432B55326889B212BAC2F30342CE
:10786000A31C6A549BB2326812BA120AEA549C1CD6
:1078700001339BB20022EA54A4B2B379112B6DD12B
:10788000DAF80430586883681A88B3F802E052BA0C
:1078900092B222F00F0C1FFA8CFC4FF2B0018C4513
:1078A0001AD19EFA9EF121F00F010904090C6145DD
:1078B00012D10322B271598849BA1FFA81FE198880
:1078C00049BA89B20EEB011101F5AA6119709979D3
:1078D0005970D979997026E09EFA9EFE0EF47F4E7B
:1078E000BEF5704F04D10122B2715A8852BA0CE031
:1078F00002F47F42B2F5704F0ED10222B2711A88A3
:1079000052BA1A709A785A70DA789A709A79DA704C
:10791000DA791A71052206E00022B2719A791A7199
:10792000DA795A710622B17961F00F01C2F1080EBD
:10793000B1711A44C168C3EB020CCEEB01018C4556
:1079400004D212F80E1002F8011BF3E7FDF7F6F966
:107950002B7843F004032B70012303E0621C2B55AA
:1079600094B200230393F379402B07D0FF2B0AD066
:10797000012B0CD12B7843F0010302E02B7843F06C
:1079800002032B7006E02B7843F00303F9E7621C37
:107990002B5594B210222049584606F0E3FE18B940
:1079A0006B7843F0400335E0B8F1000F0CD06B78F2
:1079B00043F040036B7098F8112010070AD0AB78A1
:1079C00043EA0213AB7005E05846FFF74BFB002873
:1079D00000F0408108AB0020002163E9040199F820
:1079E0000020082A00F224814FF48A71D140C9078F
:1079F00040F11E8109F108011846FFF783FBDDE91C
:107A0000042371693069994208BF904206D16B78AE
:107A100043F030036B7021E0CC0F010804AA5946F3
:107A20004046FFF737FB0028F1D13369B3F17F4FB0
:107A300005EB04006B7840F00381B28A52BA92B22F
:107A4000B2F57E4F40F0FC8043F020036B700222C1
:107A500006F1160106F0B8FE0234A4B2337EFF2B05
:107A600072D16B7843F008026A70728BCABBF269FC
:107A7000BABB328CAABB727E022A0FD1326A6AB9B3
:107A8000B28C5AB996F8262042B943F00B036B70BA
:107A900096F827202A55631C9CB2B4E0728C8AB9F0
:107AA00096F8242072B943F00A036B70737E2B554D
:107AB000601C032206F1250115FA80F006F084FE11
:107AC00004349FE096F82220002A40F0948043F08E
:107AD00009036B70737E2B55601C052206F1230190
:107AE0002CE0B38BADF81030F38BADF81230338C43
:107AF000ADF81430738CADF8163004A8FEF72AFFE9
:107B0000002878D0437CDB0675D5027CF37E9A4250
:107B100071D16B7843F004036B70437C13F00F0357
:107B20001EBFAA781343AB70737E2B55631C9BB2A8
:107B3000B27EEA54A01C042206F1240115FA80F05A
:107B400006F042FE06345DE01FB199F801303BB902
:107B500051E006F11800FFF785FA0028F5D14AE058
:107B600057B16B7843F004036B707B7C13F00F0309
:107B70001EBFAA781343AB7099F8001099F8012042
:107B80000831494404A8FFF7BDFADDE90423716A0E
:107B9000306A994208BF904204D16B7843F00303E6
:107BA0006B7030E004AA06F118013846FFF772FA4C
:107BB0000028F2D1336AB3F17F4F05EB04006B78F4
:107BC0000FD1B28C52BA92B2B2F57E4F09D143F0C6
:107BD00002036B70022206F1260106F0F5FD023465
:107BE00010E043F001036B70082206F1200106F05B
:107BF000EBFD083406E02819102206F1180106F002
:107C0000E3FD1034A4B2039B1BB1631CB2792A5567
:107C10009CB221460298FDF791F8DAF8041050461C
:107C2000FCF7B6FE029A43685360426001201EE0F2
:107C30000821B9F9020000910022FCF79DFBDEE665
:107C400043F010036B70082206F1100106F0BCFD32
:107C5000083402E728191022594606F0B5FD103401
:107C6000FBE6B8F1000F3FF4BCAD0027A9E509B071
:107C7000BDE8F08F10B508220949044606F072FDF0
:107C800048B12378FF2B08D1607800F00F00831EE5
:107C90005842584110BD012010BD002010BD00BF4A
:107CA0007C0F0108F8B5B0F8C631DB07044603D4F1
:107CB00015490320F8F798FF00F5E076012100252B
:107CC00004F5EE773046F9F745FF384684F8CB5196
:107CD000F8F706FF4FF40873A4F8F2310B4B0C4988
:107CE000B3F90030C4F8F44104F5F872384603F0F3
:107CF000BDFF3046F9F75EFF2946B4F9C401BDE87F
:107D0000F840FCF753B800BFA50701088410002015
:107D100080969800F8B5B0F8C631DB07044603D466
:107D200024490320F8F760FF00F5E0760121304692
:107D3000F9F710FF94F8CB31022B03D8013384F804
:107D4000CB3116E0DD1E01F0C7F80123AB403B2B21
:107D5000B0FBF3F505FB13009EBF94F8CB31013364
:107D600084F8CB31092804D93C2828BF3C2005469B
:107D700000E00A2504F5EE773846F8F7B1FE4FF437
:107D80000873A4F8F2310C490C4BC4F8F441694370
:107D9000B3F9003004F5F872384603F067FF304657
:107DA000F9F708FFB4F9C4010021BDE8F840FBF77A
:107DB000FDBF00BFA507010840420F00841000204E
:107DC00010B50446B0F91A00FAF776FEB0F8C631DD
:107DD000DA0703D410490320F8F706FF637E1B0778
:107DE0000BD4002005F0C0FCA8B9B4F91A00FAF7CA
:107DF00063FEBDE81040FFF755BF1022074920463B
:107E000006F0B0FC0028ECD02146B4F91A00BDE819
:107E10001040FBF7CBBF10BDA5070108CC0F010830
:107E20002DE9F04380468DB01846894614461F461A
:107E3000FFF720FF0546B8B910230693029308AE5A
:107E400007AB079003900093019706AB32460DF104
:107E50001601474805F073F8002806DB069B102B37
:107E60000CBF3546002500E000253946204605F0C8
:107E700031FC0646002D74D030B93946BDF91600E4
:107E800005F028FC0646E0B1B6F91A00FAF714FE30
:107E900018B1B0F8C631DA0706D5737E03F03003A7
:107EA000302B08BF3D4600E03D4645B93846FFF758
:107EB000E1FE002851D03D46002D3CD00EB1AF422E
:107EC00004D02946204605F005FC06462846FFF763
:107ED000D1FE58B326B1737E03F03003202B25D199
:107EE00007AE3046FCF75CFC0822074689F8002004
:107EF000A918404606F068FC98F8003083F00203A9
:107F000088F80030CCB9BC4215D036F91400FAF725
:107F1000D3FD48B1B0F8C631DB0705D50CAB03EB98
:107F2000440434F9140C1FE00134ECE7737E03F0D1
:107F30003002202A03D1002016E0204614E003F08E
:107F40000703032B03D104213046FBF7CFFE324653
:107F50004946404605F03EFC06E0FBF7B3FD05460A
:107F6000AAE70028A2D08FE70DB0BDE8F08300BFDC
:107F70005010002070B50E4618B911490320F8F7CB
:107F800033FE0029F9D0B0F91A00FAF795FD00F593
:107F9000EE7504462846F8F7A3FD4FF40873A4F8DD
:107FA000F2310849084BC4F8F44104F5F872714302
:107FB0002846B3F90030BDE8704003F057BE00BF5B
:107FC000A507010840420F0084100020F8B50746BD
:107FD0000D46164610211A462120FBF742FC0446A6
:107FE00060B1806800236DBA082287704371037105
:107FF000C370C5803146104406F0E6FB2046F8BD4C
:108000002DE9F04F85B080460E9E7578022D0F4603
:1080100092461C4640F0B8800823009300226B442F
:108020000321FCF7A9F90028C0F2AE804046FAF718
:1080300043FD21468146404605F04CFBBAF1870FCF
:1080400004464ED0BAF1880F40F09E80B9F8C63190
:10805000D90740F19980DDE90223D6F80CB0D6F8B3
:1080600008A05B4508BF524540F08E80002800F014
:108070008B80B578012D2ED00BD3022D40F084805B
:10808000404607F1080105F04DFB4846FFF70AFEA0
:108090007AE009F5E07901214846F9F75BFDF688B9
:1080A0003D4B04F13807384676BAB3F90080B6B2D2
:1080B000F8F716FD394940F21223013EA4F84E307C
:1080C0003846434604F14C02714303F0CFFD484665
:1080D000F9F770FD5BE007F118014046FAF732FD51
:1080E00052E0B9F8C6319A074ED0B378002B4BD185
:1080F000083710222A49384606F034FB002843D0BE
:10810000D4B1637E9B060CD5D4F88C20D4F8903083
:1081100052EA030105D0F168B0688B4208BF824281
:1081200034D1B6F80690B9F1000F05D13946404672
:1081300005F0F8FA4D462AE0F3882BB384B90323FF
:1081400000930F9A109B3946404605F055FA0446B5
:10815000E8B1324600F18C0352F8080F516803C3AE
:10816000637E0E4823F0300343F030036376F188DA
:10817000094B49BA89B24143B3F9003004F1840292
:1081800004F1700003F072FD002500E0012528468F
:1081900005B0BDE8F08F00BF841000200087930376
:1081A000CC0F010813B58A784B78402A01D8022BEE
:1081B00000E0032B0ED186280ED1C878CB88C0F3FF
:1081C00000145BBA00949BB2083100F00F00FEF778
:1081D0000BFC01E0002000E0012002B010BD000017
:1081E00008B50146074800F05CFC48B91022064972
:1081F000044806F0B7FA0028024818BF002008BD5E
:10820000004808BD40450020CC0F010838B50446A1
:10821000E1B1012380221449B0F9C401FAF76AFCE4
:10822000A0B104F5E07528460121F9F793FCB4F8F4
:10823000C63143F00403A4F8C6314FF4E163A4F857
:10824000CC312846BDE83840F9F7B4BCB4F8C631A3
:10825000B4F9C401044923F00403A4F8C631BDE80D
:108260003840FAF76FBC00BFAC0F010808B5102208
:108270000449054806F076FA0028034808BF0020A4
:1082800008BD00BFCC0F0108404500202DE9F04794
:108290000024054600F116074FF00109A2464FEAF7
:1082A000D40804F0070617F8083009FA06F6334236
:1082B0000AD0E0B2FEF778FB80F810A017F808307B
:1082C00023EA060607F808600134102CE7D10026DF
:1082D000AC695CB12368AB616368A168B3F9C401A0
:1082E000FAF730FC26606660A660F1E710222146AE
:1082F000284606F067FB2C61BDE8F0872DE9F04FBA
:1083000087B003F1080A02905046039117461E46B3
:10831000FFF766FF0446002800F0B480F3885BBADC
:108320009AB21AB942F210738382ABE0DFF860911F
:108330008382103F4FF00008002F70DD08F110031A
:10834000039AD518D35C032B02D0222B4AD05EE0CF
:108350000298FAF7B1FB6B780190042B42D105F13A
:10836000100B08224949584606F0FCF9002839D07C
:108370002A7CFF2A04D16A7C02F00F02022A31D043
:10838000EA7851062ED413062CD46A6852B35946A3
:108390000298FAF749FCAA7804905946D9F80800DF
:1083A000059200F093FB059A824209D8D9F808306B
:1083B0005B7C9A4204D1D9F80430019A9A4207D0E2
:1083C000334B986820B11022324906F0CBF948B9F6
:1083D0002F4B5A6832B9019A5A60049A9A60A2697E
:1083E0001A60A361AB783F2B6B7801D8022B00E0B9
:1083F000032B0CD1EA7804F11603C2F3C00101206B
:1084000002F0070200FA02F2585C02435A546B78F9
:1084100008EBC3081FFA88F8A7EBC3078CE773883B
:108420005BBA9BB22361B28852BA43EA024323612A
:10843000DAF80000DAF80410234603C356F8100FE8
:108440007168022203C3002104F1160006F0BAFA93
:108450000023A361A58A104B04F11C0630465D433E
:10846000F8F73EFB40F2232363860C4B6463B3F9B9
:10847000003004F130022946304607B0BDE8F04F25
:1084800003F0F4BB07B0BDE8F08F00BF7C0F01081C
:1084900078450020CC0F010800879303841000204A
:1084A0002DE9F0418846C108064614460831069A6F
:1084B00022201F46FBF7D5F90546A0B180680021B0
:1084C00064BA01714171C480867080F80380EA68E3
:1084D00000F10804083A204606F074FA324639469C
:1084E000204600F019FB2846BDE8F08170B505462E
:1084F0000E46144618211A462320FBF7B2F980B124
:1085000083686ABA2D0C6DBA76BA5A809D80DE8077
:1085100022689A606268DA6054F8082F1A6162680B
:108520005A6170BD054BB3F90020904204D01AB9CE
:108530000122188059801A71704700BF84450020BD
:10854000034BB3F9002082420CBF1846002070474D
:10855000844500200021FCF75BBCF8B50746848900
:108560000E46154600204DB900230822B96800F0D8
:1085700071FA96F91030022B25D10DE0BD42F3D0EF
:10858000B542F1D02346AA89A96800F063FAEB68E6
:108590006D681C44A4B2E6E702194FF6EE739A42E6
:1085A000C4BF013080B2B1681134204400232022BE
:1085B000083180B200F04EFA4FF6FF73984203D0B4
:1085C000C04380B2F8BD0020F8BD000070B598B07F
:1085D00000230593A3F5803306934C4B1B88ADF81D
:1085E0001C3040F20523ADF80E3008216FF08503F2
:1085F00008A80493F9F7CAFC05A90420FCF71CF9A4
:1086000001A8F9F7C0FCBDF806306FF400721344FE
:10861000032BF5D8DFE803F0023B7575029D284671
:10862000FCF704FC044608B9284667E00221FCF781
:108630007AF9064618B936490320F8F7D5FA606882
:1086400030B190F91030042B02D1C368082B06D04A
:10865000042208212046FCF703FB00284DD000230C
:1086600085682374EB885BBA9BB2002B45D0224609
:108670003146FFF772FF4FF6FF7398423DD169888C
:1086800049BA234640F2012289B2042031E0029E19
:10869000304696F91050FCF7C9FB044608B930463D
:1086A0002CE0406826460028C5D090F91030042BF5
:1086B00007D0FCF7BBFB0346F8B1706040681E466C
:1086C000F1E7FCF7B3FBC0B1826870600023C168BA
:1086D00040680B440028FAD15BBA93806B1C08BF3A
:1086E00063680C4908BF93F9105040F202222346F8
:1086F0002846FBF7FBFD002882D12046FFF72AFF22
:108700007EE703A901A8F9F70DFC79E7D402002060
:10871000A50701080000FFFF10B5044668B161B16C
:1087200090F91030042B0BD14268FFF716FF50B1BF
:10873000A36840BAD880002010BD6FF00D0010BDB6
:108740006FF04C0010BD6FF0010010BD38B50D4644
:108750001446042308220021FCF768FA38B1836824
:1087600000226DBA64BA1D805C809A71DA7138BDDE
:108770001FB50A4CB4F9003063B9094A0193094B9B
:1087800002920093052208234FF480610648F8F70F
:10879000CBFA2080B4F9000004B010BD8A49002053
:1087A0009F0A0108CD8500088A45002010B50446BF
:1087B00001784278054806F00DFA6188044849BA04
:1087C00089B2BDE8104006F005BA00BF4A0F0108A3
:1087D000670F0108F8B504469DF8245025701E4621
:1087E00005F0070310250F46657006989DF82810C0
:1087F00015460AB1002F68D018B1002E69D1304655
:10880000F8BD23B1022B02D00DB9002873D0A1709E
:1088100080B39DF82030E37002289DF82130237149
:1088200004D0082816D0002851D120E00246324951
:10883000304605F097FF18B9237823F02003237002
:10884000637843F008036370737863713378A371BE
:10885000072040E01C236370221D06F1080313F873
:10886000011D02F8011F9E42F9D10D2033E00520C1
:108870001DB9F8BD0320002D3DD0431C9DF81C20E0
:1088800022549DF81D20E2540230022D03D0082D01
:108890000CD0E5B9F8BD637863F07F0363707A7834
:1088A0002254431C3A78E2540230F8BD637863F0F6
:1088B0003F03637007F10803044413F8012D04F823
:1088C000012BBB42F9D10830F8BD3846F8BD002075
:1088D000F8BD63B90DE075B1BDF81C20BDF82030BE
:1088E0009A42CAD1237843F040032370CDE7022B8C
:1088F0008AD1A1708DE7F8BD7A0F0108427802F0A5
:108900000C03082B07D00C2B07D0CBB901784906F4
:1089100014D4032302E0072300E00D2312F0C00269
:108920000CD00178490658BF0233802A01D1981C27
:108930007047C02A04D103F10800704718467047F9
:108940000020704770B501B11AB926490320F8F725
:108950004BF9437803F00C03082B07D103785C062E
:1089600017D5C37813700379537012E00C2B07D11D
:1089700003785B060FD5C3781370037953700AE050
:1089800013B16FF0150070BD03785E06F9D40323B0
:1089900002E0072300E00D23447814F0C00411D056
:1089A00005786D0605D4C65C16705D1C0233455D06
:1089B0005570802C08D1C25C4A70034402205B7859
:1089C0000B7070BD204670BDC02CDAD1034401F19C
:1089D000080213F8010B02F8010D8A42F9D10820B0
:1089E00070BD00BFA507010808B501B11AB9184943
:1089F0000320F8F7F9F8437803F00C03082B09D1AA
:108A0000C37813700379537043794B7083790B707B
:108A1000022008BD0C2B0ED1C378137010F8043F50
:108A2000537001F1080310F8012F03F8012D8B4258
:108A3000F9D1082008BD3BB9037813F0400F14BFEB
:108A40006FF01500002008BD6FF0150008BD00BFD5
:108A5000A5070108F0B51AB3DC0705D511F8014BDD
:108A6000013A204492B20133570801EB47054C1CF0
:108A700003350234AC4207D014F803EC14F8026C4E
:108A800006EB0E263044F4E71A44D30703D511F859
:108A9000173000EB0320030C80B201D01844FAE732
:108AA000F0BD30B54B68456804680A689D4208BF50
:108AB000944209D1C568CB6884688A689D4206BF24
:108AC00094420120002030BD002030BD30B510B3ED
:108AD000E1B188421CD001380139002210F8015F51
:108AE00011F8014FA54202F1080303D1DAB2802A3E
:108AF000F4D10FE085EA0401D8B20B060AD40132A2
:108B0000D2B249008242C9B2F7D130BD084630BD69
:108B1000802030BD104630BD802A28BF8022F8B5A5
:108B2000D50814462A4606460F4605F04DFE630753
:108B30000ED0A4EBC504725DFF23C4F1080403FA50
:108B400004F422EA040272557B5D1C401443745500
:108B5000F8BD10F8013F43B18B42FAD100230370F6
:108B6000437813B1013005F085BB10467047000013
:108B70002DE9F04707468AB008B90020A8E000298F
:108B8000FBD000204FF0FF3406462346054631F85F
:108B900010E0BEF1000F07D1B3F1FF3F13BF013565
:108BA00003B201252DB20BE0B3F1FF3F08D0B4F1C1
:108BB000FF3F01D0B54201DD2E461C464FF0FF338A
:108BC00001300828E3D1581C04D0601C7DD0B54288
:108BD00002DD7AE0601C03D0012ED8BF4FF0FF34D5
:108BE0003D4800256B46E8464FF03A09AC4203D1B8
:108BF00083F80090A5194EE015B183F80090013379
:108C000011F815E01EF0F00F4FEA450C17D04FEAAF
:108C10001E1A0EF00F0E10F80AA010F80EE083F8DE
:108C200001E001EB0C0E83F800A09EF801E04FEA92
:108C30001E1E033310F80EE003F801EC21E0BEF134
:108C4000000F10D010F80EA09E460EF802AB01EBFC
:108C50000C0A9AF801A04FEA1A1A10F80AA083F831
:108C600001A073460DE001EB0C0E9EF801E01EF032
:108C7000F00F1FBF4FEA1E1E10F80EE083F800E051
:108C800001338C4401359CF801E00EF00F0E10F812
:108C90000EE083F800E0072D03F10103A6DD611C5F
:108CA00005D03444082C02BF3A2119700133002149
:108CB00003F8011BC8EB030393423FF65EAF414646
:108CC000384606F07BFA384602E02E461C4683E71B
:108CD0000AB0BDE8F08700BFEC0F01082DE9F047AE
:108CE0000F46054610B90020BDE8F0870029FAD0EC
:108CF0001022002105F066FE3B783A2B04D00024B8
:108D0000A1462646A04619E07A783A2A07F10103DF
:108D1000E9D11F46F3E751462B4806F06BF898B9A6
:108D200051462A4806F066F880B1284BC01A40EA3E
:108D30000616B6F5803FD6D24FF0010917F801AB01
:108D4000BAF1000FE7D119E01F4BEFE7BAF13A0F84
:108D5000C9D1B9F1000F05D1B8F1000FC3D105EBAE
:108D60000408EBE7A21C102ABDD8631CDBB2310A51
:108D700029558146EE54D4B20646DFE7B9F1000F1B
:108D800008D0A21C102AAED8631CDBB2310A2955C8
:108D9000EE54D4B2B8F1000F10D02C44C8EB040844
:108DA00005F1100201230021434504F1FF3407DCE3
:108DB000207802F8010D01332170F5E7102C92D1D3
:108DC0002846BDE8F08700BFEC0F0108FD0F010841
:108DD00010B5017801F0F003602B8AB0044603D08F
:108DE00009091B4805F0F6FE22786378110149B2A3
:108DF0001B0901F030001943C2F381020343C9B2D9
:108E0000144805F0E7FE2168134809BAC1F31301BD
:108E100005F0E0FEA188E379A279104849BA89B249
:108E200005F0D8FE282204F108016846FFF7A0FEED
:108E300001460B4805F0CEFE282204F118016846D1
:108E4000FFF796FE0146074805F0C4FE0AB010BDC4
:108E50000E1001082B1001085C10010871100108A8
:108E60009E100108B21001082DE9F843154681460D
:108E700013480F4604F060FA002D08BF10250024A7
:108E800007F1FF38A74218D00E4804F055FA661CC7
:108E900019F8040004F038FAB6FBF5F305FB136388
:108EA0000BB1A04507D1084805F01EFFA04502D030
:108EB000304604F035FA3446E4E7BDE8F88300BFF5
:108EC000CB100108F01A01087E3401080146014860
:108ED00002F0B2BD8C490020124BF0B593E834008B
:108EE000D8681E691C6084EA050122F000424A40ED
:108EF00082EA420280EA500050405969D86040F34B
:108F0000000782EA802239404A4004EB12249A602A
:108F10009A693E40604044F30004754014405D602F
:108F20006040F0BD8C4900200C4B014618688268F7
:108F30009368013B002B10B4936005DA9469A34257
:108F400008DBCBB20A2B05D01368581C10601970CF
:108F500010BC704710BC06F0A3BB00BF600200202D
:108F600008B53E20FFF7E0FF2020FFF7DDFF034BB1
:108F70001B689868BDE8084005F054BA60020020FC
:108F80002DE9804885B0814600AF0E469246FFF736
:108F9000E7FFB0460AF1FF340025C6EB0803A34201
:108FA000F5DA844B186841684B68013B002B4B6035
:108FB00004DA05F0A1FE002804DAE8E70B685A1C81
:108FC0000A6018780D2801D00A280FD100240D203E
:108FD00088F80040FFF7A8FF0A20FFF7A5FF4645E5
:108FE000D5D033462246254620462BE0082801D01E
:108FF0007F280DD14645D0D0082008F8015CFFF746
:1090000093FF2020FFF790FF08F1FF3B082003E0CB
:1090100008F1010B88F80000FFF786FFD846BCE78F
:10902000222913D15C781CB35C2C25D001331C7829
:109030008C42F7D1597820291AD80135197811B303
:1090400003F8010B19782029F8D9E9E7272906D177
:10905000E8E74B1C497822290AD02029EDD91C7851
:109060005C2C1946F5D1591C5B780132002BF0D1EC
:10907000514805F039FE8AE79C1C9B780132002B91
:10908000F6D02346D3E7002D81D0AB000E3323F07A
:109090000703EB46ADEB030D6C464DF8251030464B
:1090A00090F800E003460130BEF1000FF8D0BEF1A9
:1090B000220F02D0BEF1270F00D1013344F8213036
:1090C0001846013390F800E0BEF1000FF8D10131ED
:1090D0008D42E5D1201FBAB150F8043FA3B1194623
:1090E00013F801EBBEF1000FF5D0BEF15C0FF6D125
:1090F00091F800E0BEF1000F04D091F801E001F812
:1091000001EBF5E7013AEAD12C4B2268FB60C7F886
:109110000890002307F1080151F82380B8F1000FEF
:109120000DD10133022B16D0F4E711463B607A6073
:1091300005F0DAFE7A683B6830B108F10C08D8F81F
:1091400000000028F1D1ECE7D8F808301BB1214627
:10915000284698472CE02168194805F0C5FE0546C9
:1091600010BB184A1849194805F034FD184805F095
:10917000BBFD124BC7F80890FB602C4607F10803B3
:1091800053F824500DB10C3503E00134022CF5D115
:109190000EE00C3555F8181C0029F6D055F8142CA3
:1091A0000A4805F017FDF4E721680A4805F012FDAA
:1091B000DD46ECE660020020D4100108BC12010874
:1091C000ED100108F2100108FE1001080611010857
:1091D0007A2A01081011010808B503F04DFC00209F
:1091E00008BD08B5F7F762FE002008BD012810B5DC
:1091F00006D10020F8F7C6FA04460146074805E004
:10920000486805F037F804460146054805F0E2FCD9
:109210002046FFF75BFE002010BD00BF4013010891
:109220006613010808B5FFF757FE0146024805F02E
:10923000D1FC002008BD00BF273D010801460628DB
:1092400014D8DFE800F004060B0D0F1109000948DF
:1092500000E0094805F0BEBC0848FBE70848F9E70C
:109260000848F7E70848F5E70848F3E7084805F035
:10927000B1BC00BF881301088C13010892130108C8
:109280009A1301089F130108A2130108A5130108EE
:10929000AB130108102828D00BD803281BD003D803
:1092A000E8B1022815D07047052816D006281AD034
:1092B0007047262815D004D8162818D0202818D092
:1092C00070472A2817D02B2817D0272818D10D48E7
:1092D00014E00D4812E00D4810E00D480EE00D4876
:1092E0000CE00D480AE00D4808E00D4806E00D4886
:1092F00004E00D4802E00D4800E00D4805F06ABCAE
:10930000704700BF37140108B0130108C0130108EB
:10931000CD130108E3130108EB130108F013010852
:1093200003140108151401082A1401084E14010839
:109330005914010808B50146034805F04BFC0348E1
:10934000BDE8084005F0D0BC681401088D14010880
:1093500013B5044601A8FBF723FA20B1BDF90400B8
:10936000031B5842584102B010BD00001FB504ABAA
:10937000012403F8012D00940022FBF723F80028B4
:1093800004DA094805F0B0FC20460BE09DF80F1008
:10939000064B074A0748002914BF1146194605F035
:1093A00019FC002004B010BD1B1801081818010892
:1093B0007E34010837180108A0F13003DAB2092A17
:1093C00004D9A0F16103DAB2052A01D81846704722
:1093D0004138C3B2052B88BF4FF0FF307047000003
:1093E0007FB50C46082105460DEB0100164604F03A
:1093F0003BFA08B911480FE0009002AB0022214669
:109400002846FAF7DFFF00280ADA0D4805F0E2FBEC
:109410002046FFF73FFF0B4805F066FC01200BE0FC
:10942000094805F0D7FB2046FFF734FF32462946AE
:10943000064805F0CFFB002004B070BD4E180108AF
:10944000C11801087E340108D7180108E518010881
:109450007FB5064610460D4604F00CFF04AB012410
:1094600003F8010D0022009429463046FAF7AAFFBE
:1094700000280ADA0C4805F0ADFB2846FFF70AFF82
:109480000A4805F031FC20460CE0094805F0A2FB33
:109490002846FFF7FFFE9DF80F200648314605F0ED
:1094A00099FB002004B070BDC11801087E3401088A
:1094B000D7180108FE1801087FB506460D4610466C
:1094C000531E13F8014F1CB1303C092CF9D908E0A8
:1094D0000A22214606F0CCF80390013009D11C483D
:1094E0001CE01022002106F0C3F803900130F6D0F2
:1094F0000124039BB3F5803FF1D2022300930022A5
:1095000003AB29463046FAF75DFF00280ADA114816
:1095100005F060FB2846FFF7BDFE0F4805F0E4FBB1
:10952000012012E00D4805F055FB2846FFF7B2FE7A
:1095300031460B4805F04EFB039924B1094805F06C
:1095400049FB002001E00848F9E704B070BD00BF06
:1095500017190108C11801087E340108D71801083D
:10956000651901087B190108743E0108022808D01A
:10957000FF2808D0054A064B01280CBF18461046A4
:109580007047044870470448704700BF94190108A9
:10959000831901088B1901089019010870B5012978
:1095A00088B00C46164609D104230093002207AB6D
:1095B0002921FAF7E1FE051E0EDA09E0022905D19C
:1095C000F9F7D2FC079008B1012505E06FF0850599
:1095D000154805F089FB24E0E4B266B11C220021A5
:1095E000079805F0EFF92046FFF7C0FF01460F4846
:1095F00005F0F0FA15E02046FFF7B8FF079AD368A8
:10960000516804939368039313690293019113685B
:109610000B440093936952690146054805F0DAFA54
:109620003546284608B070BD9C190108D6190108B6
:10963000F71901082DE9F04790B002AF0026044663
:10964000FE70F9F739FA21460546CB4805F0C2FA13
:10965000082300933246FB1802212046FAF78CFEBD
:10966000061E1CDB06EB460808F1070323F0070380
:10967000E946ADEB030D0DF1080AC04805F0AAFA62
:10968000334607F108024146504604F0C1F801464E
:10969000BB4805F09FFABB4805F09CFACD46022373
:1096A0000022009311463B1D2046FAF765FE002874
:1096B00003DBB988B44805F08DFA02230093002239
:1096C0003B1D26212046FAF757FE002803DBB98808
:1096D000AE4805F07FFA0223009300223B1D0621CD
:1096E0002046FAF749FE002803DBB988A84805F0B0
:1096F00071FAA84805F06EFA082300930022FB18BF
:1097000003212046FAF738FE061E1EDB06EB46084C
:1097100008F1070323F00703E946ADEB030D0DF154
:10972000080A9D4805F056FA334607F108024146FB
:10973000504604F06DF80146984805F04BFA9848F9
:10974000CD4605F047FA012600E0002602230093EB
:109750000022BB1D10212046FAF70EFE002804DB74
:10976000B7F906108F4805F035FA0123009300225F
:10977000BB1C18212046FAF7FFFD002808DB8A48A9
:1097800005F028FAB878FFF759FD7E4805F022FA6F
:10979000012300930022FB1816212046FAF7ECFD66
:1097A000002803DB7978814805F014FA4FF00108AE
:1097B000CDF8008007EB0803002220212046FAF7AD
:1097C000DBFD002810DBCDF80080FB1C00221F21F0
:1097D0002046FAF7D1FD002806DBFB78434503D18C
:1097E0007978734805F0F6F96A4805F0F3F9012332
:1097F00000930022FB1C13212046FAF7BDFD002830
:1098000008DB97F80380B8F1010F03D1694805F030
:10981000E1F94646012300930022FB1C1421204657
:10982000FAF7AAFD002808DB97F80380B8F1010FCA
:1098300003D1614805F0CEF946460123009300228A
:10984000FB1C15212046FAF797FD002808DB97F846
:109850000380B8F1010F03D1584805F0BBF9464623
:10986000012300930022FB1C12212046FAF784FDFD
:10987000002808DB97F80380B8F1010F03D15048A6
:1098800005F0A8F94646012300930022FB1C19218C
:109890002046FAF771FD002808DB97F80380B8F13D
:1098A000010F03D1474805F095F94646012300937F
:1098B0000022FB1C1F212046FAF75EFD002808DB72
:1098C00097F80380B8F1010F03D13F4805F082F902
:1098D0004646012300930022FB1C1E212046FAF776
:1098E0004BFD002808DB97F80380B8F1010F03D186
:1098F000364805F06FF94646012300930022FB1C11
:1099000023212046FAF738FD002808DB97F803806A
:10991000B8F1010F03D12E4805F05CF94646FDB1C0
:10992000B5F8C8112B4805F055F995F8CA112A4821
:1099300005F050F9B5F8C631D80702D5274805F02B
:1099400049F9B5F8C631990702D5254805F042F91D
:10995000B5F8C6315A0702D5224805F03BF9012671
:109960002046FEF7EDFD002840D00379002B3DD0C6
:109970001D4805F02FF93AE0A21A0108D91A01088A
:10998000E91B0108F11A0108AE1A0108BD1A010805
:10999000C91A0108D11B0108D51A0108E31A0108E8
:1099A000E71A0108F31A0108061B01080F1B01083A
:1099B000231B0108361B0108401B01084A1B010834
:1099C000541B01085E1B0108681B01086F1B01087E
:1099D000791B0108881B0108921B01089A1B0108CA
:1099E000A01B0108A61B0108B01B010816B13948CD
:1099F00005F0F0F80223009300223B1D05212046CC
:109A0000FAF7BAFC002803DBB988334805F0E2F81E
:109A1000002D58D0B5F8C6313049314813F0800FC9
:109A2000304B08BF194605F0D5F82A4805F0D2F8A2
:109A300005F5E07610222C49284604F093FE002814
:109A400031D02A4805F0C6F82822294607F110002F
:109A5000FFF78EF808B36A7C254807F1100105F07E
:109A6000B9F808222349284604F07CFE38B12B7847
:109A7000FF2B06D16B7803F00F03022B01D11E4898
:109A800000E01E4805F0A6F82B7CDB0708D52B78F4
:109A9000FF2B0CBF1A481B4800E01B4805F09AF842
:109AA0000C4805F097F83835B542C3D1174805F092
:109AB0001BF9002201212046FFF770FD0022022140
:109AC0002046FFF76BFD114805F00EF93837BD460B
:109AD000BDE8F087D11B0108B71B0108931A0108E4
:109AE000DE1B0108991A0108CC0F0108EC1B0108C4
:109AF000F91B01087C0F0108081C01080E1C010855
:109B0000151C0108221C01082D1C01087E340108C7
:109B10002DE9F04F012889B0804602AF0E460BDCDC
:109B200007F10800FAF73CFE18B1B7F90800FFF793
:109B300081FD002400F06EBC4868431E13F8014FFD
:109B40003CB3303C092CF9D93168A94805F042F8FA
:109B50003068FFF7EFFB3168A64805F03BF8316845
:109B6000A54805F037F83168A44805F033F83168A6
:109B7000A34805F02FF83168A24805F02BF83168AA
:109B8000A14805F027F8A14805F0AEF8012400F03F
:109B900041BC04F06FFB05B22846FFF7D9FB002853
:109BA00000F01984B8F1020F04D12846FFF742FDF6
:109BB00000F030BC9649B06805F096F9002840F0F6
:109BC0002482B8F1040F01DC30681BE2D6F80C8067
:109BD0009048D6F800903669414605F085F910B9ED
:109BE000324602210CE041468B4805F07DF9002801
:109BF000F6D04146894805F077F928B93246032165
:109C00002846FFF7EDFBACE34146854805F06CF9CB
:109C100010B93246002151E04146824805F064F90E
:109C20000028F6D04146804805F05EF910B932466A
:109C3000262143E041467D4805F056F910B93246E9
:109C400006213BE041467A4805F04EF90028F6D05F
:109C50004146784805F048F90028F0D0414676485A
:109C600005F042F9044610BB304604F003FB07F14F
:109C70001803022223F8100D1021009228462246D4
:109C8000FAF7A0FB002807DA6C4804F0A3FF6C4841
:109C900004F0A0FF6B4877E76B4804F09BFF68482F
:109CA00004F098FFB7F908206848294607E34146C1
:109CB000674805F019F928B9324605212846FFF70B
:109CC000FBFB4EE34146634805F00EF904460028CD
:109CD00063D13146604805F007F908B9002332E046
:109CE00031465E4805F000F90028F7D031465C485F
:109CF00005F0FAF808B9012325E03146594805F086
:109D0000F3F80028F7D03146574805F0EDF808B9C8
:109D1000022318E03146554805F0E6F80028F7D050
:109D20003146534805F0E0F808B905230BE0314609
:109D3000504805F0D9F80028F7D031464E4805F0D4
:109D4000D3F8B8B9062301263B720022009607F12A
:109D5000080318212846FAF735FB002812DA47488D
:109D600004F038FF387AFFF769FA364804F0BCFF90
:109D700034464FE33146424805F0B6F80028E1D0BA
:109D8000404801E72946404804F024FF387AFFF7AD
:109D900055FA2C4804F0A8FF3CE341463B4805F047
:109DA000A3F810B9324616210EE04146384805F0B6
:109DB0009BF810B93246202106E04146354805F0AF
:109DC00093F828B9324627212846FFF741FBC8E21D
:109DD0004146314805F088F80446002840F0978055
:109DE00031462E4805F080F8002859D1012363E060
:109DF00089230108692001082E2101081C2301087C
:109E0000171F01081C2001089E230108C92301080F
:109E10001E1D0108DC1C0108E11C0108EC1C0108E6
:109E2000E3130108F61C0108EB130108FB1C0108F1
:109E3000FF1C0108031D01080A1D0108C1180108C3
:109E4000031401087E340108D7180108FE18010820
:109E5000101D01086C080108181D0108881301086D
:109E6000F72101088C130108330801089A1301082F
:109E70001C1D0108A5130108221D01086B1D010806
:109E8000921301082A1D01088A1D0108B21D01084C
:109E9000BA1D0108C71D0108D51D01083E1C010897
:109EA0003146B04805F020F800289FD03146AE4832
:109EB00005F01AF8C8B900234FF001083B720022E0
:109EC000CDF8008007F108032A212846FAF77AFA2C
:109ED000002812DAA54804F07DFEA54804F07AFEB9
:109EE000A44804F001FF444694E23146A24804F03D
:109EF000FBFF0028DFD0A14846E6A14804F06AFE37
:109F00009B4804F067FE324629469E48D7E1414609
:109F10009D4804F0E9FF0446002872D1304605F060
:109F2000AFF94FEA500909F1070323F00703EA46A6
:109F30000E28ADEB030D83460DF1080801D19348BF
:109F400006E0102801D1924802E0202804D191486F
:109F500004F040FE002117E0302801D18E48F7E7D9
:109F6000402801D18D48F3E7802801D18C48EFE7E4
:109F70008C4804F02FFE17E0421C12D04A0800EB78
:109F8000031008F8020002318B450FD9705CFFF70F
:109F900013FA721878605078FFF70EFA7B685A1C33
:109FA000EAD1814804F0A0FE012428E0CDF8009019
:109FB000434600222B212846FAF704FA002807DA44
:109FC0006A4804F007FE794804F004FE6948E9E7AE
:109FD0006B4804F0FFFD754804F0FCFD2946744809
:109FE00004F0F8FD4546C144A94505D015F8011B0C
:109FF000704804F0EFFDF7E75E4804F075FED546C3
:10A0000008E24846FFF796F9C0E56B49B06804F0EE
:10A010006BFF044600286AD1B8F1030F01D1316803
:10A0200027E0A8F10308B8F1010FD6F80C9022D070
:10A030006249D6F800A0484604F056FF20B9D6F889
:10A0400010904FF0020A17E05D49F06804F04CFFF1
:10A0500020B9D6F810904FF0010A0DE05949F06888
:10A0600004F042FF20B9D6F810904FF0000A03E048
:10A0700051465548ABE182462F2140224846FEF723
:10A0800068FD431E802B0646494628BF402607F13F
:10A0900008005FFA86FBFEF721FE00283AD0B8F1EF
:10A0A000010F07D03B7AFF2B04D1BAF1010F07D083
:10A0B000464869E5BAF1020F14BF4023412300E08E
:10A0C00040235A4607F108012846F8F713FD18B94E
:10A0D0003F4804F07FFD59E54FF0FF334361836152
:10A0E00032462B4649463B4804F074FD92E13A491A
:10A0F000B06804F0F9FE0446B8B9B8F1030F02D114
:10A100003168364863E1F66807F108003146FEF72A
:10A11000E5FD08B9324837E507F108012846F8F7A8
:10A1200011FD2A4631462F48C9E02F49B06804F096
:10A13000DBFE0446002869D1B8F1030F02D1316873
:10A140002A4844E1F06804F095F8A0F5A063B3F55F
:10A150007B4F06464ED34FF6FF724FF4A061244862
:10A160009FE000BFDD1D0108181D0108C11801088E
:10A170004E1401087E34010888130108E01D01080F
:10A18000D7180108E5180108F31E0108101E010880
:10A190002D1E01084A1E0108681E0108861E0108BE
:10A1A000A41E0108C21E0108DC1E01085914010882
:10A1B000F71E01080E1F0108131F0108631F010885
:10A1C0006B1F0108751F0108171F0108A21F010856
:10A1D000CE1F0108F11F0108182001081C200108EA
:10A1E0007D1F01083F200108652001086920010842
:10A1F000842001082846F8F75FFC08B98848C3E4C2
:10A20000A0F8C8612A463146864858E08649B068B9
:10A2100004F06AFE044670BBB8F1030F17D08349FF
:10A22000F06804F061FE002800F0EA808049F068E0
:10A2300004F05AFE002800F0E6807E49F06804F041
:10A2400053FE002800F0CA80F1687B48BAE04FF066
:10A25000FF0919F0010F04D0224601212846FFF71B
:10A260009DF919F0020F3FF491AC224602212846D5
:10A27000FFF794F98AE47149B06804F035FE0446AA
:10A2800000BBB8F1030F02D131686D489FE0F06860
:10A2900003F0F0FFFF28064606D96A484FF6FF7222
:10A2A000002104F097FC71E42846F8F705FC08B992
:10A2B000654869E480F8CA6164482A46314604F07A
:10A2C00089FCA7E0D6F80880614998F80030D6F8F4
:10A2D00000902D2B08BF08F1010840460CBF002656
:10A2E000012604F001FE10B93246132136E0594927
:10A2F000404604F0F9FD10B9324612212EE05649CD
:10A30000404604F0F1FD10B93246142126E05349CD
:10A31000404604F0E9FD10B9324615211EE05049CF
:10A32000404604F0E1FD10B93246192116E04D49CE
:10A33000404604F0D9FD10B932461F210EE04A49CB
:10A34000404604F0D1FD10B932461E2106E04749CF
:10A35000404604F0C9FD30B9324623212846FFF7B4
:10A3600005F8044656E04249404604F0BDFD044667
:10A3700078B92846FEF7E4F808B93E4804E426B167
:10A380000123037129463C481CE0067129463B48DD
:10A3900018E03B49404604F0A7FD0446A8B928460A
:10A3A000F8F78AFB10B93748FFF7EEBB2EB1012151
:10A3B000F8F799FB2946344804E03146F8F793FB57
:10A3C0003248294604F006FC24E03148494604F0AE
:10A3D00001FCFFF7DBBB2F48FFF7D6BBB8F1040F3A
:10A3E0000AD04FF0020905222B49306904F0B6FF6C
:10A3F000B0FA80F464092CE704464FF0020930E714
:10A400004FF0FF0901E04FF00109B8F1040FEAD164
:10A41000002421E720461C37BD46BDE8F08F00BF71
:10A42000AC200108C6200108E920010890190108A4
:10A43000EF200108B80D0108F22001082B210108C6
:10A440002E210108482101087621010896210108E2
:10A45000BF210108C7210108CF210108D721010828
:10A46000DF210108E3210108E8210108F0210108AA
:10A47000FD210108022201082022010847220108CB
:10A480006F22010877220108AB220108E3220108AC
:10A490001C2301086A1C01081C1D01082DE9F04F4E
:10A4A00087B006AF0546884691469A4604F0E8FE16
:10A4B00028448542A0EB050413D010F801392F2B56
:10A4C00005D1601C284403F0D5FE06460BE03A2B6C
:10A4D00001D02E2BEDD1284604F0D2FE00260446F2
:10A4E00001E00024264604F1080323F00703ADEB46
:10A4F000030D0DF1180B621C0021584604F062FA9E
:10A5000029462246584604F05FF9404604F0B8FE5A
:10A5100059461648FEF7E2FBD0B1144D10244146CF
:10A520001348FEF7DBFBD0B1114B10220021360699
:10A53000039102920193CDF810A0009623462A467B
:10A5400049460C4802F0F0FB0437BD46BDE8F08FE9
:10A5500003F098FE6A230360074D0424DFE703F04D
:10A5600091FE6A2303600422044BDFE7B849002010
:10A57000A849002050100020CC490020C8490020E4
:10A5800001282DE9F34105460C4603D17A4802F033
:10A5900075FDBBE002281AD14968784804F0A4FC94
:10A5A000002800F0B1806168754804F09DFC08B98E
:10A5B0007448B8E06168744804F096FC014620B91C
:10A5C0006D4802F0A0FC7148ADE07148ABE053DD8E
:10A5D00049686A4804F088FC58B16168684804F02A
:10A5E00083FC30B16168684804F07EFC08B16948BA
:10A5F00099E0032D25D16168634804F075FC054698
:10A6000090B9A06803F036FE04B22046FAF7D4F8F9
:10A61000214628B1584802F076FC21465E4800E009
:10A620005E4804F0D7FAA2E0A1685D48FEF756FB49
:10A63000054600286CD0102259494F4802F045FCCD
:10A6400064E0052D18D161684C4804F04DFC0028E9
:10A6500068D1E168534804F047FC0546002861D101
:10A6600001A8FAF79DF8012831D14FF0FF33BDF969
:10A6700004202169A0683DE0072D3ED161683F4874
:10A6800004F032FCC8B9E168464804F02DFCA0B9DA
:10A690006169454804F028FC054670B901A8FAF73D
:10A6A0007FF8012813D1A069BDF90480A668276945
:10A6B00003F0E0FD424603461AE061682F4804F0CB
:10A6C00013FC20B9E168374804F00EFC08B13748A4
:10A6D00029E06169364804F007FC05460028F6D1F8
:10A6E000A069A668276903F0C5FD4FF0FF3302B2E9
:10A6F00039463046FFF7D2FE39E0092D12D16168A4
:10A700001E4804F0F1FB90B12A480CE000252EE031
:10A7100003F0B8FD6A23036004222749164802F0BB
:10A72000D4FB24E0254804F0DFFA01251FE0E168AE
:10A730001C4804F0D9FB0028E6D161691C4804F0EC
:10A74000D3FB0028E0D1E169174804F0CDFB0546B2
:10A750000028D9D1A069A668276903F08BFD80463F
:10A76000206A03F087FD0FFA88F20346C0E7284607
:10A7700002B0BDE8F08100BF50100020131F010897
:10A7800018200108E3250108772601087D26010825
:10A790009E2601081B2701086B2701089F27010837
:10A7A000B8490020BD27010833290108C127010845
:10A7B0003C29010803240108CC4900204029010854
:10A7C00013B5044601A8F9F7EBFF20B1BDF9040069
:10A7D000031B5842584102B010BD000000F00700B2
:10A7E000072813D8DFE800F00406080A0C0E121040
:10A7F00008480CE008480AE0084808E0084806E075
:10A80000084804E0084802E0084800E0084804F06E
:10A81000E1B900BF902901089D290108AA29010872
:10A82000B7290108C4290108D1290108DE29010836
:10A83000EB29010800F03000202805D0302805D091
:10A84000102805D1044804E0044802E0044800E070
:10A85000044804F0BFB900BFF8290108FB2901082A
:10A86000002A0108A02A0108F0B5012893B0064685
:10A870000D4607D16B4804F037FA6B4804F034FA00
:10A88000002005E04968694804F02EFB30BBF1E781
:10A8900002F052FF0446002800F0C1802822214621
:10A8A00008A8FEF765F9237EB4F91A60054604F19D
:10A8B0001002182102A802F0ABFF324603462946D7
:10A8C0005B4804F087F9607EFFF788FF607EFFF742
:10A8D000B1FF584804F008FA2046D9E7012E40F3AA
:10A8E0009680022E74D06968534804F0FDFA04463D
:10A8F000002857D1023E012E02D0022E0CD022E0B9
:10A9000008A8F9F74DFF012898BFBDF92060AF688E
:10A9100088BF264600251CE0AF6808A83946FEF728
:10A92000DDF928B9A86803F0A5FCEF6806B2F1E7E5
:10A9300002A8F9F735FF012898BFBDF90860ED6856
:10A9400088BF264605E0A86803F094FCEF682D69EF
:10A9500006B23046FFF734FF08B9384805E03946FB
:10A9600008A8FEF7BBF920B9354804F0BDF9012469
:10A9700055E04DB108212A460DEB010002F074FFAD
:10A98000034610B92F48F0E72B460022009208A991
:10A9900002AA304602F030FE08B92B48E5E73946F6
:10A9A0002A4812E069682A4804F09EFA044678B9F9
:10A9B000AD6808A82946FEF791F90028D4D008A967
:10A9C000204602F0AFFE2348294604F003F926E0B2
:10A9D0006968214804F088FA0446C0B902F0ACFE68
:10A9E0002146054655B119B1B1F91A0002F09AFE97
:10A9F000284602F0A1FE29460546F3E719B1B1F950
:10AA00001A0002F08FFE154804F0E4F807E02B6806
:10AA100000931A461946124804F0DCF8A7E72046CE
:10AA200013B0F0BD042A0108532A01087812010866
:10AA3000A22A01087E340108131F0108B72A010861
:10AA40007D1F0108D72A0108022B0108322B0108BB
:10AA500018200108642B01081C1D01088D2B01081A
:10AA6000AC2B010870B501288AB00C460DDD486892
:10AA700003F000FC05B22846FFF7A2FE30B92168BA
:10AA8000164804F0A7F8012025E00025144804F03A
:10AA90002BF9144804F028F9002002F065FE044662
:10AAA000C8B1B4F91A600DB1AE4212D128222146C4
:10AAB0006846FEF75DF8314602460B4804F08AF816
:10AAC000607EFFF78BFE607EFFF7B4FE074804F060
:10AAD0000BF92046E1E70AB070BD00BF582C010811
:10AAE000712C01086E2A0108A52C01087E3401088A
:10AAF00008B501460B4804F06DF80B4804F0F4F873
:10AB00000A4804F0F1F80A4804F0EEF8094804F0A5
:10AB1000EBF8094804F0E8F80848BDE8084004F0FC
:10AB2000E3B800BFB32C01080F2D0108192D01084F
:10AB3000272D0108812D0108952D0108A62D01085A
:10AB40000C4AF0B514880830260AE5B200238B427F
:10AB500009D2FF2C85BFC718C654C5547D708CBF61
:10AB600002330133F3E781BF138809181B0A01F888
:10AB7000013CF0BD5C0200202DE9F0430D4685B09C
:10AB800002210446F9F7CFFE032107462046F9F7D4
:10AB9000CAFE07B108B9274845E08668264AB38847
:10ABA000F48812885BBA9BB264BA9A42A4B239D1D3
:10ABB0002249234B0A881B889A4203D9944203D323
:10ABC000012307E0944204D39C428CBF002301235D
:10ABD00000E0002333B3BF68D0F80C9019489442CA
:10ABE00098BF013207F1080898BF0A802822414621
:10ABF000FDF7BEFF4FF47A72B388B5FBF2F102FBAA
:10AC0000115502910395FA7901925BBA02469BB203
:10AC1000494600940C4803F0DDFF404602F0ACFDCD
:10AC2000012003E0094804F05FF8002005B0BDE80A
:10AC3000F08300BFC12D01085C020020F84900200C
:10AC4000FA490020D0490020F82D01083B2E0108C8
:10AC50002DE9F04F99B081231293994B00241B8862
:10AC60001194012880460F46ADF84C3038DD02289B
:10AC700000F0BF81486803F0FDFA051EC8BF01243B
:10AC800004F101034FEA830957F82330089304F1D4
:10AC90000203D8BF0325984506DD07EB0903586872
:10ACA00003F0E8FA049001E004230493E31C9845C0
:10ACB00006DD07EB0903986803F0DCFA064601E0BD
:10ACC0004FF47A760434A04506DD07EB0903D86813
:10ACD00003F0D0FA099000E00995049B002B03DAF9
:10ACE0003868FFF705FF3FE04FF0FF322521089855
:10ACF000FDF72FFF04B2621C089914A808BF0024B6
:10AD0000FDF7ECFF08B96F482CE008226E4914A843
:10AD100003F028FD50B19DF85030FF2B05D19DF870
:10AD2000513003F00F03022B00D0A4B10FA8F9F7A4
:10AD300037FD44B1002800F05781BDF93C309C42FA
:10AD400040F0528106E0012802D1BDF93C3001E01B
:10AD50005E4807E01C4611A90320F9F76DFD0028A5
:10AD600004DA5B4803F0C0FF01204AE1F5F742FE38
:10AD70004FF47A7373430D9300220023CDE90A0147
:10AD80000027CDE906234FF0FF332E460593BA4640
:10AD9000BB46013E731C4F4A00F005814D4B19889C
:10ADA0004D4B1A88013292B21A80049B0093802086
:10ADB000002302F08BFB804698B104998068FFF76E
:10ADC000BFFE14AA00214046F7F7F4FC814640B1CB
:10ADD000ACB14FF0FF3308220021F9F727FF81467D
:10ADE00018B93E4803F080FFD3E7836800221A7049
:10ADF0005A705A719A711A715A8083685C80002067
:10AE0000F6F7C0FC4B46804640F20222344902204D
:10AE1000F9F76CFA0C9038B9324803F065FF0C99D9
:10AE20004846F9F7F5FFB4E72F4A00230FA800F0D2
:10AE300037FF00282DDBBDF83E2040F201239A4267
:10AE400020D10020F6F79EFCDDF84090C8EB00080A
:10AE500041464846FFF790FE002183444846F9F7F3
:10AE6000D7FF059B474538BF4746434528BF434664
:10AE70000593DDE9062312EB080243F10003CDE957
:10AE800006231AE00E4B19880FA809B2F6F7D6FF71
:10AE900013E0164803F028FF0FE00FA8F7F770F84B
:10AEA000002827DDBDF83E304345F6D1104803F0B9
:10AEB00091FE00211098F9F7ABFF40F20128ECE772
:10AEC000D4020020582E01087C0F0108712E0108C1
:10AED000BF2E01085C020020FA490020AC1C0108CA
:10AEE0000000FFFFDF2E010840420F000A2F01087B
:10AEF000172F01081EB100210D9800F08DFE099B4F
:10AF00000AF1010A534502D0002E7FF442AFF5F753
:10AF100071FD089980463C4803F05CFEBBF1000FD0
:10AF2000C6EB050A38DD5246DDE90601D31703F00A
:10AF300015F8DDE90A23B8EB02029046334AB8FB64
:10AF4000F2F1642302FB11828DE806000C905A4650
:10AF5000514603FB0BF32E4893FBFAF3C3F1640352
:10AF600003F038FE4FF47A72B7FBF2F002FB107E6A
:10AF700001900C980C9BB3FBF2F302FB13000090C2
:10AF800005980599CDF808E0B1FBF2F102FB11023A
:10AF9000204803F01FFE03E051461F4803F01AFE4D
:10AFA0004FF0000AF5E61D4B00211980138811A906
:10AFB000013303201380F9F75FFC40F201240FA84E
:10AFC000F6F7DEFF00280BDDBDF83E30A342F6D1D8
:10AFD000134803F0FFFD00211098F9F719FFECE783
:10AFE000BBFA8BF040090CE021460E4803F0F2FD5D
:10AFF000BAE64B6808934FF004090325CDF810908A
:10B0000054E619B0BDE8F08F5C2F010840420F00F4
:10B01000782F0108C12F0108F52F0108FA490020F7
:10B02000172F01082C3001089368013B002B10B446
:10B03000936008DA9469A34202DBCBB20A2B02D1F7
:10B0400010BC04F02DBB1368581C10601970C8B2F6
:10B0500010BC704710B503F00DF904B22046F7F7A5
:10B060002BFD20B9064803F03FFE012010BD20460D
:10B07000FAF7D0F82146034803F0ACFD002010BDDC
:10B08000523001086E30010830B58FB00D4603F024
:10B09000F1F82946C4B26846FDF720FE18B90E48FB
:10B0A00003F022FE10E000231A4669462046FAF714
:10B0B0002DF958B92822694604A8FDF759FD224602
:10B0C0000146064803F086FD012003E0044803F032
:10B0D00081FD00200FB030BD9C300108CB3001084D
:10B0E000FD30010810B503F0C5F8C4B22046FAF7E8
:10B0F000F9FF10B92146084804E0FBF7F0F82146B3
:10B1000020B9064803F066FD012010BD044803F095
:10B1100061FD002010BD00BF213101084A31010846
:10B120007131010830B58BB003F0A4F8C5B22846E0
:10B13000FAF7D8FF044620B90A4803F0D5FD0120EC
:10B140000EE0383000F0ECFC282204F108016846DB
:10B15000FDF70EFD2A460146034803F03BFD0020A3
:10B160000BB030BD91310108B931010830B58BB059
:10B1700003F080F8C5B22846FAF7B4FF044620B9B8
:10B180000A4803F0B1FD01200EE0383000F00EFD5A
:10B19000282204F108016846FDF7EAFC2A46014628
:10B1A000034803F017FD00200BB030BD91310108BA
:10B1B000F831010870B58CB003F05CF8C6B23046C7
:10B1C000FAF790FF0125044620B9134803F08CFDDF
:10B1D00028461EE0114A90F82730B2F9000094F892
:10B1E0002820019294F82620009205FA03F340F6F5
:10B1F000011204F1380100F0A9FC282204F1080131
:10B2000002A8FDF7B5FC32460146054803F0E2FC12
:10B2100000200CB070BD00BF9131010862370020E2
:10B220003932010808B504490020FAF70BFA03483F
:10B2300003F05AFD002008BD260F01087A320108EC
:10B2400013B5234C234803F04FFDA36900932269F3
:10B25000A3682168204803F0BDFCE369009362699C
:10B26000E36861681D4803F0B5FCA36B0093226B93
:10B27000A36A216A1A4803F0ADFCE36B0093626B8A
:10B28000E36A616A174803F0A5FCA36D0093226D81
:10B29000A36C216C144803F09DFCE36D0093626D78
:10B2A000E36C616C114803F095FCA36F0093226F6F
:10B2B000A36E216E0E4803F08DFCE36F0093626F66
:10B2C000E36E616E0B4803F085FC002002B010BDF8
:10B2D000F03C00208F320108D2320108043301080B
:10B2E00036330108683301089A330108CC3301086A
:10B2F000FE330108303401082DE9F041514C524829
:10B3000092B003F067FC63780BB9504800E05048F6
:10B31000504DDFF86C8103F05DFC286809218268DC
:10B32000FFF782FE28680A218268FFF77DFE4A48FF
:10B3300003F050FC002606EB08031B790BB94348C9
:10B3400000E04348434F03F045FC28680921826828
:10B350003036FFF769FE902EEDD13868394D82689E
:10B360000A21FFF761FE38680A218268FFF75CFE58
:10B37000F5F740FB637806460F46002B5DD0B5F825
:10B380008A0095F880302978B5F92C200290B5F81C
:10B3900088000190D5F88400008800902F4803F0C1
:10B3A00019FCE86E296F801B61EB0701002871F121
:10B3B000000305DB2A4A002302F0D0FD064600E028
:10B3C0000026236A274993F98C50282208A8FDF704
:10B3D000CFFB94F8363094F83270228E069613F034
:10B3E000020F214B214918BF1946638F059394F82A
:10B3F0003830049394F82630039394F827300126CC
:10B400009E4025EAE5758DE86200194B1949022F27
:10B4100008BF0B460146184803F0DCFBE46964B141
:10B42000611D282208A8FDF7A3FBE369E28A014613
:10B43000124803F0CFFB2468F1E7002012B0BDE80A
:10B44000F08100BF603C00206E3401087F340108A9
:10B450008334010860020020873401089634010813
:10B4600040420F00683C00203E1C0108181D0108E6
:10B470006734010862340108DA3401083135010803
:10B48000B037002038B50546084602F0F3FEC4B2D6
:10B490002046FAF727FE28B921460B4803F09AFB0D
:10B4A000012038BD083015B1FBF78CF801E0FBF73F
:10B4B00090F8064B064A0748002D08BF1A46214659
:10B4C00003F088FB002038BD2131010867350108F1
:10B4D000623501086E35010838B50C4602F0CAFE27
:10B4E000C5B22846FAF7FEFD28B929460B4803F0F5
:10B4F00071FB012038BD90F83630094923F0020372
:10B5000043EA440380F83630064B0748002C08BF56
:10B51000194603F05FFB002038BD00BF2131010850
:10B520007E3401084211010897350108012838B519
:10B5300005460C4603DCBDE83840FFF7DDBE634935
:10B54000606803F0D1FC0028F5D0032D09D16049D3
:10B55000606803F0C9FC88B9A068BDE83840FFF70F
:10B5600079BD042D0AD15B49606803F0BDFC28B9A0
:10B57000E168A068BDE83840FFF786BD56496068BD
:10B5800003F0B2FC30B9032D7AD1A068BDE8384091
:10B59000FFF7A8BD5149606803F0A6FC00BB042D6D
:10B5A0006ED14F49A06803F09FFC20B9E068BDE868
:10B5B0003840FFF7B7BD4B49A06803F095FC20B9B0
:10B5C000E068BDE83840FFF7D1BD4749A06803F007
:10B5D0008BFC002854D1E068BDE83840FFF7EABD95
:10B5E0004249606803F080FC58B9032D48D14049B6
:10B5F000A06803F079FC002842D1BDE83840FFF78D
:10B6000011BE3C49606803F06FFC20B9032D37D1AF
:10B61000A168012007E03849606803F065FC30B993
:10B62000032D2DD1A168BDE83840FFF72BBF33496A
:10B63000606803F059FCD0B9022D21D03049A068D0
:10B6400003F052FCE0B9052D1AD12E49E06803F051
:10B650004BFC08B9012105E02B49E06803F044FCEC
:10B66000014668B92069BDE83840FFF735BF274972
:10B67000606803F039FC18B9BDE83840FFF7E0BD59
:10B68000234803F031FB234803F02EFB224803F04C
:10B690002BFB224803F028FB214803F025FB21481F
:10B6A00003F022FB204803F01FFB204803F01CFBA3
:10B6B0001F4803F019FB1F4803F016FB1E4803F058
:10B6C00013FB1E4803F010FB002038BDBF350108F6
:10B6D0008F110108C4350108C9350108CC350108AE
:10B6E0001C1D0108050D01086F0C01088C090108DB
:10B6F000D435010862350108673501081E1D0108AF
:10B70000D83501083E1C0108181D0108E920010870
:10B71000DC350108F43501082E36010867360108CA
:10B72000A0360108D936010810370108533701083F
:10B730009C370108D9370108FE370108493801084C
:10B74000F8B506460F46044623783D1B412B354489
:10B750000ED17B4803F0C8FA282D40F2EF80601C20
:10B76000FDF736FB1022A5F1290104F12900E1E0E3
:10B7700013F0C00F06D1734803F0B6FA1022294621
:10B780002046D7E003F0F802C02A11D16E4803F03A
:10B79000ABFA21886D4849BAC1F30A0103F01AFADD
:10B7A00061886B4849BA89B203F014FA0434CBE7D4
:10B7B000E02A17D1674803F097FA2188634849BA0D
:10B7C000C1F30A0103F006FA6188614849BA89B2F7
:10B7D00003F000FA2179604803F0FCF91022691F98
:10B7E000601DA7E003F0E003602B40F0A7805B48FA
:10B7F00003F07AFA237803F01803082B09D002D853
:10B8000063B9574808E0102B05D0182B06D15548CE
:10B8100002E0554800E0554803F066FA237803F04B
:10B82000040303F0FF0213B122B1514800E0514874
:10B8300003F05AFA237803F00303022B06D0032BFC
:10B8400006D0012B14BF4C484C4802E04C4800E0A5
:10B850004C4803F049FA637859060BD54A4803F07F
:10B86000B9F9637803F03003102B15D00ED8C3B9A3
:10B87000464814E0464803F0ADF9637803F030031E
:10B88000102B09D002D863B9424808E0202B05D01C
:10B89000302B06D1404802E0404800E0404803F029
:10B8A00023FA637813F0080F03F004031FD05BB191
:10B8B0003C4803F019FA637803F00303013B022BC1
:10B8C0008CBF3948394822E0394803F00DFA6378D3
:10B8D00003F00303022B06D0032B06D0012B14BF69
:10B8E0003448354813E0354811E035480FE03BB1A6
:10B8F000344803F06FF963789A070AD1324806E0BA
:10B90000324803F067F963789B0702D1214803F0BE
:10B91000EBF994F90130002B08DAA1782C4801F0FA
:10B920000F02090903F056F9032000E00220291A4A
:10B9300010222044BDE8F840FDF796BAF8BD00BFDC
:10B94000753801088E380108A8380108C538010883
:10B95000D9380108E5380108073901081539010807
:10B96000233901088139010849390108683901087A
:10B97000B4390108A9390108C3390108D0390108CF
:10B98000D8390108E1390108EB390108113A0108F9
:10B99000603A0108873A0108483A01082A3A010842
:10B9A000393A0108973A0108CA3A0108FC3A0108F5
:10B9B000093B01083D3B0108593B0108743B010864
:10B9C0008F3B0108A93B0108003B0108D33B01085C
:10B9D000FE3B010830B5036845688468C1680560AE
:10B9E00085EA040223F00043534083EA430381EADB
:10B9F000510183EA010242F3000583EA8223C26017
:10BA00000169426929402A404C40534044608360A8
:10BA100030BD036823F0004363B9436853B98368BA
:10BA200043B9C36833B9542149224E234FF0590C0E
:10BA300080E80E107047000038B503694360436921
:10BA40008360836901600446C3600F4801256B1E53
:10BA500003F0030305F0030254F8233054F82210D6
:10BA600083EA937300FB035301354B40082D44F8E0
:10BA70002230ECD12046FFF7CCFF2046FFF7AAFF8B
:10BA8000013DFAD138BD00BF6589076C2DE9F3414E
:10BA9000856804461DB919490320F5F7A5F84278D1
:10BAA00043689340C268C2EB05086A0093424FF0B6
:10BAB00000072CBF82608360478038BF5D088668BE
:10BAC000FDF70AFA711BB0FBF1F202FB110005440D
:10BAD000B4F91030E5604FF47A7245446A4301933B
:10BAE00004F11C030093A262E7623B4604F13000BC
:10BAF00000F0C6F802B0BDE8F08100BFA50701085C
:10BB000010B5428803789A42044600D313B963699A
:10BB1000A06998472046BDE81040FFF7B7BF000076
:10BB2000826843689A4210B5044603D80649032048
:10BB3000F5F75AF83030F4F7D3FF6368A360204676
:10BB4000BDE81040FFF7A2BFA5070108F8B50C46F5
:10BB5000174606469DF818109DF81C201D461BB977
:10BB600010490320F5F740F803FA01F00E4B984214
:10BB7000F6D8002363802270656026826170FDF72D
:10BB8000ABF9C5EB8503B0FBF3F202FB13000544F0
:10BB9000E560A56026822462E7832046BDE8F84080
:10BBA000FFF774BFA5070108FEFFFF7F3030F4F7F1
:10BBB00097BF4388013343807047000010B5018868
:10BBC0004288044649BA52BA92B289B2064803F092
:10BBD00001F8A188E288054849BA52BA92B289B2FE
:10BBE000BDE8104002F0F6BF143C0108373C0108E4
:10BBF000F5F7E0BFB0F90010F6F7FCB838B5044629
:10BC00000020F5F7BFFD05460020F5F7BBFD401B02
:10BC1000A042F9D338BD000030B587B004460D46C8
:10BC2000F4F729FC40B11DB10E490320F4F7DCFF05
:10BC30002046FFF7E3FF13E00B4B009003900290C8
:10BC4000012168460493CDF814D0F5F783FF21460F
:10BC500001A82A46F4F776FF01216846F5F77AFF36
:10BC600007B030BDA5070108F1BB000830B4034D93
:10BC7000C560026130BC1380F4F744BFF5BB000817
:10BC800070B41146039ABDF91050044EC6600261AB
:10BC900015801A4670BCF4F755BF00BFF5BB00080D
:10BCA00070B58AB00021079106911049098803AC4C
:10BCB00009B2054643F23906019105A80094ADF892
:10BCC0000E600494FFF7DCFF2846F6F75CF96B88FA
:10BCD000B34202D16B68A34204D005A8F4F700FF79
:10BCE000012001E04FF0FF300AB070BDD402002007
:10BCF00010B5084B0446182240F83C3B02F064FDA6
:10BD0000082384F85630002384F8543084F85730E0
:10BD100010BD00BF8C3C010837B5044600F03CFB69
:10BD200094F854301BB90321204600F060FA002536
:10BD30000821684684F83650258701F07FFE9DF87B
:10BD40000030019A23F0010343F002038DF8003024
:10BD5000009B12BA1BBA204600F000F9BDF8001093
:10BD600049BA204689B200F0E5F82046232100F0C8
:10BD700028F920461A2100F015F92946204600F03E
:10BD80003DF920460122202100F0B8F92046012289
:10BD90004FF4807100F0B2F92A4620464FF400516A
:10BDA00000F0ACF9204601224FF4804100F0A6F9E2
:10BDB000204601224FF4805100F0A0F9012384F8BD
:10BDC0002830802220460C2100F057FA042120461A
:10BDD00000F065FA042100F0FD02204600F04DFA63
:10BDE0000321204600F05BFA032100F0F002204618
:10BDF00000F043FA082220460E2100F03EFA0F21FF
:10BE0000204600F04CFA1621204600F0F0F903B06D
:10BE100030BD10B590F857300133044680F85730E4
:10BE2000204600F094FAA0F11103DBB2012BF7D900
:10BE3000192818BF84F856001921204600F0D7F9B8
:10BE4000022384F8553010BD70B51D4690F855306A
:10BE50006E1C1344144680F8553013460A46F1B25E
:10BE600000F02FFA601970BD10B5012300F15502E2
:10BE70000021044600F025FA02221146204600F077
:10BE8000FCF963683BB1228F120504D520460321DB
:10BE9000BDE81040184710BDF8B50821044600F071
:10BEA000A6F915210746204600F0F9F960F07F0257
:10BEB000D2B215210646204600F0DFF906212046C1
:10BEC00000F095F90821204600F0E9F960F07F02C2
:10BED000D2B20821204600F0D0F90121204600F01E
:10BEE000DEF903060546F8D532462046152100F056
:10BEF000C4F90821204600F07AF93946204600F0BE
:10BF000076F9C5F38010F8BD38B50D460221044618
:10BF100000F0B3F9162D07D0204600F018FA85423C
:10BF2000FAD184F8545038BD204600F010FA1F288A
:10BF3000FAD0F6E710B50A0A044601F07F0180F84E
:10BF40002D2080F82C10202100F097F994F82C2057
:10BF500020462121BDE8104000F08FB92DE9F843BB
:10BF6000054616461F4600F12D0800246FF007090C
:10BF7000E2003046394601F0E5FF09FB04F208F81B
:10BF8000010F38323046394601F0DCFF04F124015C
:10BF9000C2B2C9B22846013400F06FF9082CE7D1CB
:10BFA000BDE8F883A1F10B020F2A07D890F83720DB
:10BFB0008A4203D080F8371000F00ABA7047002098
:10BFC000704737B50D0A4185CAB22221044600F0F8
:10BFD00054F92A462321204603B0BDE8304000F042
:10BFE0004CB9000008B5052100F059F9024B00F0EA
:10BFF0000F0033F9100008BD6C3C0108113109B283
:10C000001429A8BF142121EAE171024B5A5C0521D1
:10C0100000F033B9573C010808B52C2100F03FF976
:10C02000C0F3071008BD38B50C462C21054600F0BA
:10C0300036F9072C28BF072400F00F0040EA04124D
:10C04000D2B228462C21BDE8384000F016B908B518
:10C050002C2100F024F9C0F3420008BD0529A8BF37
:10C060000521002938B50C46A8BF0C464FF02C011D
:10C070000546B8BF072400F012F920F00E0040EA90
:10C080004402D2B228462C21BDE8384000F0F5B871
:10C0900038B505460C4699B10A782D2100F0EDF827
:10C0A0002E21284600F0FBF8637800F0F80203F038
:10C0B00007031A4328462E21BDE8384000F0DDB8BA
:10C0C00038BD08B5092100F0EAF800F00F00400083
:10C0D0005B3840B208BD0029C4BF494249B25B3158
:10C0E000C1F3430242F0C002092100F0C6B808B50E
:10C0F000072100F0D4F85B3840B208BD10B5038FBB
:10C100000446B2B30B43B1F5807F03870AD002D84F
:10C11000202925D010BDB1F5007F0ED0B1F5005F0C
:10C1200020D010BD00F12E01FFF7B2FF0421204600
:10C13000FFF794FF53222F2153E02E2100F0AFF898
:10C1400040F01002D2B22E21204600F096F81721BE
:10C15000204600F0A4F840F00202D2B2172140E0DD
:10C160002E212BE00E2100F09AF840F00402D2B20A
:10C1700036E023EA0103B1F5807F03870AD002D8B5
:10C18000202921D010BDB1F5007F09D0B1F5005FA5
:10C1900021D010BD4FF0FF31BDE81040FFF75EBF6A
:10C1A000172100F07CF8172100F0FD02204600F076
:10C1B00064F8238F9B0619D52E21204600F06FF8D6
:10C1C00000F0EF022E210CE02E2100F068F840F084
:10C1D0001002D2B2F6E70E2100F061F800F0FB0287
:10C1E0000E212046BDE8104000F047B810BD70B5E4
:10C1F00004460D46204600F0AAF8A0F11103DBB278
:10C20000012B0646F6D91F28F4D0032D02D12A4669
:10C21000082126E0A84227D0162801D1192D02E0D6
:10C22000192807D1162D0AD1092211462046FFF7F9
:10C230006BFE04E00F2802D1204600F094F80F2D89
:10C240000DD103212046FFF7D2FF2946204600F0FA
:10C2500026F8E06CF5F70CFA84F8545004E02A460E
:10C2600029462046FFF750FE304670BD90F840301A
:10C27000416CC06B0022F5F76BB870B504460D46F3
:10C280001646FFF7F3FF334645F0C002616CE06BE2
:10C2900001F025FDE06BBDE87040F5F799B838B5C1
:10C2A00004460D46FFF7E2FF45F080020023616C73
:10C2B000E06B01F014FD0546E06BF5F789F82846C0
:10C2C00038BDF7B504460F4615461E46FFF7CEFFAC
:10C2D000616CE06B4023012201F0F0FC3B46616C95
:10C2E000E06B012201F0EAFC0022E06B0196009273
:10C2F0002B46616CF5F788F8E06B03B0BDE8F040C1
:10C30000F5F766B810B50446FFF7B0FF616CE06B57
:10C3100020230122BDE8104001F0D0BC07B58DE814
:10C3200006000023416CC06B0122F5F76DF803B0E5
:10C330005DF804FB10B50446416CC06B012300227C
:10C3400001F0BCFCE06BBDE81040F5F741B808B562
:10C3500090F854300F2B04D00121FFF7A0FF00F01C
:10C360001F03184608BD10B50446FFF7F0FF0F285D
:10C3700011D1E06CF5F785F900214FF49970FFF7C2
:10C380004BFC01212046FFF78AFF00F01F00082820
:10C3900084F85400F5D110BD10B50446006DF5F7D2
:10C3A00070F900213E20FFF737FC206DF5F760F9AA
:10C3B00000213E20FFF730FC01212046FFF76FFFF0
:10C3C00000F01F0310F0170F84F85430F4D110BDA3
:10C3D00038B508210446FFF70AFF08210546204624
:10C3E000FFF75DFF94F8373000F0E00203F01F0321
:10C3F00020461A430821FFF740FF29462046BDE8A2
:10C400003840FFF7F4BE43680BB10021184770476E
:10C410002DE9F0470446884616461F46FFF797FF6A
:10C420008146002C00F0D3800F2840F0DF80B8F167
:10C43000180F66D02046FFF796FFB8F1270F00F2DD
:10C440002B81DFE818F04200290128003300290180
:10C4500029013B002901290129012901290129017B
:10C46000290129012901550029018B008F007E0037
:10C4700029018400290129012901930097009B00CB
:10C480009F002901A300AA002901290129012901EE
:10C4900029014E00BA00022F03D98B490320F4F77B
:10C4A000A3FB31882046FFF745FD94E0082FF4D820
:10C4B000D6E900232046FFF751FD8CE0022FECD88F
:10C4C00031882046FFF77DFD85E0012FE5D03178EA
:10C4D000A1F10B030F2B00F2EC802046FFF762FD69
:10C4E00079E0012FD9D03378002B40F0E2806CE066
:10C4F000022FD2D8B6F900102046FFF77FFD0225A3
:10C50000D9E0012FC9D83378013B052B63D8DFE888
:10C5100003F00507620C1403082102E00F2100E07C
:10C5200016212046FFF763FECBE0238F5A0540F12A
:10C53000C8802046FFF798FCC3E02046FFF7ECFBDD
:10C54000BFE0327820212046FFF7D8FD43E0012FDD
:10C55000A3D831782046FFF766FD36E032784FF4F5
:10C56000806116E032784FF4007112E032784FF4B7
:10C5700000510EE032784FF480410AE032784FF4F7
:10C58000006106E032784FF4805102E032784FF4D7
:10C5900080712046FFF7B2FD17E0012F3FF67DAF17
:10C5A000238FDB0503D43378052B40F2828096F984
:10C5B00000102046FFF752FD07E0012F3FF66DAF58
:10C5C00096F900102046FFF786FD012573E06FF015
:10C5D0001200BDE8F087B9F10F0F5DD03B4632463F
:10C5E00041462046BDE8F04701F0EABAB8F1270F0E
:10C5F000F4D801A353F828F0CBC40008DDC5000827
:10C6000097C40008ADC40008DDC50008DDC50008FA
:10C61000BDC40008DDC50008DDC50008DDC5000893
:10C62000DDC50008DDC50008DDC50008DDC5000862
:10C63000DDC50008DDC50008F1C40008DDC500083F
:10C640005DC5000865C5000843C50008DDC50008D4
:10C650004FC50008DDC5000803C50008DDC500089A
:10C660006DC5000875C500087DC5000885C50008B2
:10C67000DDC500088DC500089BC50008DDC50008A4
:10C68000DDC50008DDC50008DDC50008DDC5000802
:10C69000E3C40008BBC50008B8F1180F9ED06FF0C6
:10C6A00085050F212046FFF7A2FD15F1860F05D164
:10C6B00094E76FF01505B9F10F0FF2D02846BDE8E9
:10C6C000F0870120BDE8F087A50701082DE9F041BA
:10C6D0000446FFF73CFE0F2806464CD00F212046AB
:10C6E000FFF7DDFD022107462046FFF7D8FD7B0757
:10C6F000054603D5636801212046984738073AD597
:10C70000162E01D0112E05D1238F590433D563681D
:10C7100002212CE0192E01D0122E2CD194F8573082
:10C720001BB916490320F4F75FFA013BDBB284F82A
:10C73000573023B994F856102046FFF758FD636828
:10C74000CBB1228FD20416D505F0E000202809D005
:10C7500002D838B1BDE8F081602807D0A02803D006
:10C76000BDE8F081042102E0062100E00721204617
:10C77000BDE8F0411847BDE8F08100BFA5070108FA
:10C7800013B50446416CC06BF4F7B4FD0121E06CB5
:10C79000F4F7AAFEE06CF4F774FF0121206DF4F7C2
:10C7A000A3FE206DF4F764FF0D4B009401220021DD
:10C7B000A06CF4F7D3FE2046FFF7AEFA1C2120460A
:10C7C000FFF76DFD032807D11C22002104F10C00A6
:10C7D00002F0F8F8002001E04FF0FF3002B010BD89
:10C7E00007C400082DE9F34104460F4690461E4653
:10C7F000FFF788FD01220DF103012046FFF78EFDB2
:10C800009DF8035005F07F05023D37B3454505D936
:10C810002046FFF78FFD6FF0680521E0236A0133A2
:10C820002362636A2B442A46394620466362FFF737
:10C8300075FD022201A92046FFF770FD6EB10122AD
:10C84000B1182046FFF76AFD2046FFF773FD072168
:10C850002046FFF724FD307002E02046FFF76AFD16
:10C86000284602B0BDE8F0812DE9F04106460D46AC
:10C870009046FFF7CEFA00273C46474512D06A683B
:10C88000A31C13447F2B05F1080514D8F36955F850
:10C89000081C2344F36130462346FFF7D5FA0137DD
:10C8A0000446EAE7338F5B0502D43046FFF7DCFA33
:10C8B0002046BDE8F0816FF08A00BDE8F0810000FD
:10C8C00008B5FFF744FD0838C0B211289ABF024BE3
:10C8D000185C022008BD00BFA43C01082DE9F84304
:10C8E0000F46164698460546002800F0B780A1F18D
:10C8F0001103152B4DD8DFE803F01827344C4C4CAE
:10C900004C204C383C40444C484C4C4C4C4C4C0B10
:10C91000B8F1010F03D857490320F4F765F9002354
:10C920007370FFF74CFB307004E0B8F1010FF2D9DF
:10C93000662333800220BDE8F883B8F1000FEAD007
:10C94000FFF7BEFF307009E0038F13F4806F03D050
:10C9500001203070BDE8F883002333700120BDE86A
:10C96000F883038F13F4007FF1E7038FC3F34033A1
:10C97000F3E7038FC3F38033EFE7038FC3F3C023E1
:10C98000EBE7038FC3F30033E7E7038FC3F3002321
:10C99000E3E74346324601F05FF810F1860F0446A4
:10C9A00060D12846FFF7D3FC0F28814611D12846D5
:10C9B000FFF7D9FC162F1CD004D8012F35D0102F2B
:10C9C0000ED046E0272F28D02F2F36D0202F1DD075
:10C9D0003FE0162F0DD013D8012F26D0102F44D1B1
:10C9E000B8F1010F97D92846FFF7FCFA02243080EE
:10C9F0002CE0B8F1000F8ED02846FFF70DFB23E0A6
:10CA0000272F0AD02F2F18D0202F2ED1B8F1000FAA
:10CA100081D02846FFF71BFB16E0B8F1000F3FF46A
:10CA20007AAF2846FFF74DFB0EE0B8F1000F3FF458
:10CA300072AF2846FFF730FA06E0B8F1000F3FF476
:10CA40006AAF2846FFF753FB30700124B9F10F0F8E
:10CA500008D10F212846FFF7CAFB03E06FF0120050
:10CA6000BDE8F8832046BDE8F8836FF08500BDE897
:10CA7000F88300BFA5070108BFF34F8F0549064B98
:10CA8000CA6802F4E0621343CB60BFF34F8F00BF6C
:10CA9000FDE700BF00ED00E00400FA050121F5F715
:10CAA00059B810B50446406908B101F097F9E0693A
:10CAB00008B101F093F90020002200236061206199
:10CAC000E061A0612080C4E9022310BDF3F792BFAA
:10CAD0002DE9F04F89B08A4615469B460446FFF77C
:10CAE000F5FFCDE90401EB0003930793554453464A
:10CAF000AB4205D013F8012B002AF9D0002300E047
:10CB00000123002702936FF075030193B846B946DD
:10CB10003E46A268974270D222687D0102EB050E64
:10CB2000DEE90201002908BFB0F1FF3F23D0DDE9B3
:10CB30000423994208BF90421DD200220023CEE96F
:10CB4000022322682A44166122682A4496612268D8
:10CB5000565322682A44506920B101F03FF92268F7
:10CB60002A44566122682A44D06920B101F036F97E
:10CB700022682A44D661039B98453CD222682A4405
:10CB80005069002837D007AA514601F05DF938B93D
:10CB900023681D44129BCBF800500120186034E03C
:10CBA000029B13B102282DD1F2E7012814D122688B
:10CBB0001544296911F07F4F1BD0079AB2EB116F12
:10CBC00017D3B8F1000F01D0904512D20023CBF853
:10CBD0000050904601930AE002280AD1B8F1000FF4
:10CBE00007D12268CDF804801544CBF800504FF0EF
:10CBF0000109039B079301378BE7129B0198C3F848
:10CC0000009002E00128F4D1D1E709B0BDE8F08F2F
:10CC100038B505460C46FFF759FF4FF47A736B435E
:10CC2000C01841F10001C4E9000138BD2DE9F04709
:10CC300088B0972990461BBF109A0792424605AAD2
:10CC40008A461CBFCDF814808DF81830ADF8061058
:10CC50000292DF0000F1120500F1200600F11C0431
:10CC60006FF0010935F9023FDBB1BAF1970F03D03C
:10CC700000976A46414607E0D8F8183019684B78A3
:10CC8000DB0000936A460231306801F0DDF80230C3
:10CC900007D0B5F9002003A901A8F5F715F94FF061
:10CCA0000009A54206F10406DCD1484608B0BDE8FB
:10CCB000F087000030B587B006AA102302AD2946E0
:10CCC00042F8143D01F0A2F8A842014620D1019B90
:10CCD000102B08D128220F48FBF74AFF01460E48C7
:10CCE00001F078FF14E00024019BA34204D3295DE6
:10CCF0000A4801F06FFF02E0094801F06BFF0134C0
:10CD0000102CF1D10724074801F064FF013CFAD14F
:10CD100007B030BDFC490020B63C01080E1F0108D9
:10CD2000F01A0108F11A01082DE9F04F00F10C0783
:10CD300087B0044638469A468B469046149EFFF7C5
:10CD4000ADFE01230493B8F1000F01D0119B2BB964
:10CD50003846F4F72FFF6FF00D006AE004AB009344
:10CD6000524605AB41462046FFF7B2FE012802D0ED
:10CD70004FF000091CE012991198059C00F0CCFFBF
:10CD8000054610B96FF00B044FE0E06901F026F89A
:10CD9000139BE561721CA36102D004F1080139E024
:10CDA0004FF0FF320023C4E902233DE009F10109FD
:10CDB000A2689145E6D222684FEA49152A44D2E991
:10CDC000020150EA0103F1D151464046039200F0BE
:10CDD000A3FF039A506122682A44516971B1109BE4
:10CDE00013612268129911982A44039200F094FF6B
:10CDF000039A139BD06122682A44936122682A44D3
:10CE0000D1690029D2D0A2F800B0731C216805D0E6
:10CE1000294408313046FFF7FBFE05E00D444FF092
:10CE2000FF320023C5E9022300243846F4F7C2FE8E
:10CE3000204607B0BDE8F08F2DE9F04300F10C0566
:10CE400085B0044628461F46884691460E9EFFF749
:10CE500025FE01230293B8F1000F00D02FB9284618
:10CE6000F4F7A8FE6FF00D002CE002AB00934A46E9
:10CE700003AB41462046FFF72BFE012802D06FF09E
:10CE80000B041BE038460C99039C00F045FF074655
:10CE90000028F4D0E06900F0A1FF0D9BA361731C92
:10CEA000E76105D004F108013046FFF7B1FE04E068
:10CEB0004FF0FF320023C4E9022300242846F4F790
:10CEC00079FE204605B0BDE8F083F0B500F10C0412
:10CED00085B0054620460E461746FFF7DFFD0123C5
:10CEE000029302AB00933A4603AB31462846FFF764
:10CEF000EFFD012802D10398FFF7D3FD2046F4F798
:10CF000059FE05B0F0BDF8B500F10C0605463046F7
:10CF10000F46FFF7C3FD0024AB689C420AD2286885
:10CF2000630117B1C25EBA4202D11844FFF7B9FDDE
:10CF30000134F1E73046BDE8F840F4F73BBE2DE997
:10CF4000F04F00F10C0485B0054620469B4689460B
:10CF500092460F9EFFF7A2FD01230293B9F1000F45
:10CF600004D0BBF1000F01D00E9B2BB92046F4F783
:10CF700021FE6FF0150049E016B1BAF1000F05D19E
:10CF80002046F4F717FE6FF00D003FE002AF009768
:10CF900003AB109A31462846FFF79AFD01288046D8
:10CFA00015D9119B00933246109B99212846FFF713
:10CFB0003DFE48B901230293009703AB109A314616
:10CFC0002846FFF785FD8046B8F1010F0CD8039B7A
:10CFD0005A465146D86900F019FF58B92046F4F76F
:10CFE000E9FD6FF0680011E02046F4F7E3FD6FF013
:10CFF00075000BE0039BB3F90020A9F800200E9AFE
:10D000009B6913602046F4F7D5FD002005B0BDE80C
:10D01000F08FF8B50646002546F80C5F044630460A
:10D02000FFF73CFD04F1120204F11C0304F130018E
:10D0300022F8025F43F8045F8B424FF00007F7D1FC
:10D0400023792761022BA2680BD12368520139464C
:10D05000186801F0B7FC23689A685868D20039460E
:10D0600002E020685201394601F0ACFC00F04EFFAE
:10D070003046BDE8F840F4F79DBD00002DE9F04FC3
:10D08000044600F10C0585B02846FFF707FDFFF7C1
:10D090001DFD2379012B804689466AD1674A684B7A
:10D0A000684969488DE80C00684B01F093FD4FF02A
:10D0B000000BA3689B456BD221684FEA4B1A514481
:10D0C000D1E90223134351D04869FFF7F3FD2368E8
:10D0D0005F485344196901F07DFD23685344196981
:10D0E00011F07F4F04D0090E5A4801F073FD02E0A1
:10D0F000594801F06FFD23685344D869FFF7DAFD02
:10D10000236853485344996901F064FD23685344EC
:10D11000D3E90267002F08BFB6F1FF3F1CD0B6EB82
:10D12000080667EB0907002E77F1000301DA4B4987
:10D1300013E0304639464A4A002300F00FFF00232F
:10D1400003923046464A394600F008FF039A0146EA
:10D15000444801F03FFD03E04349444801F03AFDF3
:10D160002368434833F90A1001F034FD0BF1010B39
:10D170009FE7022B0CD1324B00933E4A3E4B3F4976
:10D180003F4801F027FD4FF0000BA3689B4505D3F6
:10D19000284605B0BDE8F04FF4F70CBD23681968C8
:10D1A0004FEA4B1A5144D1E90223134343D08B6910
:10D1B0001868FFF77FFD23681B6853445B69186894
:10D1C000FFF778FD23682F481B685344196901F065
:10D1D00001FD23681B685344D3E90267002F08BF91
:10D1E000B6F1FF3F1CD0B6EB080667EB0907002E2F
:10D1F00077F1000301DA194913E030463946184A3D
:10D20000002300F0ABFE002303923046144A394657
:10D2100000F0A4FE039A0146124801F0DBFC03E093
:10D220001149124801F0D6FC236811481B6833F9F4
:10D230000A1001F0CFFC0BF1010BA6E7F93D010844
:10D24000B43D01080F3E01088B3D0108823D0108F5
:10D25000BC3D0108C63D0108CF3D0108D73D01088E
:10D2600040420F00E63D0108F03D0108DF3D0108A6
:10D27000DB3C0108FF3D0108F63D01080C3E0108BA
:10D280001B3E01083D3E010838B1054B0A0901F07B
:10D290000F019A5C5B5C027043700220704700BF14
:10D2A000473E010803461A78591C0AB10B46FAE7B3
:10D2B000181A7047F8B505460F4616468C18BC423A
:10D2C00006D0284614F8011DFFF7DEFF0544F6E7F7
:10D2D0007000F8BD07B502AB042243F8041D1946DF
:10D2E000FFF7E8FF03B05DF804FB38B505460C46D0
:10D2F0004CB122462946012002F0C6F9002802DB83
:10D30000241A0544F4E738BD07B5014601A8FFF724
:10D31000BBFF022101A8FFF7E8FF03B05DF804FBA3
:10D3200007B501466846FFF7D5FF08216846FFF7B5
:10D33000DCFF03B05DF804FB10B50446FFF7B2FF55
:10D3400001462046BDE81040FFF7CFBFF8B50646BE
:10D3500084890F46154600206DB90023B289B16853
:10D36000FBF778FB4FF6C57302199A4239680EDD58
:10D37000013080B20BE0AE42EFD02346AA89A96803
:10D38000FBF768FBEB686D681C44A4B2E4E73A3431
:10D39000204400232022083180B2FBF75BFBC0430E
:10D3A00080B2F8BD2DE9F3410C46804603212046AA
:10D3B000F7F7B9FA054618B92E490320F3F714FC1C
:10D3C0000221F7F7B0FA07460028F5D0EB68032BE7
:10D3D0004CD900F1080122462846AE68FFF7B6FF97
:10D3E000002843D13378803B082B30D8DFE803F0A6
:10D3F000052F2F2F2F0C151E2700AB89B968324639
:10D40000404600F081F822E0EB680093BA683346AA
:10D4100021464046F5F77CFF19E0EB680093BA68B7
:10D42000334621464046F5F7F5FF10E0EB680093E0
:10D43000BA68334621464046F5F7D4FD07E0EB686D
:10D440000093BA68334621464046F5F797FE317897
:10D45000234640F201220320F6F748FF014628B98F
:10D46000204602B0BDE8F041F7F7D2BC02B0BDE8FB
:10D47000F08100BFA507010838B50D46144600210C
:10D480001A460323F7F7D2FB28B1836800221D70E8
:10D490005C709A70DA7038BD10B5044668B190F9C6
:10D4A0001030032B0CD142680831FFF74FFF50B109
:10D4B000A36840BA5880002010BD6FF00D0010BD69
:10D4C0006FF04C0010BD6FF0010010BD2DE9F04170
:10D4D000DDF81880154600220E461F46014608F169
:10D4E00008031046FFF7C8FF044650B1806876BABB
:10D4F0006DBA8680C58027B142463946083001F0B2
:10D5000063F92046BDE8F081F7B506460C46002ACF
:10D5100038D0072B36D99188D088083B40BA49BA11
:10D52000009389B202F1080382B28120FFF7CEFF97
:10D53000074638B3237EFF2B04F108020CBF0021FD
:10D5400004F11801F5F736F9054610B901463846D9
:10D5500013E000231A4619461846F7F737F983688F
:10D5600009495E8004464560034640F202220220DB
:10D57000F6F7BCFE014628B9204603B0BDE8F040EE
:10D58000F7F746BC03B0F0BD0000FFFF38B5054615
:10D590000C4619B301F17000F3F7A2FA2846F5F72B
:10D5A0008BFA38B1D0F810329C4203D100F5FC70F0
:10D5B000F3F796FA04F11C00F3F792FA04F138003D
:10D5C000F3F78EFA04F15400F3F78AFA10220021DF
:10D5D000204601F0F7F900236383637638BD00002D
:10D5E00008B51022034901F0BDF8B0FA80F04009F7
:10D5F00008BD00BFCC0F01082DE9F74F9046009001
:10D600001E469DF83070894609B900205CE0082B61
:10D61000FBD80846FFF7E4FF0028F6D1824604460F
:10D620004FF0980B2A4B0BFB0AF29D1849462846EF
:10D630000192FBF736FA019A78B1B8F1000F42D0A7
:10D64000002E40D0224B02F11000414632461844D1
:10D6500001F0BAF82E766F7635E02846FFF7C0FF66
:10D6600010B1002C08BF2C460AF1010ABAF1080FCC
:10D67000D8D1002CC9D0BDF80030638310224946B0
:10D68000204601F0A1F8B8F1000F07D036B13246BC
:10D69000414604F1100001F097F82676677607F00E
:10D6A0000707022F04BF032384F894304FF4097353
:10D6B000A4F886304FF40473C4F88840638664632A
:10D6C0002465204600E0284603B0BDE8F08F00BF87
:10D6D000244A00202DE9F04107460E4611B90020EA
:10D6E000BDE8F0810846FFF77BFF0028F7D10C4D1D
:10D6F0000446A846B5F91A3013B10FB1BB4209D19F
:10D7000031462846FBF7CDF920B1982000FB048074
:10D71000BDE8F0810134082C05F19805EAD1DEE777
:10D72000244A002010B50446FFF7D4FF01462046E6
:10D73000BDE81040FFF72ABF38B510B100F19804DA
:10D7400000E0074C074DAC4205D22046FFF748FFEA
:10D7500018B19834F7E7002038BD204638BD00BF27
:10D76000244A0020E44E002008B5FFF7E5FF10B181
:10D77000437E1B07F9D508BDF8B501460020FFF729
:10D78000A9FF044610B3437E13F0050F1ED0B0F975
:10D790001A00F5F791F90E4BD0F8D461B3F9007087
:10D7A00004F138052846F3F79BF940F21723A4F853
:10D7B0004E3004F14C023B4631462846FEF756FAFD
:10D7C000637E23F0070343F0070363762046F8BD2A
:10D7D0008410002010B5144600B119B90B4903207C
:10D7E000F3F702FA2AB1537E03F00703013B012B42
:10D7F00001D8002010BD137E0B70127E04F11001C1
:10D8000000F0E2FFB4F91A0010BD00BFA50701083F
:10D81000F0B503EB43048C424FF0000122D80170B5
:10D8200005465E1E0F464FF03A0E994219D0147805
:10D830002409092C94BF3034573494462C709CF83A
:10D84000004004F00F04092C94BF30345734B14227
:10D850006C700CBF3C467446AC700132013103352C
:10D86000E3E7F0BD0846F0BD2DE9F04112B9002014
:10D87000BDE8F0811378002BF9D014462646013418
:10D880007378002BFAD107464FF0010C964217D35C
:10D890003478A4F130055FFA85F8B8F1090F06F184
:10D8A000FF3E23D9A4F14105052D02D8A4F1370587
:10D8B0001CE0A4F16105052D11D8A4F1570515E070
:10D8C000BCF1000FD3D1013FB84205D23A780178BC
:10D8D000397000F8012BF6E71846BDE8F081BCF17D
:10D8E000000FC4D14FF0010C7646CFE7724518D82F
:10D8F000A6F1020E16F8016CA6F130045FFA84FC62
:10D90000BCF1090F0ED9A6F14104052C02D8A6F1ED
:10D91000370407E0A6F16104052C02D8A6F15704EC
:10D9200000E0002401338B42A1D845EA04143C7086
:10D930004FF0000C0137D7E710B5044686B0B0F9B8
:10D940000210214801F046F96179204801F042F9BE
:10D95000A1791F4801F03EF91E4801F03BF92379F7
:10D9600063B11A0602D51C4801F034F923795B062D
:10D9700002D51A4801F02EF9194800E0194801F0C3
:10D98000B3F9237853B104F1080218216846FFF770
:10D990003FFF0146144801F01DF902E0134801F071
:10D9A000A3F963785BB122780832224418216846D3
:10D9B000FFF72EFF01460E4801F00CF902E00D487A
:10D9C00001F092F906B010BD573E0108643E01080F
:10D9D0006F3E0108783E0108803E01088B3E010839
:10D9E0007E340108963E01089A3E0108AA3E0108CD
:10D9F000BC3E0108CC3E01087FB50C46054600B18F
:10DA000019B90D490320F3F7EFF80A4601AE2321B7
:10DA100000F0D8FF304600F04BF90023B3FBF4F2DE
:10DA200004FB1232F15CA85C013341400C2BA95479
:10DA3000F4D104B070BD00BFA507010810B50446BD
:10DA4000FFF7DAFF034B1A78511C19702378534003
:10DA5000237010BD5E020020062938B504460D462D
:10DA6000104636D006D8032922D029D8B1B30229CE
:10DA700011D09DE017294AD004D8082951D0152982
:10DA800032D095E0252948D0292900F0898019292C
:10DA900040F08E8035E0012B03D848490320F3F78E
:10DAA000A3F80A4604F12C0100F08EFE284638BD8A
:10DAB000072BF2D9082204F12E0100F085FE7AE04E
:10DAC000022BEAD1228F520701D5082204E00380FD
:10DAD0006CE0022BE1D1628D028067E0022BDCD189
:10DAE00094F8373013800AE0012BD6D1238F13F03E
:10DAF000200F02D00123037058E00023037001209F
:10DB000038BD012BC9D1238F13F0020FF1E7012B90
:10DB1000C3D194F92820027048E0022BBDD1032222
:10DB2000DAE7072BB9D9238F5B074CBF2B460223BB
:10DB30004FF000024CBF04F12E0104F12C01042B24
:10DB40004270027018D0082B03D0022B33D1134639
:10DB500019E00A7882F0020202704A7842708A78EC
:10DB60008270CA78C2700A7902714A7942718A79E0
:10DB70008271CA79C27119E00B7883F002030370D5
:10DB80004B7843700223FF240022C470FE2482706D
:10DB900004714271CA5C827119444B78C3710AE006
:10DBA000042B7FF47AAF04F10C011160184638BDE4
:10DBB0006FF0850038BD082038BD00BFA5070108FB
:10DBC00070B515461C4619296AD8DFE801F00D69C1
:10DBD00019293939496969696969696969696969C5
:10DBE0006969694E69616958022C03D02F49032085
:10DBF000F2F7FAFF1388FF2BF8D880F837304DE0A2
:10DC0000022CF3D800F12C0602220021304600F04D
:10DC1000D9FE22462946304600F0D6FD022070BDCE
:10DC2000082CE3D800F12E0608220021304600F02F
:10DC3000C9FE22462946304600F0C6FD082070BDC8
:10DC4000022CD3D11388022B06D0082B2BD1038FA3
:10DC500043F00403038721E0038F23F004030CE067
:10DC6000022CC3D11388438518E01278038F12B1B8
:10DC700043F0200301E023F020030387CEE712786E
:10DC8000038F12B143F00203F7E723F00203F4E736
:10DC9000012CABD192F9003080F82830204670BDBD
:10DCA0006FF0850070BD6FF0690070BDA5070108B9
:10DCB0000C22014900F088BD107AFF1F10B586B014
:10DCC00006AC04F8093D012301930DF117030093FD
:10DCD0002346F3F799FB9DF8170006B010BDF0B589
:10DCE00085B01F4604AB002403F8012D0122054630
:10DCF0000E4601920094F3F787FB3B4622463146DD
:10DD00002846FFF7DBFF05B0F0BD00000121014808
:10DD1000F3F720BFE44E00202DE9F04780460E4681
:10DD2000FFF7F4FF294C002514F8013C9E420AD16C
:10DD300032464146204600F015FD20B9244B1224FE
:10DD400004FB053428E00135282D04F11204EBD141
:10DD5000204B1B68272B33D81D4B0025122202FBBA
:10DD600005F91B4F19F803A0BAF1000F25D107EBF5
:10DD7000090463789E4207D010225146A01C00F08F
:10DD800021FE07F809A06670122000FB05703246DC
:10DD90004146023000F018FD23780F480133DBB212
:10DDA000012B08BF0B4A237002BF136801331360B5
:10DDB000F3F700FF2046BDE8F0870135282DCED1CE
:10DDC0000548F3F7F7FE0020BDE8F087EE4E00208F
:10DDD000EC4E0020E84E0020E44E002010B5044632
:10DDE000FFF794FF4CB123783BB1013BDBB22370CA
:10DDF0001BB9044A1368013B13600348BDE8104097
:10DE0000F3F7D8BEE84E0020E44E002070B515466A
:10DE100006460C46FFF77AFF72782B6893420AD3C6
:10DE2000B11C204600F0D0FC73782B600548F3F756
:10DE3000C1FE204670BD2A600248F3F7BBFE0020F9
:10DE400070BD00BFE44E00202DE9F04117460646A4
:10DE50008846FFF75BFF72783B68B3EBC20F05D1D2
:10DE6000B01C002501244FF0FF3316E02648F3F7DD
:10DE7000A1FE6FF00100BDE8F081591C37D190F888
:10DE800000E018F80510714537D02B46C4B1BEFA32
:10DE90008EF46409A4B1013501309542EDD33CB153
:10DEA00000233B601848F3F785FE0220BDE8F081AF
:10DEB0005D1C05D11448F3F77DFE2046BDE8F081D6
:10DEC0001E4418F80310B2784A40072142FA01F4C0
:10DED000E40748B202D40139F8D1084600EBC30385
:10DEE0003B600948F3F766FE0120BDE8F081002C95
:10DEF000E6D00478B4FA84F4CBE7002CCBD0B1FAA6
:10DF000081F46409C7E700BFE44E002070B5FFF755
:10DF1000FDFE0A4C002504F5347604F8025C04F892
:10DF2000015C204610220021123400F04BFDB44267
:10DF3000F3D10348BDE87040F3F73CBEEE4E00203D
:10DF4000E44E0020D0400B1CD1409C46203AD340E8
:10DF500018435242634693401843704753B94AB935
:10DF6000002908BF00281CBF4FF0FF314FF0FF30E1
:10DF700000F07EB9ADF1080C6DE904CE00F006F8B2
:10DF8000DDF804E0DDE9022304B070472DE9F04735
:10DF90008C460E460446089D002B50D18A421746F7
:10DFA0006CD9B2FA82FEBEF1000F0BD0CEF1200484
:10DFB00020FA04F401FA0EF644EA060C02FA0EF70F
:10DFC00000FA0EF44FEA1749220CBCFBF9F01FFAD5
:10DFD00087F809FB10C642EA064600FB08F3B34285
:10DFE00009D9F61900F1FF3280F02281B34240F2E4
:10DFF0001F8102383E44F61AA2B2B6FBF9F309FBC0
:10E00000136642EA064403FB08F8A04509D9E4195F
:10E0100003F1FF3280F00A81A04540F20781023B04
:10E020003C44C8EB040443EA00400021002D62D0C8
:10E0300024FA0EF400232C606B60BDE8F0878B425D
:10E0400007D9002D55D0002185E841000846BDE8DC
:10E05000F087B3FA83F1002940F09080B34202D3F5
:10E06000824200F2F880841A66EB03060120B4466F
:10E07000002D40D085E81010BDE8F08712B90127C7
:10E08000B7FBF2F7B7FA87FEBEF1000F35D1F31BED
:10E090004FEA17481FFA87FC0121B3FBF8F0220C66
:10E0A00008FB103642EA06460CFB00F3B34207D9E0
:10E0B000F61900F1FF3202D2B34200F2CE801046D0
:10E0C000F61AA2B2B6FBF8F308FB136642EA06445E
:10E0D0000CFB03FCA44507D9E41903F1FF3202D27B
:10E0E000A44500F2B5801346CCEB040443EA00409B
:10E0F0009CE729462846BDE8F087CEF1200106FAC4
:10E100000EF307FA0EF720FA01F94FEA1748CE404E
:10E1100049EA0309B6FBF8FA4FEA194408FB1A6604
:10E120001FFA87FC44EA06430AFB0CF29A4200FA03
:10E130000EF40AD9DB190AF1FF3180F087809A4288
:10E1400040F28480AAF1020A3B449B1A1FFA89F923
:10E15000B3FBF8F108FB113349EA034301FB0CF66A
:10E160009E4207D9DB1901F1FF326BD29E4269D979
:10E1700002393B449B1B41EA0A418EE7C1F1200E64
:10E1800022FA0EF48B40234320FA0EF706FA01F42C
:10E190004FEA134C26FA0EF63C43B6FBFCF9270C6B
:10E1A0000CFB19661FFA83F847EA064609FB08F7D5
:10E1B000B74202FA01F200FA01FA08D9F61809F199
:10E1C000FF3041D2B7423FD9A9F102091E44F61BE4
:10E1D000A0B2B6FBFCF40CFB146640EA064704FB55
:10E1E00008F8B84507D9FF1804F1FF3028D2B84520
:10E1F00026D9023C1F4444EA0940C8EB0707A0FBAC
:10E2000002894F4544464E4614D329D065B3BAEB34
:10E21000040367EB060707FA0EFECB40CF404EEA39
:10E22000030385E888000021BDE8F0871346F8E67F
:10E230001046E0E6B8EB020469EB03060138E5E7B7
:10E240000446D8E7114695E78146C0E78A467CE751
:10E25000023B3C4448E708460AE702383E442FE7C1
:10E26000C245E7D33E46D1E72946BDE8F08700BF67
:10E27000704700BF0A22002101F054B90A2300228E
:10E2800001F0BCB8014B1868704700BF6002002065
:10E290008B891A072DE9F0410D46804635D44A682E
:10E2A000002A6BDDEC6A002C47D003F48052002179
:10E2B00092B2D8F80060C8F80010002A62D06A6DE7
:10E2C0005F0705D569686B6B521A0BB12B6CD21ABC
:10E2D0000023296A4046A047441C39D0AB892A69EB
:10E2E0002A60DB044FF000026A6045D4696BC8F80D
:10E2F000006011B305F14403994202D0404600F09A
:10E30000AFFB00206863BDE8F0810E69AEB10C6818
:10E310000E6098070CBF4B690023A41B8B600AE0BA
:10E3200023463246AF6A296A4046B8470028A4EB24
:10E330000004064404DD002CF2DC0020BDE8F0817E
:10E34000AB8943F04003AB814FF0FF30BDE8F08173
:10E35000D8F800201D2AF3D8184BD34003F001034E
:10E3600083F00101002BEBD0AB892C696960D904E3
:10E370002C60BBD5002AB9D16865B7E70A6C002AC2
:10E3800090DCDAE70123296A4046A047431C024695
:10E3900002D0AB89EC6A93E7D8F80030002BF8D0B4
:10E3A0001D2B01D0162B02D1C8F80060C5E7AB8940
:10E3B00043F04003AB81BDE8F08100BF0100402085
:10E3C0000B6933B310B5044682B008B18369ABB1B1
:10E3D000114B994219D0114B994218D0104B9942C8
:10E3E00008BFE168B1F90C3013B9002002B010BDCC
:10E3F000204602B0BDE81040FFF74ABF019100F08F
:10E4000019F90199044B9942E5D16168EAE7A168DD
:10E41000E8E70020704700BF203F0108003F0108E7
:10E42000E03E010820B1054B01461868FFF7C8BF60
:10E43000034B0449186800F043B900BF6002002094
:10E44000403F0108C1E3000800207047014900F087
:10E4500037B900BFC1E300080020704770B56823DA
:10E460004D1E03FB05F50E4605F1740100F03EFB61
:10E47000044640B100210C30666005F1680221605D
:10E48000A06000F09FFA204670BD00BF1F4B70B522
:10E490001D68AB69064613B9284600F039F84835BF
:10E4A0006B68AC68013B05D521E0013B5A1C04F1C7
:10E4B00068041CD0B4F90C20002AF6D100250123F1
:10E4C0004FF6FF72E281A38165662560A5606560F5
:10E4D00025616561A5612946082204F15C0000F010
:10E4E00071FA6563A563A564E564204670BD2B6879
:10E4F0000BB11D46D4E704213046FFF7AFFF28607B
:10E5000008B10546CCE70C23336070BD403F0108DD
:10E510003D4B3E491A682DE9F04F90424FF0000301
:10E520008364C364036508BF012383B008BF8361AC
:10E5300081620746FFF7AAFF78603846FFF7A6FF1B
:10E54000B8603846FFF7A2FF7D68F8600024042316
:10E55000AB812C606C60AC606C66EC812C616C6192
:10E56000AC61214605F15C00082200F02BFABE6880
:10E57000DFF89CB0DFF89CA0DFF89C90DFF89C806F
:10E58000C5F824B001230922C5F828A0C5F82C90AD
:10E59000C5F830802D622146F381B2813460746009
:10E5A000B460746634617461B46106F15C00082281
:10E5B000019300F007FAFD68366212200222C6F8C5
:10E5C00024B0C6F828A0C6F82C90C6F830802146A2
:10E5D000A881EA812C606C60AC606C662C616C6117
:10E5E000AC6105F15C00082200F0ECF9019B2D62A2
:10E5F000C5F824B0C5F828A0C5F82C90C5F830801F
:10E60000BB6103B0BDE8F08F403F01084DE4000856
:10E6100069ED000891ED0008CDED0008EDED000872
:10E62000024B0349186800F04BB800BF403F010897
:10E63000C1E30008836903B96AE77047704700BF08
:10E64000704700BF704700BF704700BF024B0349CF
:10E65000186800F00FB800BF6002002059E40008FD
:10E66000024B0349186800F005B800BF60020020A3
:10E6700049E400082DE9F04110F148071BD0884615
:10E6800000267D68BC68013D0FD4A389012B05F1EC
:10E69000FF3506D9B4F90E300133204601D0C0470A
:10E6A00006436B1C04F16804EFD13F68002FE8D1EA
:10E6B0003046BDE8F0813E463046BDE8F08100BFFF
:10E6C0002DE9F84310F148071FD0884606464FF061
:10E6D00000097D68BC68013D11D4A389012B05F1B7
:10E6E000FF3508D9B4F90E3001332146304602D047
:10E6F000C04749EA00096B1C04F16804EDD13F688A
:10E70000002FE6D14846BDE8F883B9464846BDE843
:10E71000F88300BF70B50F4E0F4D761BB61018BFB3
:10E72000002405D0013455F8043B9847A642F9D19E
:10E730000A4E0B4D761BF1F729FDB61018BF0024C9
:10E7400006D0013455F8043B9847A642F9D170BD74
:10E7500070BD00BF8840010888400108884001085A
:10E7600088400108032A70B426D940EA01039B07B8
:10E7700011D004780D78AC4222D10244431C05E04C
:10E7800013F8014B11F8015FAC4219D19342F7D154
:10E79000002070BC70470C4603461E682568AE42D8
:10E7A0001846214603F1040304F10404E1D1043ABC
:10E7B000032A18462146F0D8002ADAD11046E8E7A5
:10E7C000601B70BC704700BF844641EA000313F031
:10E7D00003036DD1403A41D351F8043B40F8043B68
:10E7E00051F8043B40F8043B51F8043B40F8043B2B
:10E7F00051F8043B40F8043B51F8043B40F8043B1B
:10E8000051F8043B40F8043B51F8043B40F8043B0A
:10E8100051F8043B40F8043B51F8043B40F8043BFA
:10E8200051F8043B40F8043B51F8043B40F8043BEA
:10E8300051F8043B40F8043B51F8043B40F8043BDA
:10E8400051F8043B40F8043B51F8043B40F8043BCA
:10E8500051F8043B40F8043B403ABDD2303211D36A
:10E8600051F8043B40F8043B51F8043B40F8043BAA
:10E8700051F8043B40F8043B51F8043B40F8043B9A
:10E88000103AEDD20C3205D351F8043B40F8043B6A
:10E89000043AF9D2043208D0D2071CBF11F8013B68
:10E8A00000F8013B01D30B8803806046704700BF2E
:10E8B000082A13D38B078DD010F003038AD0C3F13D
:10E8C0000403D21ADB071CBF11F8013B00F8013B1F
:10E8D00080D331F8023B20F8023B7BE7043AD9D3DE
:10E8E000013A11F8013B00F8013BF9D20B780370B3
:10E8F0004B7843708B788370604670478842F0B5E0
:10E900000DD98B1898420AD28118002A51D09A1A30
:10E9100013F8014D01F8014D9342F9D1F0BD0F2AD2
:10E9200048D941EA00039B0746D100F1100401F1E8
:10E930001003154653F8106C44F8106C53F80C6C27
:10E9400044F80C6C53F8086C44F8086C103D53F80C
:10E95000046C44F8046C0F2D03F1100304F110044F
:10E96000E8D8A2F1100323F00F0302F00F0E1033CA
:10E97000BEF1030F1944034421D91E1F0D467446EE
:10E98000043C55F8047B46F8047F032CF8D8AEF11C
:10E99000040424F0030404342344214402F0030259
:10E9A00062B1013B0A4411F8014B03F8014F8A425E
:10E9B000F9D1F0BD0346F3E70346F2E7F0BD724636
:10E9C000EEE700BF70B4840746D0541E002A41D041
:10E9D000CDB2034602E0621EE4B3144603F8015BC5
:10E9E0009A07F8D1032C2ED9CDB245EA05250F2C74
:10E9F00045EA054519D903F110022646103E0F2EAF
:10EA000042F8105C42F80C5C42F8085C42F8045C86
:10EA100002F11002F2D8A4F1100222F00F0204F069
:10EA20000F041032032C13440DD91E462246043A1B
:10EA3000032A46F8045BFAD8221F22F003020432AC
:10EA4000134404F003042CB1C9B21C4403F8011BA5
:10EA5000A342FBD170BC704714460346C2E700BF17
:10EA600030B481B151F8043C0439002BB8BFC91847
:10EA70001D4B1A682AB18A420AD908680C18A242AA
:10EA800025D04A60196030BC70478B4203D81A46C3
:10EA90005368002BF9D1146815198D420CD007D892
:10EAA00008680C189C4218D04B6030BC516070470D
:10EAB0000C23036030BC704709680C44111999425B
:10EAC0001460E0D10ACB0C4453601460DBE7146897
:10EAD00052684A6020440860D4E71C685B684B6059
:10EAE000204408605160CEE7BC51002070B5CD1CB9
:10EAF00025F0030508350C2D38BF0C25002D0646E2
:10EB00003BDBA94239D827490A6852B113685B1B1D
:10EB100004D436E023685B1B1AD522465468002CC7
:10EB2000F8D149681F4C002936D029463046F1F704
:10EB300031FB431C21D0C41C24F00304A04205D0A7
:10EB4000211A3046F1F726FB013016D0256004E08B
:10EB50000B2B0DD923601C44256004F10B0020F021
:10EB60000700231DC31A02D05A42E25070BD70BD87
:10EB700094420ED063685360EFE70C2333600020AB
:10EB800070BD0B2B03D8536814460B60E5E71446A1
:10EB9000E0E713461446F8E73046F1F7FBFA606009
:10EBA000C3E700BFBC5100200EB410B5044683B0CB
:10EBB00018B183690BB9FFF73DFD06A80346019024
:10EBC000059AA168204600F0F5FE03B0BDE81040AC
:10EBD00003B070470FB410B50A4B1C6882B024B163
:10EBE000A36913B92046FFF725FD05A80346019048
:10EBF000049AA168204600F0DDFE02B0BDE8104096
:10EC000004B07047600200202DE9F0410E468046B6
:10EC100000283ED08369002B39D084682F4B9C425A
:10EC200043D02F4B9C4256D02E4B9C4208BFD8F865
:10EC30000C40A3891B073DD52369002B3AD0013E28
:10EC4000A36816F8015F013BA360B5B1002B04DB9C
:10EC500023685A1C22601D70F2E7A769BB42224656
:10EC60002946404601DB0A2DF2D100F019FD0130A2
:10EC7000E6D14FF0FF30BDE8F081002B21DB2368A7
:10EC80000A22591C21601A701046BDE8F081FFF776
:10EC9000D1FCD8F81830D8F80840002BBED1404637
:10ECA000FFF7C8FC0D4B9C42BBD1D8F80440A389A8
:10ECB0001B07C1D42146404600F054FD0028BED0B9
:10ECC000D7E7224640460A2100F0EAFC0130D0D0C6
:10ECD0000A20BDE8F081D8F80840AAE7203F0108E3
:10ECE000003F0108E03E0108024B01461868FFF7AB
:10ECF0008BBF00BF6002002038B50C46054608B146
:10ED00008369B3B1114B9C4218D0114B9C4217D070
:10ED1000104B9C4208BFEC682846214601F080F960
:10ED200080B994E80C00013B511C84E80A0010787B
:10ED300038BDFFF77FFC054B9C42E6D16C68EBE7E2
:10ED4000AC68E9E74FF0FF3038BD00BF203F010855
:10ED5000003F0108E03E0108024B01461868FFF73A
:10ED6000CBBF00BF6002002010B50C46B1F90E10F9
:10ED7000F1F72EFA002803DB636D0344636510BDD1
:10ED8000A38923F48053A38110BD00BF00207047E6
:10ED90002DE9F0411646B1F90C201F46D3050C466B
:10EDA000054607D500220223B1F90E10F1F71DFA2E
:10EDB000B4F90C20B4F90E1022F48052A2813B4623
:10EDC00032462846BDE8F041F1F706BA10B50C46C8
:10EDD000B1F90E10F1F709FAA389421C0EBF23F412
:10EDE000805343F480536065A38110BDB1F90E10C8
:10EDF000F1F7F6B970B411F0FF0434D085070FD0E5
:10EE00000378002B5AD09C422BD0431C05E013F80A
:10EE1000012B002A4FD0944223D09A071846F6D1EE
:10EE20000E0206F47F462643036846EA064601E0E2
:10EE300050F8043F86EA0305A5F10132A3F1013140
:10EE400022EA050221EA0303134313F0803FEFD0C7
:10EE5000037823B932E010F8013F002B2ED09C42FA
:10EE6000F9D170BC704784070BD00378002BF8D021
:10EE7000431C03E002780133002AF2D099071846B8
:10EE8000F8D10268A2F1013323EA020313F0803FB4
:10EE900008D150F8042FA2F1013323EA020313F042
:10EEA000803FF6D00378002BDBD010F8013F002B19
:10EEB000FBD170BC7047104670BC7047184670BCE0
:10EEC000704700BF000000000000000000000000CC
:10EED0000000000000000000000000000000000032
:10EEE000A2EB0300704700BF02780B78012A28BF0D
:10EEF0009A42F5D16DE9044540EA0104CDE9026783
:10EF00006FF0000C4FEA447212B380EA010414F06F
:10EF1000070F6AD100F0070420F0070004F0030592
:10EF200021F007014FEAC505F0E8042314F0040FAF
:10EF3000F1E804670CFA05F462EA040266EA0406E2
:10EF40000AD063EA0403624667EA0407664603E000
:10EF5000F0E80423F1E8046782FA4CF582EA06043B
:10EF6000A4FA8CF46CBB83FA4CF583EA0705A5FA86
:10EF70008CF595B950E9022351E9026782FA4CF504
:10EF800082EA0604A4FA8CF483FA4CF583EA0705B6
:10EF9000A5FA8CF52543DBD09CB92DBAB5FA85F4DA
:10EFA00024F0070427FA04F1DDE9026723FA04F3E9
:10EFB00003F0FF0001F0FF01FDE80445A0EB0100B4
:10EFC000704724BAB4FA84F424F0070426FA04F152
:10EFD000DDE9026722FA04F202F0FF0001F0FF010E
:10EFE000FDE80445A0EB0100704714F0030F3CD18D
:10EFF00010F0030428D150F8082B51F8083B82FA8E
:10F000004CF582EA0305A5FA8CF55DB950F8042C9D
:10F0100051F8043C82FA4CF582EA0305A5FA8CF516
:10F02000002DE8D02DBAB5FA85F424F0070423FAB0
:10F0300004F122FA04F202F0FF0001F0FF01FDE802
:10F040000445A0EB010070474FEAC40420F0030020
:10F0500050F8082B21F0030151F8083B0CFA04F496
:10F0600062EA040263EA0403C9E710F003041AD059
:10F07000A1EB040120F00300E40750F8042B06D0B4
:10F080000FD28B785FFAA2F4E41A06D12BB1CB78B9
:10F090005FFAB2F4E41A00D11BB920465DF8104BB8
:10F0A000704701F1040150F8042BCC0721F0030153
:10F0B00051F8043B48D824D222F07F4482FA4CF520
:10F0C00094EA1325A5FA8CF50AD165B951F8043BE9
:10F0D00084EA0204B4EB036F0ED150F8042BEBE783
:10F0E0004FEA132355E035F07F454DD10878FDE810
:10F0F0000445C0F1000070474FEA126203F0FF03BD
:10F1000047E002EA1C4482FA4CF594EA1345A5FA5A
:10F110008CF50AD165B951F8043B84EA0204B4EBDA
:10F12000034F0CD150F8042BEBE74FEA134330E0C8
:10F1300015EA1C4528D10B884FEA124229E04FEA14
:10F14000124203EA1C4324E002F0FF0482FA4CF569
:10F1500094EA1365A5FA8CF50AD165B951F8043B18
:10F1600084EA0204B4EB032F09D150F8042BEBE737
:10F170004FEA13630DE015F0FF0F05D10B684FEA5E
:10F18000122223F07F4304E04FF00000FDE8044525
:10F19000704712BA1BBA82FA4CF482EA0304A4FA4A
:10F1A0008CF5B5FA85F402FA04F203FA04F34FEA97
:10F1B0001260FDE80445A0EB1360704780EA01028D
:10F1C000844612F0030F4FD111F0030F32D14DF8E6
:10F1D000044D11F0040F51F8043B0BD0A3F10132A0
:10F1E0009A4312F0803F04BF4CF8043B51F8043BB3
:10F1F00016D100BF51F8044BA3F101329A4312F02B
:10F20000803FA4F101320BD14CF8043BA24312F031
:10F21000803F04BF51F8043B4CF8044BEAD023462E
:10F220000CF8013B13F0FF0F4FEA3323F8D15DF8E0
:10F23000044B704711F0010F06D011F8012B0CF8A8
:10F24000012B002A08BF704711F0020FBFD031F820
:10F25000022B12F0FF0F16BF2CF8022B8CF80020A7
:10F2600012F47F4FB3D1704711F8012B0CF8012B2A
:10F27000002AF9D1704700BF000000000000000024
:10F2800090F800F06DE9024520F007016FF0000CE6
:10F2900010F0070491F820F040F049804FF000048E
:10F2A0006FF00700D1E9002391F840F000F1080069
:10F2B00082FA4CF2A4FA8CF283FA4CF3A2FA8CF3A1
:10F2C0004BBBD1E9022382FA4CF200F10800A4FA08
:10F2D0008CF283FA4CF3A2FA8CF3E3B9D1E904235C
:10F2E00082FA4CF200F10800A4FA8CF283FA4CF393
:10F2F000A2FA8CF37BB9D1E9062301F1200182FA4D
:10F300004CF200F10800A4FA8CF283FA4CF3A2FA52
:10F310008CF3002BC6D0002A04BF04301A4612BA60
:10F32000B2FA82F2FDE8024500EBD2007047D1E963
:10F33000002304F00305C4F100004FEAC50514F0F2
:10F34000040F91F840F00CFA05F562EA05021CBFC3
:10F3500063EA050362464FF00004A9E7002A41D0A2
:10F3600040EA010313F00303F0B425D1032A23D9A3
:10F3700004680D68AC421FD1043A35D0A4F10135C0
:10F3800025EA040414F0803F31D1071D0D1D0DE066
:10F3900057F8043B0E68A3F10134B34224EA030496
:10F3A0000AD1043A20D014F0803F23D1032A294601
:10F3B000384605F10405EBD803780C789C4202F13D
:10F3C000FF320CD182B114B916E06AB17BB110F8EA
:10F3D000013F11F8014FA34202F1FF32F5D0181B93
:10F3E000F0BC7047104670471046F0BC7047184696
:10F3F000F0BC70470020F3E72046F1E72DE9F04F1D
:10F40000474C83460E46D4F800E000E026463446DA
:10F4100014F8015B0EEB0500407800F0080000F0E6
:10F42000FF080028F2D12D2D5CD02B2D04BF75785C
:10F43000B41C002B3ED0102B60D09A46B8F1000FC0
:10F440000CBF6FF000404FF000400027B0FBFAF90E
:10F45000BC460AFB19000CE0303DAB4219DD7E1CB6
:10F4600005D0CC4523D820D00AFB0C5C012714F82A
:10F47000015B0EEB0506767816F0040FECD116F062
:10F48000030606D0012E14BF57263726AD1BAB420C
:10F49000E5DC7B1C16D0B8F1000F10D16046002AC5
:10F4A00039D0DFB91160BDE8F08F8542DCDD4FF067
:10F4B000FF37DCE7302D1AD00A239A46BEE7CCF19D
:10F4C000000CEBE7B8F1000F4FF022030CBF6FF018
:10F4D00000404FF00040CBF80030F2B1611E1160E7
:10F4E000BDE8F08FB41C75784FF00108A1E72378D0
:10F4F00003F0DF03582B08D008239EE7302D9CD162
:10F50000207800F0DF00582897D14FF0100A657876
:10F510005346023492E7BDE8F08FBDE8F08F00BF9C
:10F52000C402002010B4044C13460A460146206869
:10F5300010BCFFF763BF00BF600200202DE9F04F51
:10F54000494C82460E46D4F800E000E02646344698
:10F5500014F8015B0EEB0500407800F0080000F0A5
:10F56000FF0C0028F2D12D2D54D02B2D04BF75781F
:10F57000B41C5BB1102B5ED04FF0FF38B8FBF3F832
:10F5800003FB08FB6FEA0B0B994607E0302D46D0D2
:10F590000A23DFF8D88099464FF0050B002738463C
:10F5A0000CE0303DAB4219DD7E1C05D0404522D831
:10F5B0001FD009FB0050012714F8015B0EEB050674
:10F5C000767816F0040FECD116F0030606D0012E63
:10F5D00014BF57263726AD1BAB42E5DC002F0FDBEF
:10F5E000BCF1000F00D0404242B17FB91160BDE8CC
:10F5F000F08F5D45DDDD4FF0FF37DDE7BDE8F08FD3
:10F600002223CAF800304FF0FF305AB3611E116058
:10F61000BDE8F08FB41C75784FF0010CA9E7237892
:10F6200003F0DF03582B0DD0082399464FF0070B4A
:10F630006FF06048B2E7302D0ED1207800F0DF0087
:10F64000582809D14FF0100965784B464FF00F0B41
:10F6500002346FF07048A1E74FF00F0B6FF0704865
:10F6600099469BE7BDE8F08FC4020020999999194B
:10F6700010B4044C13460A460146206810BCFFF73C
:10F680005DBF00BF6002002010B4044C13460A4660
:10F690000146206810BCF0F79FBD00BF600200204B
:10F6A000F8B50E461446054610B18369002B41D0CB
:10F6B000254B9C4243D0254B9C4242D0244B9C423C
:10F6C00008BFEC68A389A269A2601A0721D5236943
:10F6D000FBB122686169D31A8B42F7B221DA013398
:10F6E000A168501C0139A1602060167062699A42BD
:10F6F00006D0A389DB0701D50A2F01D03846F8BD13
:10F7000021462846FEF75CFE0028F7D04FF0FF3771
:10F71000F4E72146284600F025F80028F6D12369B1
:10F72000D7E721462846FEF74BFE0028EED1226897
:10F730000123D5E7FEF77EFF034B9C42BBD16C68EB
:10F74000C0E7AC68BEE700BF203F0108003F0108EA
:10F75000E03E0108024B0A4601461868FFF7A0BFC9
:10F7600060020020384B70B51D6806460C4615B186
:10F77000AB69002B42D0354B9C4245D0344B9C4268
:10F7800058D0344B9C4208BFEC68B4F90C2093B2BB
:10F7900019070CD52069A8B113F001021ED06369C6
:10F7A00000225B42A361A260F0B1002070BDDD06C3
:10F7B00042D558072AD4206942F00803A3819BB29E
:10F7C0000028E9D103F42072B2F5007FE4D030467E
:10F7D000214600F06FF8A3892069DDE7990758BF3B
:10F7E0006269A2600028E0D1B4F90C301A06DDD5B8
:10F7F00043F04003A3814FF0FF3070BD2846FEF771
:10F8000019FF124B9C42B9D16C68BEE7616B51B1D4
:10F8100004F14403994204D03046FFF721F9B4F9CA
:10F820000C200023636300232069636022F024021C
:10F830002060C1E7AC68A8E742F0400209233360CA
:10F840004FF0FF30A28170BD60020020203F010810
:10F85000003F0108E03E010870B50C46B1F90E10FA
:10F86000002990B015461E4613DB01AAF0F7C2FC32
:10F8700000280EDB029A02F47042A2F50052B2FA9E
:10F8800082F252094FF48063002032602B6010B086
:10F8900070BDA38900221B06326004D540230020DE
:10F8A0002B6010B070BD4FF4806300202B6010B04F
:10F8B00070BD00BF8A8992070B4606D501F1470249
:10F8C00001211A601A6159617047F0B583B001AB2C
:10F8D0006A460C460546FFF7BFFF009906462846D4
:10F8E000FFF704F9B4F90C30D0B1019A124F009926
:10F8F000AF6243F08003A3812060206161611AB987
:10F900003343A38103B0F0BD2846B4F90E10F0F7DD
:10F9100076FCB4F90C300028F2D043F00103EFE795
:10F920009A05EFD404F1470243F002030121A381B9
:10F93000226022616161E5E74DE400089368013BC4
:10F94000002B10B4936007DBCCB21368581C106016
:10F950001970204610BC70479469A34202DBCCB2F8
:10F960000A2CF2D110BCFFF79BBE00BF93B1F8B5D3
:10F9700014460F460646D51801E0AC4208D03A4678
:10F9800014F8011B3046FFF7D9FF431CF5D1F8BD31
:10F990000020F8BD00207047936810B5144613B9D5
:10F9A0005360184610BD00F0D1FB0023A3606360D4
:10F9B00010BD00BF2DE9F04F9DB08846144603935B
:10F9C000814618B18369002B00F00B818B4B984561
:10F9D00000F00D818A4B984500F00C81894B9845C9
:10F9E00008BFD9F80C80B8F80C301D0740F1EF8043
:10F9F000D8F81030002B00F0EA8030238DF82A3040
:10FA00002378814DDFF804A20021202209918DF88E
:10FA10002920002B00F08580252B264603D117E0F6
:10FA2000252B00F0868016F8013F002BF8D1B6EBAD
:10FA3000040B76D022465B4641464846FFF796FFC8
:10FA400001306ED0099B32785B440993002A68D05C
:10FA500000234FF0FF31721C0493079306938DF837
:10FA600053301A930591012604E0049906FA03F332
:10FA70000B430493144664482178052200F0E8FC07
:10FA8000621C431B0028F0D1049BD80644BF2022EF
:10FA90008DF853201907217844BF2B228DF853206D
:10FAA0002A2968D0A1F13002092A0BD8079B14F843
:10FAB000011F03EB830302EB4303A1F13002092A88
:10FAC000F5D907932E293FD00322504800F0C0FCFF
:10FAD00048B10499CAEB0000402202FA00F041EA62
:10FAE000000301340493217849488DF82810062238
:10FAF000013400F0ADFC00285FD0464BEBB103AB06
:10FB000000934246444B04A94846AFF300800746A1
:10FB10007A1C06D0099B3B4409932378002B7FF481
:10FB20007BAFB8F80C305B0658D409981DB0BDE81F
:10FB3000F08FB6EB040B8BD07CE7039B073323F0ED
:10FB4000070308330393E5E761782A291DD0A1F163
:10FB500030020023092A04F101040593B4D814F8F3
:10FB6000011F03EB830302EB4303A1F13002092AD7
:10FB7000F5D90593A8E7039A116804320029039286
:10FB800015DB0791617801349CE7039B1A680592A5
:10FB9000002A03F104030393B8BF4FF0FF3204F1CE
:10FBA0000203AEBFA178A17805921C468CE74942BA
:10FBB00043F0020307910493E4E703AB009342464A
:10FBC000154B04A9484600F0CDF80746A0E741468A
:10FBD0004846FFF7C7FD00283FF40FAF4FF0FF3056
:10FBE000A4E7FEF727FD054B98457FF4F3AED9F85F
:10FBF0000480F8E6D9F80880F5E600BF203F010848
:10FC0000003F0108E03E01084C4001085440010853
:10FC100058400108000000006DF9000810B4044CC1
:10FC200013460A460146206810BCFFF7C3BE00BF5A
:10FC3000600200202DE9F0470C4691460969A26850
:10FC4000DDF820808A42B8BF0A46C9F8002094F83F
:10FC5000431006461F4611B10132C9F8002023683F
:10FC600099065DD5D9F800200232C9F80020236832
:10FC700013F0060F19461DD1E1688A1A002AD8BF71
:10FC8000194617DD04F1190A002505E0E368D9F8E3
:10FC900000209B1AAB420CDD012352463946304608
:10FCA000C047013005F10105F0D14FF0FF30BDE84C
:10FCB000F087216894F84330003318BF01238A0687
:10FCC0000AD5E1185A1C302081F84300224494F8E8
:10FCD000451082F84310023304F14302394630469E
:10FCE000C0470130E1D0236803F00603042B29D07C
:10FCF000A36822699342C8BF4FF000092FDD9B1A09
:10FD000099441A34002501E04D4528D001232246AC
:10FD100039463046C047013005F10105F4D1C4E74A
:10FD200013F0060F08D1E168D9F800208A1A002ADA
:10FD3000D8BF1946A6DCBDE794F84330003318BF9E
:10FD40000123C9E7D9F80000E168A3682269091A0C
:10FD5000934221EAE179D2DCB9F1000FD1D1002040
:10FD6000BDE8F0872DE9F0430C46097E85B06E2989
:10FD7000064617460C98984604F1430C5AD01AD8F8
:10FD8000632900F0128100F2D68000295CD0582946
:10FD900040F0F58084F8451022680368DFF864E2DB
:10FDA000150603F104011ED4550653BF1B680160FC
:10FDB0001B88016019E0732900F0CF807ED86F297D
:10FDC00000F0E480702940F0DA80226842F02002DE
:10FDD0002260782384F845300368DFF82CE21506AA
:10FDE00003F10401E0D51B680160D00744BF42F075
:10FDF00020022260002B40F09080226822F0200236
:10FE000022601021002284F843206068A06000284E
:10FE1000C0F28880226822F004022260002B62D1A6
:10FE2000002840F08180654608296AD0C5EB0C03A4
:10FE300023610CE023681A0640F1D58003686269EB
:10FE4000191D01601B681A60002365462361CDF807
:10FE500000803B4603AA21463046FFF7EBFE013007
:10FE600021D02A46236939463046C04701301AD08E
:10FE70002368039813F0020FE36819D01A1A002AB6
:10FE800016DD04F11909002504E0E36803981A1A45
:10FE9000AA420DDD01234A4639463046C0470130AB
:10FEA00005F10105F1D14FF0FF3005B0BDE8F08359
:10FEB0009842B8BF184605B0BDE8F083752965D0F3
:10FEC00078295CD1226884E76168A1602D2000292F
:10FED000C3F1000384F8430021DB22F00402DFF8C1
:10FEE00024E122600A216546B3FBF1F201FB1230E6
:10FEF00013461EF8002005F8012D002BF4D1082927
:10FF000094D12368D90791D5626823699A428DDC20
:10FF1000302305F8013C013D88E7102172E7DFF846
:10FF2000E4E00A21002BDED19EF8003084F8423054
:10FF300004F1420578E7642901D069291FD12268BC
:10FF40000368150603F104013AD51B680160002B14
:10FF5000BADBDFF8B0E00A2157E703686268191DD1
:10FF600001601D680021284600F072FA002846D082
:10FF7000401B60602061002384F8433067E7012361
:10FF800084F84210236104F14205F4E723681A065D
:10FF90001ED503681A1D1B680260227EDFF864E02C
:10FFA0006F2A14BF0A2108212CE703681A68191D5B
:10FFB0000123016004F1420584F842202361DAE75D
:10FFC000550653BF1B680160B3F900300160BEE7FE
:10FFD00013F0400F036803F1040215BF02601B68B1
:10FFE0001B880260D9E713F0400F0368626903F1D0
:10FFF000040101601B6814BF1A801A6024E760685E
:020000040801F1
:10000000B8E700BF6040010874400108838903F02D
:100010000903092B01D000207047FEF703BA00BF87
:10002000F8B50C46054610B18369002B45D0424B0C
:100030009C4247D0414B9C426FD0414B9C4208BFF1
:10004000EC68B4F90C2093B200219F06616031D4B2
:100050005E0722D5616B61B104F14403994202D07D
:100060002846FEF7FDFC236C636000206063002BD4
:1000700043D12369002B52D0B4F90C70BEB2B30740
:1000800022D12269226028466369656A216AA847ED
:100090000028606009DD0020F8BDD80644D51907A6
:1000A0002ED442F00402A281E3E7A3891DD143F0DC
:1000B0002003A3814FF0FF30F8BDFEF7BBFA1E4BC3
:1000C0009C42B7D16C68BCE71E4B1F4918680123DE
:1000D000A38106F00906FEF7CDFA092EA781D0D13B
:1000E00021462846FEF7D4F8CBE7002243F0400330
:1000F000A38162604FF0FF30F8BDE36B2360F8BD71
:1001000021462846FEF75CF90028D3D1B4F90C202B
:10011000A060A06122F00802C3E7AC6891E7214625
:100120002846FFF7C7FBA7E742F0400209232B60F0
:100130004FF0FF30A281F8BD203F0108003F0108C9
:10014000E03E0108403F01080D0001089368002BC4
:1001500076D02DE9F04F8B8985B00C4619070190B8
:10016000164629D522693AB303F002081FFA88F02F
:10017000356800282FD04FF00009B44FC846B2466A
:10018000B84543464A4628BF3B460198B8F1000FA0
:1001900050D0216AA66AB047002871DDDAF808302D
:1001A0001B1A8144C0EB0808CAF80830002BE7D1BD
:1001B000002005B0BDE8F08F21460198FFF7D2FA84
:1001C000002840F03A81A389356803F002081FFA3D
:1001D00088F00028CFD113F001095BD14F46029679
:1001E0001FB39A05D4F808802CD54745C246C0F005
:1001F000A48013F4906F40F0B180206852464946C5
:10020000FEF77CFBA0682368C8EB00005344A060A5
:1002100023603846029A93681B1A81443F1A936000
:10022000002BC5D0A389002FDBD1D5F800906F68D3
:100230000835D5E7D5F80090D5F8048008359FE754
:100240000020704720682369984203D861698F4273
:1002500080F0B780B84528BFB84642464946FEF709
:100260004DFBA3682268C8EB03034244A3602260ED
:10027000002B49D121460198FEF7A2F8002843D06F
:10028000B4F90C3043F040034FF0FF30A38105B0C8
:10029000BDE8F08F8046029082468146B9F1000F9A
:1002A0002AD0029B002B4CD0206823696269C84584
:1002B000C34628BFCB4698425F4604D9A36813447F
:1002C0009B4500F39080934520DB1346A76A216A83
:1002D00001985246B847071ED2DDB8EB070823D075
:1002E000B368DB1BBA44C7EB0909B360002B3FF4CA
:1002F0005FAFB9F1000FD4D10023D5F800A0D5F835
:10030000049002930835C9E7404683E75A465146B0
:10031000FEF7F4FAA2682368CBEB02025B44B8EB69
:100320000708A2602360DBD121460198FEF748F858
:100330000028A5D1CDF80880D2E72068B846BA4693
:100340005CE74A460A21504600F082F800286FD048
:1003500001300123CAEB00080293A5E76269206817
:10036000216902EB4208C1EB000A08EBD8780AF1D8
:1003700001004FEA680838444045424684BF804641
:1003800042465B0542D511460198FEF7AFFB834616
:10039000002855D052462169FEF716FAA38923F4A6
:1003A000906343F08003A381CAEB08030BEB0A00C0
:1003B000C4F81480C4F810B02060A360B846BA46F0
:1003C0001CE76FF00043BB4228BF3B464A4693FB05
:1003D000F1F30198A66A01FB03F3216AB0470028F4
:1003E0003FF718AF4CE71A4651460393FEF786FADB
:1003F0002268039B01981A4422602146FDF7E0FF22
:10040000039B00287FF43CAF1F4666E7019800F08D
:100410006FF883460028C7D1019D21692846FEF761
:100420001FFBB4F90C300C2223F080032A6029E76B
:10043000012309F10108029336E74FF0FF30B8E6D7
:10044000019A0C231360B4F90C301BE700FCFF7F0A
:1004500001F0FF01102A2BDB10F0070F08D010F875
:10046000013B013A8B422DD010F0070F42B3F6D179
:10047000F0B441EA012141EA014122F007047FF092
:1004800000070023F0E80256083C85EA010586EAE9
:10049000010685FA47F5A3FA87F586FA47F6A5FA25
:1004A00087F68EB9EED1F0BC01F0FF0102F0070231
:1004B00032B110F8013B013A83EA010313B1F8D1DC
:1004C0000020704701387047002D06BF35460338BD
:1004D000073815F0010F07D1013015F4807F02BFF6
:1004E000013015F4C03F0130F0BC0138704700BF47
:1004F000F9B1F8B506461546B2B10C4600F01CF845
:10050000854201D82046F8BD29463046FEF7EEFA6E
:10051000074668B12A462146FEF756F9304621467D
:10052000FEF79EFA3846F8BDFEF79AFA2846F8BD5F
:10053000F8BD1146FEF7DABA51F8040C0028BEBF28
:10054000091851F8043CC018043870474E4D492032
:1005500048414E444C4552004D454D204D414E4181
:1005600047452048414E444C455200425553204691
:1005700041554C542048414E444C4552005553413E
:100580004745204641554C542048414E444C455225
:10059000004445425547204D4F4E2048414E444C63
:1005A00045520044554D4D592048414E444C45520A
:1005B000000A49535220737461636B206F76657231
:1005C000666C6F77656400537461636B20706F694C
:1005D0006E74657220636F727275707465642C201E
:1005E000726573657420746F20746F70206F66205D
:1005F000737461636B000A436F6E74657874206274
:1006000065666F726520686172646661756C743AC4
:100610000020202072303A2030782530386C780A5B
:1006200020202072313A2030782530386C780A202A
:10063000202072323A2030782530386C780A202019
:100640002072333A2030782530386C780A00202028
:100650007231323A2030782530386C780A202020E8
:100660006C723A2030782530386C780A202020705F
:10067000633A2030782530386C780A202070737205
:100680003A2030782530386C780A0A004653522FC9
:100690004641523A0020434653523A2030782530A2
:1006A000386C780A0020484653523A20307825307A
:1006B000386C780A0020444653523A20307825306E
:1006C000386C780A0020414653523A203078253061
:1006D000386C780A0020424641523A203078253062
:1006E000386C780A004D4D4641523A20307825301A
:1006F000386C780A004D697363004558435F524572
:10070000543A2030782530386C780A00417474658A
:100710006D7074696E6720746F207265636F6E739D
:10072000747275637420737461746520666F7220CF
:10073000646562756767696E672E2E2E00496E20AC
:100740004744423A0A2020736574202470633D3088
:1007500078256C780A20206672616D6520300A2049
:100760002062740A000A49535220737461636B203B
:100770006F766572666C6F7765642062792061744C
:10078000206C656173742025642062797465732E12
:100790000A0048415244204641554C542048414E9D
:1007A000444C4552004641494C4544204153534531
:1007B0005254494F4E2E0025700A002A2A2A2052F0
:1007C000494F54206B65726E656C2070616E696371
:1007D0003A0A25730A0A002A2A2A2068616C74657D
:1007E000642E0A0A006D61696E28293A20546869EE
:1007F000732069732052494F542120285665727323
:10080000696F6E3A20554E4B4E4F574E20286275F9
:10081000696C646469723A202F686F6D652F656C2E
:100820006F7065732F50464531352F52494F54290B
:10083000290A0069646C65006D61696E005F510092
:1008400069090108710901087A0901088309010889
:1008500089090108910901089A090108A3090108F9
:10086000AC090108B4090108BC090108737461747A
:1008700065006E616D650009706964207C20252D1E
:100880003231737C20252D397351207C20707269A0
:10089000207C20737461636B20202820757365644D
:1008A00029207C2062617365206164647220207C51
:1008B0002063757272656E7420202020200A000962
:1008C00020202D207C206973725F737461636B201C
:1008D00020202020202020202020207C202D2020AF
:1008E0002020202020202D207C2020202D207C2036
:1008F000253669202825356929207C20253130704E
:10090000207C20253130700A000925336869207C5D
:1009100020252D323073207C20252D387320252E64
:100920003173207C20253369207C202536692028DE
:1009300025356929207C2025313070207C20253107
:100940003070200A007C0053554D00092535732076
:10095000252D3231737C25313373253673202536AE
:10096000692028253569290A0073746F70706564E1
:1009700000736C656570696E6700626C206D7574DC
:10098000657800626C20727800626C2073656E641A
:1009900000626C207265706C7900626C20616E7907
:1009A000666C00626C20616C6C666C00626C206D21
:1009B000626F780072756E6E696E670070656E6446
:1009C000696E67000044004000000200030002401E
:1009D0000200024007070026004800400000040013
:1009E000090C0240080C0240070700270706040212
:1009F0000107070503020000003001400700024024
:100A0000060002400500024004000240050000000C
:100A10000010000001000000003800400F040240F8
:100A20000E0402400D0402400C04024005000000C8
:100A3000004000000000000000000040FFFFFFFF3A
:100A400001000000001C0000000C0040FFFFFFFF41
:100A50000800000000320000020252494F54206E8C
:100A60006574776F726B20737461636B2065786156
:100A70006D706C65206170706C69636174696F6E14
:100A800000416C6C2075702C2072756E6E696E67FB
:100A900020746865207368656C6C206E6F770075D4
:100AA00064700073656E642064617461206F7665A4
:100AB000722055445020616E64206C697374656EB9
:100AC000206F6E2055445020706F727473000000C8
:100AD0009F0A0108A30A0108C118000800000000CD
:100AE000000000000000000075736167653A202572
:100AF00073205B73656E647C7365727665725D0AE4
:100B00000075736167653A2025732073656E6420F4
:100B10003C616464723E203C706F72743E203C64A1
:100B20006174613E205B3C6E756D3E205B3C64658C
:100B30006C617920696E2075733E5D5D0A004572B7
:100B4000726F723A20756E61626C6520746F2070EE
:100B5000617273652064657374696E6174696F6E28
:100B60002061646472657373004572726F723A201B
:100B7000756E61626C6520746F20706172736520A0
:100B800064657374696E6174696F6E20706F7274DE
:100B9000004572726F723A20756E61626C652074E6
:100BA0006F20636F7079206461746120746F2070AE
:100BB00061636B657420627566666572004572726A
:100BC0006F723A20756E61626C6520746F20616C83
:100BD0006C6F63617465205544502068656164657D
:100BE00072004572726F723A20756E61626C652098
:100BF000746F20616C6C6F63617465204950763648
:100C000020686561646572004572726F723A207582
:100C10006E61626C6520746F206C6F636174652017
:100C20005544502074687265616400537563636550
:100C300073733A2073656E7420257520627974652C
:100C400028732920746F205B25735D3A25750A008F
:100C500075736167653A20257320736572766572D6
:100C6000205B73746172747C73746F705D0A0073BF
:100C700074617274007573616765202573207365F4
:100C800072766572207374617274203C706F727436
:100C90003E0A004572726F723A2073657276657211
:100CA00020616C72656164792072756E6E696E6721
:100CB000206F6E20706F727420256C750A0045726B
:100CC000726F723A20696E76616C696420706F721F
:100CD0007420737065636966696564005375636346
:100CE0006573733A2073746172746564205544505F
:100CF00020736572766572206F6E20706F7274203B
:100D00002568750A0073746F70004572726F723ACD
:100D10002073657276657220776173206E6F742020
:100D200072756E6E696E670A0053756363657373DF
:100D30003A2073746F707065642055445020736559
:100D400072766572006572726F723A20696E7661B2
:100D50006C696420636F6D6D616E6400010000005A
:100D600003000000060C0240050C0240070C024084
:100D70000A0C02405B6175746F5F696E69745F6E27
:100D8000657469665D206572726F7220696E697440
:100D900069616C697A696E6720617438367266328F
:100DA000787820726164696F202325750A00617468
:100DB00038367266327878006970763600293A11D2
:100DC000676E72635F6E65746465763A20706F73E8
:100DD0007369626C79206C6F737420696E746572CC
:100DE000727570742E007E7E20534E49502025323D
:100DF00069202D2073697A653A2025337520627940
:100E000074652C20747970653A20004E455454590D
:100E100050455F554E44454620282569290A004E15
:100E20004554545950455F4E45544946202825693C
:100E3000290A004E4554545950455F5349584C4F68
:100E40005750414E20282569290A004E45545459CF
:100E500050455F4950563620282569290A004E45DD
:100E600054545950455F49434D5056362028256902
:100E7000290A004E4554545950455F554450202886
:100E80002569290A004E4554545950455F554E4B2B
:100E90004E4F574E20282569290A007E7E20504B50
:100EA00054202020202D2025326920736E69707314
:100EB0002C20746F74616C2073697A653A20253335
:100EC0006920627974650A00504B5444554D503A7C
:100ED00020646174612072656365697665643A00B7
:100EE000504B5444554D503A206461746120746FE6
:100EF0002073656E643A00504B5444554D503A206F
:100F0000726563656976656420736F6D6574686981
:100F10006E6720756E657870656374656400706BCC
:100F20007464756D7000FF02000000000000000096
:100F300000000000001A52504C0001020000366C04
:100F40006F00FF7F3F1F0F0703012020207479707F
:100F5000653A2025336868752020636F64653A2000
:100F600025336868750A00202020636B73756D3A1D
:100F700020307825303468780A00FFFFFE800000BA
:100F8000000000000000000000000000FF01000061
:100F9000000000000000000000000001FF0200004F
:100FA000000000000000000000000001FF0200003F
:100FB000000000000000000000000002FF0200002E
:100FC0000000000000000001FF0000000000000021
:100FD0000000000000000000000000000000000011
:100FE000000000000000000000000001303132333A
:100FF00034353637383961626364656600303132C2
:101000003334353637383941424344454600696CFC
:101010006C6567616C2076657273696F6E206669B6
:10102000656C643A20256868750A007472616666AA
:10103000696320636C6173733A20307825303278AD
:10104000202845434E3A20307825782C20445343BD
:10105000503A20307825303278290A00666C6F7754
:10106000206C6162656C3A2030782530356C780AE6
:10107000006C656E6774683A2025687520206E657F
:101080007874206865616465723A2025752020684F
:101090006F70206C696D69743A2025750A00736F52
:1010A0007572636520616464726573733A20257399
:1010B0000A0064657374696E6174696F6E2061649F
:1010C00064726573733A2025730A00303030303013
:1010D000303030007368656C6C3A20696E636F72F3
:1010E000726563742071756F74696E670068656CF2
:1010F00070004465736372697074696F6E00436F4A
:101100006D6D616E6400252D3230732025730A00E9
:101110007368656C6C3A20636F6D6D616E64206EF0
:101120006F7420666F756E643A2025730A007265CD
:10113000626F6F74005265626F6F7420746865200F
:101140006E6F6465007073005072696E747320690D
:101150006E666F726D6174696F6E2061626F757417
:101160002072756E6E696E67207468726561647353
:101170002E0070696E67360050696E67207669616F
:101180002049434D5076360072616E646F6D5F6921
:101190006E697400696E697469616C697A6573203F
:1011A0007468652050524E470072616E646F6D5FC7
:1011B0006765740072657475726E732033322062D5
:1011C0006974206F662070736575646F2072616E3C
:1011D000646F6D6E657373006966636F6E666967D1
:1011E00000436F6E666967757265206E6574776F10
:1011F000726B20696E7465726661636573006669FF
:1012000062726F757465004D616E6970756C6174A2
:101210006520746865204649422028696E666F3AE9
:101220002027666962726F757465205B6164647CF7
:1012300064656C5D2729006E6361636865006D619C
:101240006E616765206E65696768626F72206361B1
:101250006368652062792068616E6400726F7574DE
:1012600065727300495076362064656661756C74EA
:1012700020726F75746572206C6973740072706C83
:101280000072706C20636F6E666967757261746955
:101290006F6E20746F6F6C20282772706C206865E9
:1012A0006C702720666F72206D6F726520696E66A4
:1012B0006F726D6174696F6E290000002E11010854
:1012C00035110108D991000845110108481101089C
:1012D000E3910008721101087811010851AC00086F
:1012E0008811010894110108ED910008A911010865
:1012F000B411010825920008D8110108E111010874
:10130000119B0008FE1101080712010881A50008C1
:10131000371201083E12010869A800085C12010892
:101320006412010865AA00087D12010881120108F3
:101330002DB50008000000000000000000000000C3
:1013400050524E4720696E697469616C697A6564B0
:1013500020746F2063757272656E742074696D6598
:101360003A2025640A0050524E4720696E6974691C
:10137000616C697A656420676976656E2076616C58
:1013800075653A2025640A004F464600534C454592
:1013900050005354414E4442590049444C45005278
:1013A00058005458005245534554002530387800B1
:1013B0002873686F727429206164647265737300A6
:1013C0006C6F6E67206164647265737300736F7510
:1013D0007263652061646472657373206C656E6707
:1013E0007468006368616E6E656C007061676500AB
:1013F0006E6574776F726B206964656E7469666977
:10140000657200545820706F776572205B696E209A
:1014100064426D5D006D61782E2072657472616E3C
:10142000736D697373696F6E730043534D4120721E
:101430006574726965730043434120746872657313
:10144000686F6C64205B696E2064426D5D00656E40
:101450006372797074696F6E00656E63727970740F
:10146000696F6E206B65790075736167653A202539
:1014700073203C69665F69643E20736574203C6B31
:1014800065793E203C76616C75653E0A002020201F
:101490002020205365747320616E20686172647728
:1014A0006172652073706563696669632073706536
:1014B00063696669632076616C75650A2020202067
:1014C00020203C6B65793E206D6179206265206F3C
:1014D0006E65206F662074686520666F6C6C6F7730
:1014E000696E670A202020202020202A20226164A3
:1014F000647222202D2073657473202873686F72C4
:10150000742920616464726573730A20202020208E
:1015100020202A2022616464725F6C6F6E67222033
:101520002D2073657473206C6F6E67206164647224
:101530006573730A202020202020202A2022616445
:1015400064725F73686F727422202D20616C696110
:101550007320666F72202261646472220A20202048
:10156000202020202A20226368616E6E656C222074
:101570002D207365747320746865206672657175BB
:10158000656E6379206368616E6E656C0A20202049
:10159000202020202A20226368616E22202D2061D5
:1015A0006C69617320666F7220226368616E6E657C
:1015B0006C220A202020202020202A202263736D04
:1015C000615F7265747269657322202D2073657482
:1015D000206D61782E206E756D626572206F6620B9
:1015E0006368616E6E656C2061636365737320610F
:1015F0007474656D7074730A202020202020202AC6
:1016000020226363615F7468726573686F6C642223
:10161000202D2073657420454420746872657368BA
:101620006F6C6420647572696E6720434341206962
:101630006E2064426D0A202020202020202A2022B3
:101640006E696422202D2073657473207468652090
:101650006E6574776F726B206964656E7469666914
:10166000657220286F72207468652050414E2049B1
:1016700044290A202020202020202A20227061676F
:101680006522202D2073657420746865206368616D
:101690006E6E656C20706167652028494545452060
:1016A0003830322E31352E34290A202020202020B7
:1016B000202A202270616E22202D20616C696173C6
:1016C00020666F7220226E6964220A20202020206A
:1016D00020202A202270616E5F696422202D206103
:1016E0006C69617320666F7220226E6964220A2021
:1016F0002020202020202A2022706F77657222204F
:101700002D20545820706F77657220696E206442D6
:101710006D0A202020202020202A20227265747249
:10172000616E7322202D206D61782E206E756D62A2
:101730006572206F662072657472616E736D697375
:1017400073696F6E730A202020202020202A202217
:101750007372635F6C656E22202D20736574732035
:1017600074686520736F7572636520616464726567
:101770007373206C656E67746820696E206279747B
:10178000650A202020202020202A202273746174E2
:101790006522202D20736574207468652064657649
:1017A0006963652073746174650A202020202020FD
:1017B000202A2022656E637279707422202D207396
:1017C00065742074686520656E6372797074696FE2
:1017D0006E206F6E2D6F66660A202020202020204C
:1017E0002A20226B657922202D207365742074686D
:1017F0006520656E6372797074696F6E206B6579B0
:1018000020696E2068657861646563696D616C202C
:10181000666F726D61740A00756E006572726F7228
:101820003A20756E61626C6520746F207365742058
:101830006F7074696F6E00737563636573733A20BC
:101840002573736574206F7074696F6E0A0065721A
:10185000726F723A20756E61626C6520746F2070D1
:101860006172736520616464726573732E0A4D75CD
:101870007374206265206F6620666F726D617420DC
:101880005B302D39612D66412D465D7B327D283AD6
:101890005B302D39612D66412D465D7B327D292AD5
:1018A0000A286865782070616972732064656C69C4
:1018B0006D6974656420627920636F6C6F6E732943
:1018C000006572726F723A20756E61626C65207489
:1018D0006F207365742000737563636573733A20BA
:1018E0007365742000206F6E20696E746572666186
:1018F00063652025686920746F2025730A00206FB6
:101900006E20696E74657266616365202568692062
:10191000746F2025690A006572726F723A20756EC5
:1019200061626C6520746F207061727365207661EE
:101930006C75652E0A4D75737420626520612031C7
:10194000362D62697420756E7369676E65642069EF
:101950006E74656765722028646563206F72206805
:101960006578290A00206F6E20696E746572666161
:1019700063652025686920746F2000307825303435
:10198000780A004C61796572203200495076360041
:10199000616C6C00556E6B6E6F776E00202020209E
:1019A0002020202020202050726F746F636F6C20E5
:1019B0006F722064657669636520646F65736E2756
:1019C000742070726F7669646520737461746973D2
:1019D000746963732E005265736574207374617447
:1019E00069737469637320666F72206D6F64756CC0
:1019F00065202573210A002020202020202020207F
:101A000020205374617469737469637320666F7204
:101A10002025730A20202020202020202020202084
:101A20005258207061636B657473202575202062A5
:101A3000797465732025750A20202020202020201D
:101A4000202020205458207061636B65747320251A
:101A50007520284D756C7469636173743A2025751F
:101A600029202062797465732025750A20202020A2
:101A70002020202020202020545820737563636587
:101A800065646564202575206572726F7273202508
:101A9000750A00776972656400776972656C6573B1
:101AA000730049666163652025326420200020436D
:101AB00068616E6E656C3A20256875200020506163
:101AC00067653A202568752000204E49443A203049
:101AD00078256878004C6F6E67204857616464729F
:101AE0003A2000257320000A2020202020202020DA
:101AF0002020002054582D506F7765723A202568B9
:101B00006964426D20002053746174653A2000209E
:101B10006D61782E2052657472616E732E3A2025A5
:101B20007520002043534D412052657472696573DE
:101B30003A202575200050524F4D49534320200034
:101B40004155544F41434B20200041434B5F524588
:101B5000512020005052454C4F414420200052411A
:101B6000574D4F444520200043534D412020004114
:101B700055544F4343412020004D41435F4E4F5F3A
:101B8000534C4545502020004D54553A256875204A
:101B90002000484C3A2575202000364C4F2020006C
:101BA0005254522020005254525F4144562020008B
:101BB00049504843202000536F757263652061646B
:101BC0006472657373206C656E6774683A2025686B
:101BD000750A2020202020202020202020004C6971
:101BE0006E6B20747970653A20257300696E657498
:101BF0003620616464723A200025732F25752020F9
